:100000000C94A7040C94CF040C94CF040C94CF044C
:100010000C94CF040C94CF040C94CF040C94CF0414
:100020000C94CF040C94CF040C944C260C94CF0465
:100030000C94CF040C94CF040C94CF040C94CF04F4
:100040000C945B090C94CF040C94CF040C94CF0453
:100050000C94CF040C94CF040C94CF040C9430096E
:100060000C94CF040C94CF040C94CF040C94CF04C4
:100070000C94CF040C94CF040C94CF040C94CF04B4
:100080000C945B100C94CF040C94CF040C94CF040C
:100090000C94CF040C94CF040D0A416C6C206E6F4D
:1000A000646573202D20287229656164696E672C50
:1000B0002028702970696E673A000D0A50617573C7
:1000C00065642C2070726573732027502720746F2D
:1000D00020756E7061757365000D0A57616B652040
:1000E0007768696368206E6F64653A000D0A53741F
:1000F00061727475702C204920616D20636F6F727E
:1001000064696E61746F722E0D0A000D0A456E747B
:100110006572206E65772050414E4944000D0A45B6
:100120006E746572206E6577206368616E000D0ADB
:1001300053747265616D206D6F646520746F20610A
:100140006464723A000D0A456E7465722073686FBC
:10015000727420616464723A000D0A006E6F74203C
:100160007965742076616C6964000D0A49507636B1
:1001700020364C4F5750414E204946203D20006EBE
:100180006F74207965742076616C6964000D0A498A
:100190005076362045746865726E65742049462035
:1001A0003D2000506172743D524600556E6B6E6F7B
:1001B000776E3F00425553595F52585F4141434B60
:1001C0005F4E4F434C4B0052585F4141434B5F4F92
:1001D0004E5F4E4F434C4B0052585F4F4E5F4E4F59
:1001E000434C4B0054585F415245545F4F4E0052B0
:1001F000585F4141434B5F4F4E00425553595F5446
:10020000585F4152455400425553595F52585F411F
:1002100041434B00504C4C5F4F4E005452585F4F7F
:1002200046460052585F4F4E00425553595F54584E
:1002300000425553595F525800505F4F4E00526173
:1002400064696F205374617465203D200050414EF5
:10025000204944203D203078000D0A723D726561CE
:1002600064696E67206E3D6E616D6520773D7761D4
:100270006B6520503D70617573653A20000D0A640E
:100280003D64756D7020743D7461626C6520693DDC
:10029000696E666F20703D70696E6720733D737480
:1002A0007265616D20633D6368616E000D0A50697F
:1002B0006E67696E67206E6F646520000D0A4E6F71
:1002C000726D616C206D6F6465000D0A537461720C
:1002D0007475702C204920616D20636F6F726469A2
:1002E0006E61746F72206F6E20636820002C20682E
:1002F0006F7073203D2000206F6E20636820000D1A
:100300000A4173736F63696174696E6720746F204B
:10031000000D0A000D0A0D0A5245472044554D5064
:100320000D0A0020525353493D00204C51493D00D5
:100330000D0A50696E6720726573706F6E73652069
:1003400066726F6D20000D0A50696E6720726571CC
:10035000756573742066726F6D206E6F6465200022
:100360002066726F6D20706172656E7420000D0AD8
:1003700044726F7070696E67206368696C642000F6
:100380000D0A0020202020202020202020202020B6
:10039000202020202020202020202020202020205D
:1003A00020000D0A0D0A2020204C6F6E672041644A
:1003B000647220202020202053686F7274204164D2
:1003C000647220202020202020495076362041646D
:1003D00064720D0A0020202020000D0A000D0A4E34
:1003E0006574776F726B20547265650D0A000D0A93
:1003F0005461626C6520446174613A0D0A000D0A13
:100400004261642064657374206E6F6465202852B5
:100410005029000D0A0020486F7073203D20000D08
:100420000A4173736F636961746564206E6F6465FC
:1004300020000D0A526F7574652064617461206636
:10044000726F6D20436F6F7264000D0A526F757486
:1004500065206461746120746F206368696C640056
:100460001201000202000040EB03182000100102FC
:100470000301090243000201008032090400000167
:1004800002020100052400100105240103010424D7
:1004900002060524060001070584032000FF090465
:1004A0000100020A00000007058502200000070580
:1004B000060220000012010002EF020140EB0322BD
:1004C00020001001020301090264000301008032D0
:1004D000080B00020202FF0009040000010202FFF3
:1004E0000005240010010524010001042402000578
:1004F0002406000107058303080010090401000217
:100500000A000000070581024000000705020240C2
:10051000000009040200010300000009211101008C
:10052000012235000705840320001006FFFF0901A2
:10053000A10109020903150026FF00750895208115
:100540000209040905150026FF007508952091028F
:1005500009060907150026FF0075089504B102C0B9
:10056000120100020202FF40EB03192000100102F9
:100570000301090243000201008032090400000166
:100580000202FF00052400100105240100010424DB
:100590000200052406000107058303080010090472
:1005A0000100020A00000007058102400000070563
:1005B000020240000012010002020C0740EB03227D
:1005C00020001001020301090239000201008032FB
:1005D0000904000002020C07000705810240000028
:1005E00007050202400000090401000103000000A9
:1005F00009211101000122350007058303200010A5
:100600000C03410054004D0045004C002403410000
:1006100056005200200055005300420020005200B6
:1006200055004D00200043004F004F005200440091
:10063000040309040D0A52657374617274696E676C
:10064000204D41432026204E574B0D0A000D0A52E3
:10065000657374617274204D41432E0D0A000D0ABA
:1006600052657374617274204D41432E0D0A00016E
:100670000101000201010003010100040101000663
:10068000010100070101000A0101000B0101000C3A
:100690000101000D0101000E010100110101001412
:1006A0000101001601010002020100010102000225
:1006B0000102000301020004010200050102001B07
:1006C0000201000101010102010101030101010414
:1006D0000101010501010101010201020102010301
:1006E000010201000101FD020101FD010101FD0600
:1006F0000101FD030101FD040101FD50414E49448A
:100700003A203078424141440041746D656C0000EC
:100710000000000D0A004E756D6265720909537480
:100720006174650909495020416464726573730DF1
:100730000A00736963736C6F7770616E20756E6306
:100740006F6D70726573735F6864723A2065727260
:100750006F7220756E737570706F7274656420555A
:10076000445020636F6D7072657373696F6E0D0A0C
:1007700000736963736C6F7770616E20756E636F61
:100780006D70726573735F6864723A206572726F20
:100790007220636F6E74657874206E6F7420666F5C
:1007A000756E640D0A00736963736C6F7770616EA8
:1007B00020756E636F6D70726573735F6864723AF3
:1007C000206572726F7220756E6B6E6F776E20632C
:1007D0006F6D70726573736564206D6361737420EF
:1007E000616464726573730D0A00736963736C6F7F
:1007F0007770616E20756E636F6D70726573735F75
:100800006864723A206572726F7220636F6E7465ED
:100810007874206E6F7420666F756E640D0A0073B5
:100820006963736C6F7770616E20756E636F6D7046
:10083000726573735F6864723A206572726F7220BA
:10084000636F6E74657874206E6F7420666F756E5A
:10085000640D0A00736963736C6F7770616E207545
:100860006E636F6D70726573735F6864723A206552
:1008700072726F7220636F6E74657874206E6F741D
:1008800020666F756E640D0A00736963736C6F7711
:1008900070616E20756E636F6D70726573735F68E3
:1008A00064723A206572726F7220756E6B6E6F772C
:1008B0006E20636F6D70726573736564206D636124
:1008C000737420616464726573730D0A00736963E5
:1008D000736C6F7770616E20756E636F6D7072658B
:1008E00073735F6864723A206572726F7220636F0F
:1008F0006E74657874206E6F7420666F756E640D0B
:100900000A00736963736C6F7770616E20756E6334
:100910006F6D70726573735F6864723A206572728E
:100920006F7220636F6E74657874206E6F742066CA
:100930006F756E640D0A0045464765666700202B9B
:100940002D2E3031323334353637383968001124A2
:100950001FBECFEFD0E2DEBFCDBF14BE88E10FB621
:10096000F89480936000109260000FBE15E0A0E044
:10097000B1E0EAE7F7E001E00BBF02C007900D929B
:10098000A63CB107D9F71CE1A6ECB5E001C01D9269
:10099000A13EB107E1F70E942B080C94EA740C9475
:1009A000000080910F11089580E01C9981E0089566
:1009B0002D982C988DE090E00197F1F72D9A0895ED
:1009C00008950895089581E06FE140E00E94950A3E
:1009D00008950E94E304282F8151823058F022307C
:1009E00049F0213039F080E090E02E3129F481E0A7
:1009F00090E0089581E090E00895CF93DF93EC01BB
:100A00000E94E304863021F0813011F084E407C0B5
:100A100086E06FE140E00E94950A888380E4DF91E0
:100A2000CF91089583E067E040E00E94950A089521
:100A300081E160E245E00E94950A882311F08BE491
:100A400008958AE4089581E160E144E00E94950AF6
:100A5000089581E16FE040E00E94950A089589E0E1
:100A60006FE040E00E94950A089588E060E645E066
:100A70000E94950A089585E06FE040E00E94950A83
:100A8000089588E06FE140E00E94950A089586E0AD
:100A90006FE140E00E94950A8093C7051092AA1169
:100AA00008951F93CF93DF93EC0114E26991812F96
:100AB0000E94300A1F5F1C32C9F7DF91CF911F914E
:100AC00008951F93682F192F80E20E94300A81E257
:100AD000612F0E94300A1F9108951F93682F192FCC
:100AE00082E20E94300A83E2612F0E94300A1F9145
:100AF0000895282F8EE268E043E00E94760A089568
:100B00002C988DE090E00197F1F782E06FE140E0F2
:100B100023E00E94760A83E090E00197F1F70895C0
:100B20000E94D404882311F080E408950E94800577
:100B30008BE490E00197F1F70E94E304883011F014
:100B400083E408952C9A80E408951F93162F66304D
:100B500010F082E414C0882329F483E068E043E0C5
:100B600021E004C083E068E043E020E00E94760AD0
:100B700083E067E040E0212F0E94760A80E41F9125
:100B800008950E94D404882379F02C9881EE96E091
:100B90000197F1F781E060E00E94A5050E94E3045F
:100BA000883011F083E4089580E408950F931F9333
:100BB000182F062F603110F082E41AC00E94D4046E
:100BC000882311F084E414C0112329F081E160E14D
:100BD00044E021E004C081E160E144E020E00E94C3
:100BE000760A81E16FE040E0202F0E94760A80E4DF
:100BF0001F910F9108951F93182F803110F082E4F8
:100C00000DC00E94D404882311F084E407C085E05D
:100C10006FE040E0212F0E94760A80E41F91089542
:100C20001F93182F8B50803110F082E421C00E9456
:100C3000D404882311F084E41BC00E94410581176D
:100C4000B1F088E06FE140E0212F0E94760A0E9417
:100C5000E304863011F0893021F48DE291E00197B0
:100C6000F1F70E944105811711F083E401C080E48F
:100C70001F9108958091C605882329F48CE10E9474
:100C80005C0A8093C6058091C6050895FF920F9374
:100C90001F93082F0E94E304182F0E943A06833006
:100CA00021F00E943A068730B1F4163029F4F02E74
:100CB000F69410E000E00CC0163169F4F8CF86E03D
:100CC00060E645E00E94950A110F110F182B0F5F87
:100CD0000F15A8F303C00E945080182F812F1F9179
:100CE0000F91FF9008951F93182F0E943A068230AB
:100CF00031F485E060E847E0212F0E94760A0E94E7
:100D00003A06833031F484E060E245E0212F0E940E
:100D1000760A1F9108950F931F93182F883051F072
:100D2000863041F0893031F0863121F0893111F07F
:100D300082E455C00E94D404882311F084E44FC09B
:100D40000E94E9048823E1F70E943A06823039F4D0
:100D50000E94E40C882319F0163109F416E00E9471
:100D6000E304082F1817D1F1183019F40E948005F8
:100D70002FC0193159F48930E1F082E06FE140E091
:100D800029E00E94760A063181F40CC0163189F4FC
:100D9000893079F082E06FE140E029E00E94760A34
:100DA000093119F483E090E002C089E691E00197EF
:100DB000F1F782E06FE140E0212F0E94760A0830CF
:100DC00019F489E691E002C083E090E00197F1F721
:100DD0000E94E304811711F083E401C080E41F91B5
:100DE0000F910895FF920F931F93DF93CF9300D03D
:100DF0000F92CDB7DEB7F82E8B019091AC11892FF1
:100E00008250823010F484E430C0992389F0CB0101
:100E10006F2D40E02BE934E10E944A25882341F000
:100E20008AE189831B821A82CE0101960E94B30B4C
:100E3000F7FE02C082E419C00E94E9048823E1F7AA
:100E400089E10E948B060E94E3048931C9F7F80109
:100E5000858196819093A9118093A811F2E0FF0EED
:100E6000C8016F2D0E94E30980E40F900F900F904E
:100E7000CF91DF911F910F91FF900895DF93CF9352
:100E800000D000D00F92CDB7DEB70E94E3048A8372
:100E90008A81813151F08A81863039F08A818130AE
:100EA00021F08A81863109F071C08091AC118823CC
:100EB00031F41D821C821B820E94F50920C0833000
:100EC00009F496C0813079F40E94F50981E090E040
:100ED0009D838C838AE18B83CE0103960E94B30BA2
:100EE0001D821C820CC08BE994E10E94A3258823FB
:100EF00009F47EC08AE18B831D821C8242C09091DE
:100F0000911080E020919010AC01420F511D9A0188
:100F10005093911040939010809195108F3F41F421
:100F2000809196108F3F21F4842F807F09F060C05C
:100F30001B8258E821363507E1F088E82236380769
:100F400040F448E02330340761F020503048C9F4C1
:100F50000AC088E82336380771F02356384C89F4E4
:100F60000EC085E10DC00E94E40C882351F084E19D
:100F700007C080E105C080919910813011F487E1AC
:100F80008B83CE0103960E94B30B32C08A818230DC
:100F900049F08A81823131F08A81893119F08A8160
:100FA000893031F51092AA111B821D821C8282E0C9
:100FB00060EE45E00E94950A89838981833051F073
:100FC000843018F4823050F403C0853039F404C002
:100FD00081E103C083E101C082E18B838B8188239F
:100FE00021F0CE0103960E94B30B86E10E948B068E
:100FF0000F900F900F900F900F90CF91DF91089569
:101000000E943A06823011F486E108958091C70566
:1010100008950F931F930DEF13E0C8010197F1F7A7
:101020000E94BF090E94D80482E06FE140E023E003
:101030000E94760AC8010197F1F78EE06CE00E94E9
:10104000300A89E06FE040E027E00E94760A80E401
:101050001F910F91089510926400109265000E94F4
:101060007F0880E880936100109261008DB18760F5
:101070008DB98EB183608EB98FEF87B981B980E069
:1010800090E00E949F0B0E949F100E942A270E94BE
:1010900045270E94B86A0E94BB1878940E940A14DF
:1010A0000E94FF0B0E9427270E948A280E94A735D2
:1010B000F4CF9C01F999FECF32BD21BDF89A80B5DD
:1010C00008959C01F999FECF1FBA32BD21BD60BDC4
:1010D0000FB6F894FA9AF99A0FBE089584B1866013
:1010E00084B9299A209A289A80E58CBD81E08DBD2B
:1010F00008958EBD0DB407FEFDCF8EB508950895F9
:101100009C01CB01B90121E638E00E94EC800895F2
:10111000DF93CF930F92CDB7DEB7FC01362FCA0114
:101120002FB72983F894BF01432F50E00E94800815
:1011300089818FBF0F90CF91DF91089529E538E025
:101140000E94D0800895DF93CF930F92CDB7DEB782
:10115000FC01362FCA012FB72983F894BF01432F12
:1011600050E00E949E0889818FBF0F90CF91DF9140
:101170000895DF92EF92FF920F931F93DF93CF9327
:1011800000D0CDB7DEB78091C805882311F011E0FB
:101190005CC081E08093C805D0906600F89461E05F
:1011A0000E94A505E090B100F090810000918000C0
:1011B0001092B100109281001092800020E030E087
:1011C00063E056E04FEF6093B100509381001092BE
:1011D000B200109285001092840046BB47BBB89BBA
:1011E000FECF80918400909185009A83898310922C
:1011F00081001092B10089819A818A5F934020F426
:101200008091660081500AC089819A8186509440FD
:1012100010F411E00CC0809166008F5F809366002F
:101220002F5F3F4F83E0283E380769F610E081E0EA
:1012300060E00E94A505E092B100F0928100009369
:101240008000112311F4D0926600812F0F900F902F
:10125000CF91DF911F910F91FF90EF90DF90089554
:101260001F920F920FB60F920BB60F9211242F936D
:101270003F934F935F936F937F938F939F93AF931E
:10128000BF93EF93FF9385B58D7F85BD0E94FF0CC3
:10129000FF91EF91BF91AF919F918F917F916F914E
:1012A0005F914F913F912F910F900BBE0F900FBE0A
:1012B0000F901F9018951F920F920FB60F920BB6BA
:1012C0000F9211240F931F932F933F934F935F938C
:1012D0006F937F938F939F93AF93BF93EF93FF93FE
:1012E0008FE00E945C0A082F182F83FF02C00E9423
:1012F0003E0714FF02C00E94FF0C12FF10C0289886
:1013000080E28EBD0DB407FEFDCF8EB51EBC0DB4C0
:1013100007FEFDCF8EB5289A0E9447050AC007FF39
:1013200008C08EE00E945C0A682F6F778EE00E94F2
:10133000300AFF91EF91BF91AF919F918F917F9173
:101340006F915F914F913F912F911F910F910F904E
:101350000BBE0F900FBE0F901F901895249A259AE0
:101360000E94BC09EFE6F0E080818062808383E424
:1013700080938100B59A08950E946E0808950E9496
:10138000AE090E94BC09EFE6F0E0808180628083B4
:1013900083E480938100B59A08951F93CF93DF93E0
:1013A000EC01162F289880E60E947908812F0E9470
:1013B000790889910E9479081150D9F7289ADF910C
:1013C000CF911F910895DF93CF930F92CDB7DEB7E2
:1013D0002FB72983F8942C9A2C980E94CD098981E3
:1013E0008FBF0F90CF91DF910895EF92FF921F93DF
:1013F000DF93CF930F92CDB7DEB78FB78983F89481
:10140000289880E20E94790880E00E947908182FCD
:1014100083508D37A8F410938F1080E9E82E80E177
:10142000F82E80E00E947908F70181937F01115026
:10143000C1F780E00E94790880930F11289A07C0B5
:10144000289A10928F1010920F111092101189810A
:101450008FBF0F90CF91DF911F91FF90EF90089574
:101460000F931F93DF93CF930F92CDB7DEB7062F65
:10147000182F106C8FB78983F8942898812F0E94B9
:101480007908802F0E947908289A89818FBF1F735D
:10149000123061F4602F6F71663011F0663121F403
:1014A00081E08093650F02C01092650F0F90CF917D
:1014B000DF911F910F9108951F93DF93CF930F92A8
:1014C000CDB7DEB7182F10688FB78983F8942898A6
:1014D000812F0E947908812F0E947908289A99818A
:1014E0009FBF0F90CF91DF911F910895DF92EF92F0
:1014F000FF920F931F93D82EF62EE42E022F0E94F8
:101500005C0A6F2D6095682310E002C0000F111F68
:10151000EA94E2F7F0226F298D2D0E94300A1F9184
:101520000F91FF90EF90DF900895FF920F931F931C
:10153000062FF42E0E945C0A082310E002C01595C5
:101540000795FA94E2F7802F1F910F91FF9008956D
:10155000FC011182818180830895DC0111969C91A8
:101560001197FD01E90FF11D22818C91981711F45B
:101570002FEF06C0892F8F5F87FD80E011968C9337
:10158000822F0895FC019081818120E0981321E051
:10159000822F0895FC018081282F30E08181281B53
:1015A000310937FF02C020583F4F822F0895089518
:1015B00086E69FE00E94CA0A089586E69FE00E94A0
:1015C000CA0A08958CEE9FE00E94CA0A08958CEE24
:1015D0009FE00E94AD0A089590E08091C90588239C
:1015E00009F491E09093C905089580E00895089565
:1015F00004C00E9427270E948A2886E69FE00E9456
:10160000CA0A8823B1F386E69FE00E94AD0A0895D6
:101610000F931F93CF93DF93EC01062F18811F5F69
:1016200017FF12C010E010C080916E108823A9F43B
:1016300080910B05813021F080910C05882369F0A1
:101640000E9427270E948A288981181769F38881B8
:10165000FE01E80FF11D02831883DF91CF911F91E6
:101660000F910895682F81E080936E1086E69FE0C9
:101670000E94080B10926E100895682F8091C90582
:10168000882329F478948CEE9FE00E94080B08953B
:10169000DF92EF92FF920F931F93CF93DF93EC01B2
:1016A000D42E00E0E62EFF240894E108F1080E9401
:1016B000F80A182F802F90E08E159F0534F01D300A
:1016C00021F01A3011F0183091F7DD2019F0812F38
:1016D0000E943D0B1A3029F01D3019F0183089F4A2
:1016E0000AC01882802FDF91CF911F910F91FF9038
:1016F000EF90DF9008950023D1F2015018822197D6
:10170000D6CF19930F5FD3CFCF93DF93EC0102C0F5
:101710000E943D0BFE01219684918823C9F7DF9139
:10172000CF910895CF93DF93EC0103C00E943D0B4E
:10173000219688818823D1F7DF91CF91089586E69D
:101740009FE00E94A80A8CEE9FE00E94A80A0E94D7
:101750000B29089590916F108091701020E09813DC
:1017600021E0822F08950F931F93482F192F009186
:101770006F10E02FF0E020917010CF0101966AE029
:1017800070E00E941A8330E082179307B9F0DF01FE
:10179000AA0FBB1FAE0FBF1FAF58BF4E842F912F94
:1017A0009C01F90183E001900D928150E1F7802FB7
:1017B0008F5F8A3008F080E080936F101F910F9147
:1017C0000895DF93CF930F92CDB7DEB7809170105D
:1017D0008983998189818F5F898389818A3008F023
:1017E000198289818093701023E0929F90011124C7
:1017F0002F583F4EC9010F90CF91DF91089558C0E7
:101800000E94E10BFC0180818431D1F0853178F4B4
:10181000813109F446C0823120F4803109F048C09A
:101820001BC08231D9F1833109F042C034C0863106
:1018300071F0863150F1873159F18A31C9F534C0E0
:1018400080919B118823A1F50E94ED0C31C001808D
:10185000F281E02D09952CC080919B11882341F1E4
:1018600080E990E10E945A1C2091991030919A10C1
:101870008091A0119091A1112817390719F40E94A5
:10188000371116C00E946C2213C00E94311210C082
:101890000E9488200DC00E949E190AC00E949B19B8
:1018A00007C00E94A11904C0818192810E9407246F
:1018B0000E94AA0B882309F0A3CF08958093A71153
:1018C0000E94100608951F93DF93CF93CDB7DEB724
:1018D00028970FB6F894DEBF0FBECDBF182F8FEF3D
:1018E0009FEF90939F1180939E119093A1118093ED
:1018F000A01110929B119093A3118093A211909329
:10190000A5118093A4111092A6111092AA1181E042
:101910008093AB110E9409081093A7111F3F19F083
:10192000812F0E94100681E00E94730688E00E94C9
:101930008B060E94E20487E164E042E021E00E941D
:10194000760A86E10E948B0680E090E068E043E939
:1019500051E10E94A30881E00E9479058FEF9FEF7B
:101960000E9461058FEF9FEF0E946D058CE260EF92
:1019700044E022E00E94760A80919311898380914D
:1019800094118A83809195118B83809196118C8319
:10199000809197118D83809198118E8380919911F8
:1019A0008F8380919A118887CE0101960E945105FC
:1019B0000E94AC1C28960FB6F894DEBF0FBECDBFB8
:1019C000CF91DF911F9108958091CA05089580936A
:1019D000000108958091000108958091CA0588232F
:1019E00069F0E091EB11F0E0EE0FFF1FE551FE4EC4
:1019F000838194818C509E4F94838383089587E0E4
:101A00000E945C0AE091EB11F0E0EE0FFF1FE55140
:101A1000FE4E23813481280F311D3483238381AD11
:101A200092AD019692AF81AF87E060E00E94300AEC
:101A300016BC85B5826085BD089583E098E09093DB
:101A400013118093121180919C11809314118F5F58
:101A500080939C118FEF9FEF909316118093151137
:101A6000909318118093171187E08093191188E0E3
:101A700062E171E10E94F20608950F931F93DF93D4
:101A8000CF93CDB7DEB76A970FB6F894DEBF0FBE1F
:101A9000CDBF8EE00E945C0A682F6F7E8EE00E94B0
:101AA000300A85B58D7F85BD8091EB118A31C8F1F3
:101AB0001092CA0580915B12882381F1A4E0B2E103
:101AC000FD012FEF3FEF808191818217930708F48A
:101AD0009C01329682E1E432F807A9F74BE060E01E
:101AE0008E010F5F1F4F8D919C9111978217930765
:101AF00029F4F801E60FF11D40836F5F4F5F1296E6
:101B00004B3189F7662351F08091ED110E94FA82E2
:101B1000FE01E90FF11D81810E94CD180E940D196F
:101B200028C08F5F8093EB110E94100680915B129A
:101B3000882311F00E941D0D87E060E00E94300AAA
:101B400080915A12882329F016BC85B5826085BD24
:101B500008C08EE00E945C0A682F60618EE00E94DF
:101B6000300A84E190E06DE37DE00E9400108093F4
:101B7000EC116A960FB6F894DEBF0FBECDBFCF91C1
:101B8000DF911F910F9108951F93182F8091CA051F
:101B90008823B1F080915A12882321F085B58D7F7A
:101BA00085BD08C08EE00E945C0A682F6F7E8EE0C3
:101BB0000E94300A8091EC110E94080F1092CA0511
:101BC000EEEEF1E11182108217AA16AA329682E196
:101BD000E432F807B9F717AB8AE08093EB11109263
:101BE000EC118FEF0E94630C86E00E948B0688E068
:101BF0000E9446068093ED118BE00E9410060E9421
:101C00003A06823021F481E080935A1202C0109289
:101C10005A1280915A12882361F083E084BD88E0D3
:101C200085BD86E987BD80916E00816080936E00DE
:101C300008C08EE00E945C0A682F60618EE00E94FE
:101C4000300A81E08093CA050E943D0D1F910895DE
:101C50001F9310E08091DA118F3FE1F011E0809145
:101C6000D6119091D71190939F1180939E1120913E
:101C7000D8113091D9113093A3112093A2110E9451
:101C80006D058091DA110E945E0C8091DE118F5FEC
:101C90008093A611812F0E9497121F910895909111
:101CA000A7119F3FA9F481E08093CA0586E1E5ED85
:101CB000F1E1DF011D928A95E9F79093DA118BE04B
:101CC0008093A71180910001803811F08093A711B3
:101CD0004091A7114B3148F4242F30E0809100014E
:101CE00090E001962817390741F41092CA058FEF4A
:101CF0008093A7110E94280E0895842F0E945E0CE5
:101D00000E941D0D8091A7118F5F8093A71184E120
:101D100090E06FE47EE00E9400100895DF93CF937F
:101D20000F92CDB7DEB79C01009711F421E030E0AF
:101D30008FB78983F89430937C1220937B1289812A
:101D40008FBF0F90CF91DF910895DF93CF930F92C4
:101D5000CDB7DEB78FB78983F8942091791230918F
:101D60007A1289818FBFC9010F90CF91DF910895B9
:101D7000DF93CF930F92CDB7DEB78FB78983F894F7
:101D800020915C1230915D1240915E1250915F1271
:101D900089818FBFB901CA010F90CF91DF9108955A
:101DA0000F931F93CF93DF938C010E94A50EE80140
:101DB000C80FD91F012B29F00E94A50EC817D907FB
:101DC000D9F7DF91CF911F910F9108959091CB0595
:101DD0009F5F09F491E0EFE7F2E121E0808189174C
:101DE00009F420E0359682E1E33EF807B9F7E2E630
:101DF000F2E18081891709F420E0359682E1EB3722
:101E0000F807B9F7222321F39093CB05892F089582
:101E1000982FEFE7F2E120E030E08081891751F45C
:101E2000F901EE0FFF1FEE0FFF1FE20FF31FE35844
:101E3000FD4E16C02F5F3F4F35962431310569F7AF
:101E4000E2E6F2E120E030E08081891769F4F901EF
:101E5000EE0FFF1FEE0FFF1FE20FF31FE05AFD4EC4
:101E600011821082128208952F5F3F4F35962530E0
:101E7000310551F70895DF92EF92FF920F931F9370
:101E8000DF93CF9300D00F92CDB7DEB780915C1275
:101E900090915D12A0915E12B0915F120196A11D0A
:101EA000B11D80935C1290935D12A0935E12B0936B
:101EB0005F128091010190910201019790930201BC
:101EC00080930101892B49F00DE712E136E1D32E11
:101ED0007E010894E11CF11C27C088EE93E09093EA
:101EE00002018093010100E612E126E1D22E7E017B
:101EF0000894E11CF11CF80180819181009769F040
:101F0000019791838083892B41F4D98283819481C5
:101F10009B838A83C7010E94B30B0B5F1F4FF2E1C3
:101F200009371F0741F7D0CFF801808191810097D1
:101F300069F0019791838083892B41F4D982838151
:101F400094819B838A83C7010E94B30B0B5F1F4F51
:101F5000F2E1013E1F0741F70F900F900F90CF91D4
:101F6000DF911F910F91FF90EF90DF900895EF9216
:101F7000FF920F931F93DF93CF930F92CDB7DEB7EE
:101F8000AC01009719F4FB01099531C0E0E6F2E1DC
:101F900020E080819181892B31F5E22EFF24870199
:101FA000000F111F000F111F0E0D1F1D005A1D4E97
:101FB000F80151834083748363830E94E60EF80125
:101FC00082838FB78983F8940E944C1089818FBFD8
:101FD000F701EE0FFF1FEE0FFF1FEE0DFF1DE05A82
:101FE000FD4E828105C02F5F3596253091F680E049
:101FF0000F90CF91DF911F910F91FF90EF90089577
:102000000F931F93DF93CF930F92CDB7DEB7AC0141
:10201000009719F4FB01099538C08FB78983F894AC
:10202000EDE7F2E100E080819181892B51F5202FCD
:1020300030E0F901EE0FFF1FEE0FFF1FE20FF31F5D
:10204000E358FD4ECA014115510511F481E090E0BD
:10205000918380838901000F111F000F111F020F50
:10206000131F03581D4EF801748363830E94E60E0C
:10207000F80182830E944C1089818FBFF801828110
:1020800005C00F5F3596043171F680E00F90CF9157
:10209000DF911F910F9108958091CC05882351F411
:1020A000109295001092940082E08093710081E07C
:1020B0008093CC0508951F920F920FB60F920BB626
:1020C0000F9211242F933F934F935F936F937F93BE
:1020D0008F939F93AF93BF93EF93FF938091791268
:1020E00090917A12019690937A128093791280914E
:1020F0005C1290915D12A0915E12B0915F120196F8
:10210000A11DB11D80935C1290935D12A0935E128D
:10211000B0935F120E943B0FFF91EF91BF91AF917F
:102120009F918F917F916F915F914F913F912F91EF
:102130000F900BBE0F900FBE0F901F901895E1E906
:10214000F0E080818A60808388EE93E0909399002C
:102150008093980080919400909195000E94558002
:102160000895089508950895282F8091A0119091C1
:10217000A11168177907E9F080919B118823C9F0B4
:102180007093CE056093CD052093CF051092D005B6
:10219000CB010E941122882319F480E090E002C054
:1021A00085E090E06AED70E10E94001081E080938C
:1021B000AA1108951F93DF93CF93CDB7DEB7609731
:1021C0000FB6F894DEBF0FBECDBF81E698E89A83C4
:1021D000898380919D118B838F5F80939D11809166
:1021E0009E1190919F119D838C838091A01190915D
:1021F000A111998788879D878C878091CD059091C3
:10220000CE059B878A878091CF058E870E94000824
:102210008F870E94D104888B8091CD059091CE0547
:102220000E944C1B182F8E831F8290E00E94ED1A93
:10223000882331F0812F90E00E94091B882331F41C
:1022400080E1BE016F5F7F4F0E94F20660960FB67D
:10225000F894DEBF0FBECDBFCF91DF911F910895DF
:102260008091111162E171E10E94F206089580915E
:102270009D1090E08F7790708230910579F08330D7
:1022800091051CF40197F9F406C08330910569F0BB
:102290000597C9F411C00E943713089580919B10CF
:1022A00090919C100E945513089580919B109091DD
:1022B0009C100E94A419089560918F10605180E9CC
:1022C00090E10E94216E0895AF92BF92CF92DF926B
:1022D000EF92FF920F931F93CF93DF937C01162F02
:1022E0006A01B22EA02E2091A0113091A111821767
:1022F000930709F487C08FEFE8168FEFF80609F40B
:1023000081C080919B11882309F47CC081E698E804
:10231000909313118093121180919D118093141149
:102320008F5F80939D1180919E1190919F1190934A
:1023300016118093151130931A1120931911F092F0
:102340001C11E0921B1130931E1120931D11C70127
:102350000E941122082FC7010E94361BEC015E2D3E
:102360004F2D06C0CE010E94361B5C2F4D2FEC0175
:102370002097C1F75093171140931811B0921F1175
:1023800090E009C0E92FF0E0EE5EFE4ED6018D919F
:102390006D0186879F5F9117A8F3209117113091E7
:1023A00018118091A0119091A1112817390751F1AE
:1023B0002F5F3F4F39F1125F1093111181E080932D
:1023C000AA11C7010E94ED1A882319F0C7010E94C3
:1023D000091BAA2061F0002319F487E090E002C0F5
:1023E00085E090E00E94D00E0E9430110BC00023C7
:1023F00019F487E090E002C085E090E060E371E1CD
:102400000E940010DF91CF911F910F91FF90EF90EC
:10241000DF90CF90BF90AF9008950F93022F25E0EB
:102420000E9464110F9108950F93DF93CF9300D012
:10243000CDB7DEB77A83698362E0AE014F5F5F4F4D
:1024400026E000E00E9464110F900F90CF91DF9181
:102450000F9108950F9321E000E00E9464110F9105
:10246000089580E090E89093131180931211809169
:102470009C11809314118F5F80939C1180919E1109
:1024800090919F1190931611809315118091A01136
:102490009091A11190931811809317118FEF90E4F0
:1024A00090931A118093191186E080931B118091EB
:1024B000A61180931C118BE062E171E10E94F2068B
:1024C00008950F931F93CF93DF93EC018FEFCF3FCE
:1024D000D80761F488E00E944606182F00E088E0E3
:1024E0000E944606C82FD0E0C02BD12BCE010E94FF
:1024F0006D05D0939F11C0939E1180E090E00E94E3
:1025000061051092A1111092A011DF91CF911F913E
:102510000F91089508955F9808955F9808955F98C2
:1025200008950895089508950895089508950895C3
:102530008DE792E00E94840B89E592E00E94840B73
:1025400008956F927F928F929F92AF92BF92CF9297
:10255000DF92EF92FF920F931F93DF93CF93CDB74C
:10256000DEB7A8970FB6F894DEBF0FBECDBF84E1EB
:1025700093E00E94840B2BE8E22E24E0F22E9BEEE7
:10258000C92E91E0D92E4E010894811C911C83E044
:10259000682E81E0782ED7018C910E945C0A182F5A
:1025A000EDB7FEB738970FB6F894FEBF0FBEEDBF7C
:1025B0003196ADB7BEB712969C928E9211977382E8
:1025C0006282D582C482868317820E943C81EDB7E5
:1025D000FEB738960FB6F894FEBF0FBEEDBFC4012C
:1025E0000E94920B07E0A12EBB24C501002E02C061
:1025F000959587950A94E2F780FD02C080E301C0BB
:1026000081E30E943D0B015080F781E191E00E943F
:10261000920B0894E11CF11C80E190E0C80ED91ED9
:1026200095EBE91694E0F90609F0B5CF81E193E066
:102630000E94840BA8960FB6F894DEBF0FBECDBFE4
:10264000CF91DF911F910F91FF90EF90DF90CF908E
:10265000BF90AF909F908F907F906F9008955F9AFA
:102660008AE090E06BE872E10E940010089580918A
:102670009D10813091F45F9A8AE090E06BE872E1FE
:102680000E940010E0918F10E051F0E0E057FF4E03
:1026900016868EE990E10E94920B089588EE93E0F1
:1026A0006EE473E10E9400100895EF92FF920F9381
:1026B0001F937C015F9A81E090E06BE872E10E94D9
:1026C000001086E493E00E94840B00D000D000D07C
:1026D000EDB7FEB731960DEA11E1ADB7BEB7129670
:1026E0001C930E93119784E191E093838283F5828A
:1026F000E4820E943C818DB79EB706960FB6F8948F
:102700009EBF0FBE8DBFC8010E94920B83E0B70130
:102710000E94B4101F910F91FF90EF9008955F9A5F
:1027200081E090E06BE872E10E94001008955F9AEA
:1027300089E190E06BE872E10E94001008950F9328
:102740001F93882349F080933F0670933E06609361
:102750003D0681E08093400680913F06882309F47E
:1027600056C08091400690E00E94E91BFC018081E8
:10277000882311F490E032C080913F06813069F5E2
:102780008CEA92E00E94840B00D000D000D0EDB71C
:10279000FEB731960DEA11E1ADB7BEB712961C93A4
:1027A0000E93119784E191E0938382838091400698
:1027B000848315820E943C818DB79EB706960FB622
:1027C000F8949EBF0FBE8DBFC8010E94920B60910E
:1027D000400682E070E00E94B41091E080914006D3
:1027E0008F5F809340068A3060F4992319F481E06A
:1027F00090E002C08AEF90E06DE378E10E94001063
:1028000006C010923E0610923D0610923F061F91A0
:102810000F9108959F92AF92BF92CF92DF92EF9265
:10282000FF920F931F93DF93CF93CDB7DEB7EC9753
:102830000FB6F894DEBF0FBECDBF10923C060E94CB
:10284000D80A882309F407C48091AA11882309F0C3
:1028500002C40E94F80A082F112707FD10950431C1
:10286000110511F41092D1058091D105882321F131
:1028700010923B0680913B06E82FF0E0ED52FA4FB4
:1028800000838F5F80933B06843658F40E94D80AF9
:10289000882339F00E94F80A082F112707FD1095A8
:1028A000E9CF8091390690913A0660913B0643ED5D
:1028B00055E00E942A12CFC38091D20587FD4DC0FA
:1028C000992787FD90958F779070892B09F445C0E3
:1028D000802F0E943D0B0D30110519F00A301105B3
:1028E00081F480913B06E82FF0E0ED52FA4F108220
:1028F0008F5F80933B068091D20580688093D205DC
:102900002CC080913B060830110539F4E82FF0E027
:10291000ED52FA4F1082815006C0E82FF0E0ED52E0
:10292000FA4F00838F5F80933B0680913B0684368D
:1029300040F08091D20580688093D20510923B06CA
:102940008AC30E94D80A882309F485C30E94F80A22
:10295000082F112707FD1095BBCF8091D20587FF67
:1029600004C0082F112707FD109581E191E00E9416
:10297000920B09361105A1F10A361105ACF40035A8
:10298000110509F444C3013511052CF40134110576
:1029900009F057C343C30336110509F4DEC20436F8
:1029A000110509F04EC314C00337110509F4BFC265
:1029B000043711052CF40037110509F042C39FC2FA
:1029C0000437110541F00737110509F03AC304C374
:1029D0000E94A11236C30E94421D0E943B1F31C3B8
:1029E0002DB73EB72A5030400FB6F8943EBF0FBE09
:1029F0002DBFEDB7FEB7319603ED15E0ADB7BEB70D
:102A000012961C930E93119787E191E09383828332
:102A10008091A0119091A111958384838091A2113E
:102A20009091A311978386838091A4119091A51111
:102A3000918780870E943C81EDB7FEB73A960FB62A
:102A4000F894FEBF0FBEEDBFC8010E94920B00D0EC
:102A500000D000D0EDB7FEB73196ADB7BEB7129635
:102A60001C930E93119783E491E09383828380916A
:102A7000A711848315820E943C81EDB7FEB736967C
:102A80000FB6F894FEBF0FBEEDBFC8010E94920BB7
:102A90008DE492E00E94840B00D000D000D0EDB70E
:102AA000FEB731960DEA11E1ADB7BEB712961C9391
:102AB0000E9311978FE491E09383828380919E110E
:102AC00090919F11958384830E943C81EDB7FEB75E
:102AD00036960FB6F894FEBF0FBEEDBFC8010E9438
:102AE000920B81E191E00E94920B0E94E304082F77
:102AF00010E08EE392E00E94840B0115110519F499
:102B000089E392E04AC00130110519F481E392E0B3
:102B100044C00230110519F489E292E03EC006304B
:102B2000110519F483E292E038C00830110519F458
:102B30008BE192E032C00930110519F484E192E092
:102B40002CC00131110519F487E092E026C0023152
:102B5000110519F48AEF91E020C00631110519F42E
:102B60008FEE91E01AC00931110519F484EE91E05D
:102B700014C00C31110519F488ED91E00EC00D312F
:102B8000110519F487EC91E008C00E31110519F414
:102B900084EB91E002C08BEA91E00E94840B81E11A
:102BA00091E00E94920B10919311B0909411A0901B
:102BB0009511909096116091971170919811809154
:102BC000991190919A112DB73EB72C5030400FB605
:102BD000F8943EBF0FBE2DBFEDB6FEB60894E11CC3
:102BE000F11CE3EDCE2EE5E0DE2EADB7BEB71296BA
:102BF000DC92CE92119722E531E0F70133832283F4
:102C0000212F3B2D4A2D592D00E20E94807FC901C2
:102C1000BA01D70114962C93149715969C93159787
:102C200016964C93169717967C93179718961C93A5
:102C300018971996BC9219971A96AC921A971B96E8
:102C40009C920E943C81EDB7FEB73C960FB6F8947B
:102C5000FEBF0FBEEDBFC6010E94920B80919B117B
:102C6000882319F428E631E002C02EE631E08DB762
:102C70009EB708970FB6F8949EBF0FBE8DBFEDB7F5
:102C8000FEB7319603ED15E0ADB7BEB712961C93B3
:102C90000E93119783E791E0938382833583248396
:102CA0008091A611868317820E943C81EDB7FEB702
:102CB00038960FB6F894FEBF0FBEEDBFC8010E9454
:102CC000920B88E00E94460600D000D000D0EDB7FD
:102CD000FEB73196ADB7BEB712961C930E931197FF
:102CE0002DE831E033832283848315820E943C8166
:102CF000EDB7FEB736960FB6F894FEBF0FBEEDBF28
:102D0000C8010E94920B0E943A06833059F0873026
:102D100069F0823021F466EEA62EB12C0AC0A82EEE
:102D2000BB2407C057EEA52EB12C03C044EDA42E42
:102D3000B12C83EA91E00E94840B8DE10E945C0A31
:102D40002DB73EB7285030400FB6F8943EBF0FBEA7
:102D50002DBFEDB7FEB7319603ED15E0ADB7BEB7A9
:102D600012961C930E9311972BE931E03383228343
:102D7000B582A482868317820E943C81EDB7FEB79C
:102D800038960FB6F894FEBF0FBEEDBFC8010E9483
:102D9000920B00D000D000D0EDB7FEB73196ADB7A2
:102DA000BEB712961C930E93119788EA91E0938315
:102DB000828335EBE32E31E0F32EF582E4820E942C
:102DC0003C81EDB7FEB736960FB6F894FEBF0FBE46
:102DD000EDBFC8010E94920B00D000D000D0EDB72B
:102DE000FEB73196ADB7BEB712961C930E931197EE
:102DF00089EB91E09383828388E090E095838483DC
:102E00000E943C81EDB7FEB736960FB6F894FEBF30
:102E10000FBEEDBFC8010E94920B00D000D000D0C1
:102E2000EDB7FEB73196ADB7BEB712961C930E93B1
:102E3000119788EC91E093838283F582E4820E946B
:102E40003C81EDB7FEB736960FB6F894FEBF0FBEC5
:102E5000EDBFC8010E94920B00D000D000D0EDB7AA
:102E6000FEB73196ADB7BEB712961C930E9311976D
:102E700087ED91E09383828388EE91E0958384834C
:102E80000E943C81EDB7FEB736960FB6F894FEBFB0
:102E90000FBEEDBF8DE891E00E94840B8091E81B8E
:102EA0008F3F61F08E010F5F1F4FC80168ED7BE11E
:102EB0000E94ED79C8010E94920B04C08FE791E057
:102EC0000E94840B8AE691E00E94840B8091E81BAB
:102ED0008F3F61F08E010F5F1F4FC80161E57CE1FC
:102EE0000E94ED79C8010E94920B04C08CE591E02C
:102EF0000E94840B89E591E00E94840BA2C085E4C6
:102F000091E00E94840B83ED95E062E341E00E9432
:102F1000480B83ED95E00E946080682F809339060E
:102F200090933A0682E0792F0E94B4108AC08EE214
:102F300091E00E94840B83ED95E062E341E00E9402
:102F4000480B83ED95E00E94608090933A06809351
:102F5000390681E08093D10574C08DE191E00E9433
:102F6000840B83ED95E062E341E00E94480B83ED22
:102F700095E00E946080182F8BE091E00E94840B06
:102F800083ED95E062E341E00E94480B812F0E94AF
:102F9000630C80919E1190919F110E9461128CEEA2
:102FA00090E00E94840B81E080939B1183ED95E07B
:102FB0000E94608090933A0680933906009709F446
:102FC00040C00E946D058091390690913A06909319
:102FD0009F1180939E1135C089ED90E00E94840B73
:102FE00083ED95E062E341E00E94480B83ED95E0BC
:102FF0000E94608090933A06809339060E94FF0BEE
:103000008091390690913A060E94391C1AC08AEBC9
:1030100090E00E94840B0E94EC0A13C088E990E0C3
:103020000E94840B83ED95E062E341E00E94480B2F
:103030008091D305803729F481E060E070E00E9440
:103040009F138091D205882331F48AEF90E068E9DC
:1030500072E10E940010EC960FB6F894DEBF0FBE2E
:10306000CDBFCF91DF911F910F91FF90EF90DF9037
:10307000CF90BF90AF909F90089580E060E070E0A7
:103080000E949F1308958FE260E00E94300A82E060
:1030900060E070E00E94B41084EF91E063E478E1B6
:1030A0000E940010809341060895CF92DF92EF9224
:1030B000FF920F931F93DF93CF93CDB7DEB728977F
:1030C0000FB6F894DEBF0FBECDBF6E010894C11CD1
:1030D000D11C80E090E068E0A6010E94A308760180
:1030E00086019E01275F3F4FF80180818F3FA9F441
:1030F0000F5F1F4F02171307B9F727C088E00E9420
:103100004606F70181937F01E017F107B9F780E0E8
:1031100090E068E0A6010E94880880E190E062E00B
:10312000A6010E94A308F601808191818F5F9F4FC5
:1031300099F484E190E0F6019183808380E190E04E
:1031400062E0A6010E94880807C080E00E9409088A
:1031500086E00E948B06D2CF28960FB6F894DEBF89
:103160000FBECDBFCF91DF911F910F91FF90EF90D8
:10317000DF90CF9008958AB1806A8AB98DB1806C52
:103180008DB90E9497130E94551881E00E94C40DCA
:103190008CEB92E00E94840B0895FF920F931F9393
:1031A000F82E0E94630C8FEF9FEF0E9461128AEC51
:1031B00092E00E94840B00D000D000D0EDB7FEB7A3
:1031C00031960DEA11E1ADB7BEB712961C930E937E
:1031D000119784E191E093838283F48215820E94A7
:1031E0003C818DB79EB706960FB6F8949EBF0FBE72
:1031F0008DBFC8010E94920B81E080939B1160916A
:10320000A0117091A11180919E1190919F110E9427
:103210001B6A1F910F91FF9008958091AC1183302C
:1032200029F40E94E22780E00E94C40D0895EF92E5
:10323000FF920F931F938FEF92E00E94840B00D0B8
:1032400000D000D0EDB7FEB731960DEA11E1ADB771
:10325000BEB712961C930E9311978FE491E093835F
:1032600082838091D8119091D911958384830E9493
:103270003C818DB79EB706960FB6F8949EBF0FBEE1
:103280008DBFC8010E94920B87EF92E00E94840BD1
:1032900000D000D000D0EDB7FEB73196ADB7BEB7C5
:1032A00012961C930E931197A4E1EA2EA1E0FA2E38
:1032B000F382E2828091DA11848315820E943C813C
:1032C0008DB79EB706960FB6F8949EBF0FBE8DBF02
:1032D000C8010E94920B8DEE92E00E94840B00D0F8
:1032E00000D000D0EDB7FEB73196ADB7BEB712969D
:1032F0001C930E931197F382E2828091DE118483F6
:1033000015820E943C818DB79EB706960FB6F89441
:103310009EBF0FBE8DBFC8010E94920B8091D81135
:103320009091D9116091DA110E94281A1F910F9182
:10333000FF90EF9008950E94272308950E9427236D
:1033400008950E9424230895EF92FF920F931F93F4
:103350007C0180E393E00E94840B00D000D000D079
:10336000EDB7FEB731960DEA11E1ADB7BEB71296D3
:103370001C930E9311978FE491E093838283F582DF
:10338000E4820E943C818DB79EB706960FB6F894F2
:103390009EBF0FBE8DBFC8010E94920B8AE293E0D0
:1033A0000E94840B0E94D10400D000D000D0EDB761
:1033B000FEB73196ADB7BEB712961C930E93119718
:1033C000B4E1EB2EB1E0FB2EF382E282848315821E
:1033D0000E943C818DB79EB706960FB6F8949EBFAB
:1033E0000FBE8DBFC8010E94920B83E293E00E9442
:1033F000840B0E94000800D000D000D0EDB7FEB7CB
:103400003196ADB7BEB712961C930E931197F38207
:10341000E282848315820E943C818DB79EB7069616
:103420000FB6F8949EBF0FBE8DBFC8010E94920BCD
:1034300081E191E00E94920B5F9A8AE090E06BE854
:1034400072E10E9400101F910F91FF90EF9008957C
:1034500008950895EF92FF920F931F93CF93DF93F8
:10346000E82EEB018A0181E080934606F880B9815D
:10347000AA817B816C813D812E819F81E5E5F6E00B
:1034800041E050E080818F15A9F481818B1791F480
:1034900082818A1779F48381871761F48481861782
:1034A00049F48581831731F48681821719F4878165
:1034B0008917A1F04F5F5F4F3E964A30510511F7D3
:1034C000E4E5F6E041E050E08081882351F04F5F71
:1034D0005F4F3E964A305105B9F735C04A30510525
:1034E00090F5CA01880F991FBC0123E0660F771F72
:1034F0002A95E1F7681B790B9B012A5B394FF9018B
:10350000E1928881D90111968C93119789818183E9
:103510008A8182838B8183838C8184838D8185835F
:103520008E8186838F8187831A961C930E931997B9
:103530001C961C921E921B97DB01AD5AB94F8C91C1
:103540008E7F8C9302C04FEF5FEFCA01DF91CF9166
:103550001F910F91FF90EF900895DC01E4E5F6E0F4
:1035600021E030E08081882371F191818C9198175E
:1035700051F5928111968C911197981721F59381AD
:1035800012968C9112979817F1F4948113968C915E
:1035900013979817C1F4958114968C9114979817E6
:1035A00091F4968115968C911597981761F49781EF
:1035B00016968C911697981731F4908517968C91E2
:1035C0001797981741F02F5F3F4F3E962A303105ED
:1035D00049F62FEF3FEFC90108958A309105B0F405
:1035E000880F991FFC0143E0EE0FFF1F4A95E1F79A
:1035F000E81BF90BEA5BF94F8081882339F020E062
:1036000081859285892B19F421E001C020E0822F69
:1036100008958A30910510F080E00895880F991F71
:10362000FC0163E0EE0FFF1F6A95E1F7E81BF90B61
:10363000ED5AF94F80818695817009F081E00895F7
:1036400008958A30910588F4880F991FFC01A3E042
:10365000EE0FFF1FAA95E1F7E81BF90BEA5BF94FA4
:103660001082128611861486138608958A30910579
:1036700018F020E030E00EC0880F991FFC0123E015
:10368000EE0FFF1F2A95E1F7E81BF90BEA5BF94FF4
:1036900021853285C90108950F931F93CF93DF933E
:1036A000EC018A309105D0F4CE01880F991F8C016E
:1036B00043E0000F111F4A95E1F7081B190B0A5B45
:1036C000194FF8018081882349F0CE010E94ED1A3C
:1036D000882331F4F801C185D285E6CFC0E0D0E07F
:1036E000CE01DF91CF911F910F910895AC01E4E5D8
:1036F000F6E021E030E08081882329F08185928501
:103700008417950741F02F5F3F4F3E962A303105D1
:1037100091F720E030E0C90108959C018A309105BD
:1037200060F5880F991FFC01A3E0EE0FFF1FAA951B
:10373000E1F7E81BF90BEA5BF94F418552852F5FF2
:103740003F4FC901880F991FFC0163E0EE0FFF1F77
:103750006A95E1F7E81BF90BEA5BF94F0BC0808132
:10376000882329F0818592858417950741F02F5F82
:103770003F4F3E962A30310591F720E030E0C901F5
:1037800008958A30910518F020E030E00EC0880FCF
:10379000991FFC0123E0EE0FFF1F2A95E1F7E81BBC
:1037A000F90BEA5BF94F23853485C90108958A3006
:1037B000910570F4880F991FFC0143E0EE0FFF1F85
:1037C0004A95E1F7E81BF90BEA5BF94F74876387C9
:1037D00008958A30910518F020E030E00CC0880F81
:1037E000991F9C0163E0220F331F6A95E1F7281BA4
:1037F000390B2A5B394FC9010895CF93DF93EC0150
:103800000E94ED1A882399F0CA30D10580F4CE01C8
:10381000880F991FFC01A3E0EE0FFF1FAA95E1F7A7
:10382000E81BF90BED5AF94F80818E7F8083DF9181
:10383000CF91089580E090E0089580E090E00895B1
:1038400021E0880F991FFC0133E0EE0FFF1F3A952E
:10385000E1F7E81BF90BEA5BF94F8081882331F02F
:1038600081859285009719F02F5FEBCF20E0822FA2
:103870000895CF93DF93EC010E94361B0097A1F4CB
:10388000CA30D105A0F4CE01880F991FFC0153E086
:10389000EE0FFF1F5A95E1F7E81BF90BED5AF94FB0
:1038A00080818160808303C0BE010E941412DF9179
:1038B000CF910895EF92FF920F931F93CF93DF93D1
:1038C0007C01DC011B960D911C911C97C8010E9484
:1038D000ED1A8823D1F10A301105B8F5C801880F17
:1038E000991FFC01A3E0EE0FFF1FAA95E1F7E81B6B
:1038F000F90BED5AF94F90E0D7011D968C9187FD99
:1039000091E0990F80818D7F892B8083C801880F7A
:10391000991FEC0173E0CC0FDD1F7A95E1F7C81B0E
:10392000D90BCD5AD94F888180FF08C0C80160E00B
:1039300070E00E94141288818E7F8883C8010E94E3
:10394000B310F70185858F778587DF91CF911F9120
:103950000F91FF90EF9008958CE8E6E4F6E0DF0128
:103960001D928A95E9F70895909343068093420645
:10397000709345066093440680EA90E066EC7CE133
:103980000E94001081E08093AA1108958091420660
:10399000909143060E941122882319F480E090E060
:1039A00002C085E090E06AE97EE10E94001008957F
:1039B000DF93CF930F92CDB7DEB79C01AB018A3076
:1039C000910508F05AC0880F991FFC01A3E0EE0F83
:1039D000FF1FAA95E1F7E81BF90BEA5BF94F80811D
:1039E000882331F48EEF93E00E94840B80E046C080
:1039F000232B09F442C02185328521153105E9F1D7
:103A000081E089836115710519F4A0E0B0E002C07E
:103A1000DB011A96C901880F991FFC0163E0EE0FC4
:103A2000FF1F6A95E1F7E81BF90BEA5BF94F80810C
:103A3000882321F189818F5F898381859285892BF4
:103A400041F44115510519F0FA0136832583898126
:103A500015C0109711F02D933D93C901880F991F40
:103A6000FC0123E0EE0FFF1F2A95E1F7E81BF90B9D
:103A7000EA5BF94F21853285CDCF81E00F90CF9160
:103A8000DF9108952F923F924F925F926F927F92B3
:103A90008F929F92AF92BF92CF92DF92EF92FF925E
:103AA0000F931F93DF93CF93CDB7DEB7E6970FB693
:103AB000F894DEBF0FBECDBF8091DF049091E0048B
:103AC000A091E104B091E20489839A83AB83BC8323
:103AD0008EEE93E00E94840B84E5882E86E0982E7B
:103AE00001E0602E712C15E0212E312C2C0E3D1E94
:103AF0002E010894411C511CF4012081222309F459
:103B000071C01181D280C380B48065817681878144
:103B100090854DB75EB7465150400FB6F8945EBFE2
:103B20000FBE4DBFEDB6FEB60894E11CF11CEDB71B
:103B3000FEB73282218245EB54E0F7015383428382
:103B4000F201E20FF11D2081332727FD3095F701A7
:103B50003583248377826682F40121853285220FA2
:103B6000331FF901A3E0EE0FFF1FAA95E1F7E21B57
:103B7000F30BEA5BF94F2081F201E20FF11D208186
:103B8000332727FD3095F70131872087F401218500
:103B90003285F70133872287F40123853485F701C5
:103BA00035872487212F3D2D4C2D5B2D00E20E946F
:103BB000807FC901BA01F70126879787408B718BF7
:103BC000128BD38AC48AB58A0E943C814DB75EB7F6
:103BD0004A5E5F4F0FB6F8945EBF0FBE4DBFC10186
:103BE0000E94920B8EE090E0880E991E0894611C52
:103BF000711C92ED891696E0990609F07DCF8DED46
:103C000093E00E94840B00E010E0EE2455E0852E46
:103C1000912C8C0E9D1E47EDA42E44E0B42E3E0147
:103C20000894611C711C01C08601EDB7FEB738977E
:103C30000FB6F894FEBF0FBEEDBFADB7BEB711967D
:103C4000928281821396BC92AE921297C801880F1D
:103C5000991FFC0123E0EE0FFF1F2A95E1F7E81BF7
:103C6000F90BEA5BF94F8081F301E80FF11D8081C8
:103C7000992787FD909515969C938E931497179688
:103C80001C930E9316970E943C814DB75EB7485F18
:103C90005F4F0FB6F8945EBF0FBE4DBFC4010E94C8
:103CA000920BC8010E94761B009719F0E3948C01D7
:103CB000BCCFC8010E948D1B6C01009771F08AED8A
:103CC00093E00E94840B10E005C085ED93E00E9414
:103CD000840B1F5F1E15C8F3A7CFC801880F991F5B
:103CE000FC0113E0EE0FFF1F1A95E1F7E81BF90B3B
:103CF000EA5BF94F018512850115110511F0EA946F
:103D0000D8CFE6960FB6F894DEBF0FBECDBFCF91E9
:103D1000DF911F910F91FF90EF90DF90CF90BF90B8
:103D2000AF909F908F907F906F905F904F903F905B
:103D30002F900895EF92FF920F931F93DF93CF93ED
:103D4000CDB7DEB760970FB6F894DEBF0FBECDBF1C
:103D50008EE693E00E94840B00D000D000D0EDB737
:103D6000FEB731960DEA11E1ADB7BEB712961C93BE
:103D70000E93119794EEE92E94E0F92EF382E282ED
:103D80008091440690914506958384830E943C81EE
:103D90008DB79EB706960FB6F8949EBF0FBE8DBF27
:103DA000C8010E94920B80E693E00E94840B00D031
:103DB00000D000D0EDB7FEB73196ADB7BEB71296C2
:103DC0001C930E931197F382E282809142069091A8
:103DD0004306958384830E943C818DB79EB70696E7
:103DE0000FB6F8949EBF0FBE8DBFC8010E94920B04
:103DF00081E698E89A83898380919D118B838F5FF8
:103E000080939D1180919E1190919F119D838C8331
:103E10000091420610914306C8010E944C1BAC0160
:103E20002091440630914506009791F0388B2F87FA
:103E300084E08E871D861C861B870A871986188654
:103E40005F834E8380E1BE016F5F7F4F0E94F20669
:103E500060960FB6F894DEBF0FBECDBFCF91DF9155
:103E60001F910F91FF90EF90089586E162E171E15B
:103E70000E94F20608953F924F925F926F927F9256
:103E80008F929F92AF92BF92CF92DF92EF92FF926A
:103E90000F931F93DF93CF93CDB7DEB7C255D040BA
:103EA0000FB6F894DEBF0FBECDBF8091311C8823C2
:103EB000C9F18091331C8823A9F18091461C8F3F62
:103EC00011F4AA240DC0DE011196E6E3FCE180E1C5
:103ED00001900D928150E1F71F86188AAA24A394BD
:103EE0008091611C8F3F09F468C02A2D30E0C90120
:103EF000A4E0880F991FAA95E1F7FE013196E80F1B
:103F0000F91FA1E5BCE180E10D9001928150E1F73C
:103F1000F4E0220F331FFA95E1F7FE013196E20F2C
:103F2000F31F48C04091BD1C4D7F5091BE1C809135
:103F3000CD1B8F3F11F4AA2415C0DE011196EDEBC5
:103F4000FBE180E101900D928150E1F749875A87AA
:103F50001B868FEF8C878EEF8D871E861F86188AB3
:103F6000AA24A3948091E81B8F3F39F12A2D30E0D9
:103F7000C901E4E0880F991FEA95E1F7FE01319647
:103F8000E80FF91FA8EDBBE180E10D90019281508F
:103F9000E1F774E0220F331F7A95E1F7FE013196C5
:103FA000E20FF31F4087518712868FEF83878EEFD2
:103FB0008487158616861786A39482EA93E00E946A
:103FC000840B64E5862E66E0962E51E0652E712CFA
:103FD00041E2442E512C4C0E5D1E362CF4018081A2
:103FE000882309F46FC01181D280C380B4806581B9
:103FF0007681878190852DB73EB72E5030400FB621
:10400000F8943EBF0FBE2DBFEDB6FEB60894E11C7E
:10401000F11CEDB7FEB75282418227EE34E0F70182
:1040200033832283212F3D2D4C2D5B2D00E20E94F6
:10403000807FC901BA01F701248395834683778382
:104040001087D186C286B386758664860E943C81BD
:104050002DB73EB7225F3F4F0FB6F8943EBF0FBE5D
:104060002DBFC2010E94920B30E1C32ED12CCC0E89
:10407000DD1E00E010E024C0F6013082B80124E02B
:10408000660F771F2A95E1F721E030E02C0F3D1FE6
:10409000620F731FC2010E94ED79002321F083E8B3
:1040A00093E00E94840BC2010E94920B80E893E08F
:1040B0000E94840B0F5F1F4F80E190E0C80ED91E55
:1040C0000A15D0F2EEE0F0E08E0E9F1E0894611CFF
:1040D000711CF2ED8F16F6E09F0609F07ECFCE5AE6
:1040E000DF4F0FB6F894DEBF0FBECDBFCF91DF918B
:1040F0001F910F91FF90EF90DF90CF90BF90AF9006
:104100009F908F907F906F905F904F903F90089519
:10411000EF92FF920F931F93CF93DF9390919110A3
:1041200080E020919010820F911D28E8833692073D
:1041300009F0A4C08CE990E10E94AD1ABC018FEF98
:104140006F3F780719F1CB01880F991FFC0123E01D
:10415000EE0FFF1F2A95E1F7E81BF90BEA5BF94F19
:104160008081882399F0218532852115310521F43C
:10417000CB010E94211B0AC080919A1090919B1044
:104180008217930719F0C9010E94B41C80919A10FC
:1041900090919B100E941122182F40919A105091DB
:1041A0009B108091A4106CE970E10E942A1AEC0126
:1041B000909327118093261183E698E8909313112A
:1041C0008093121180919D11809314118F5F8093C1
:1041D0009D1180919E1190919F1190931611809343
:1041E00015118091971090919810909318118093C9
:1041F00017118091A0119091A11190931A118093A1
:10420000191182E080931B1180919A1090919B105C
:1042100090931D1180931C1180919C1080931E110E
:1042200080919D1080931F1180919E10809320118A
:1042300080919F10809321118091A0108093221172
:104240008091A110809323118091A210809324115A
:104250008091A31080932511112319F480E090E040
:1042600002C085E090E065E37FE10E94001081E0FC
:104270008093AA11CE010E942F1377C08356984CC9
:1042800019F0C0E0D0E071C087E990E10E94AD1A5A
:10429000BC01BFEF8F3F9B07B1F0880F991FFC0156
:1042A00013E0EE0FFF1F1A95E1F7E81BF90BEA5B2D
:1042B000F94F81859285009721F4CB010E94211B43
:1042C00002C00E94B41C8091A21067E970E140E036
:1042D00050E00E942A1AEC0183E69CE890931311A7
:1042E0008093121180919D11809314118F5F8093A0
:1042F0009D1180919E1190919F1190931611809322
:1043000015118091971080931711809198108093C8
:104310001811809199108093191180919A108093AF
:104320001A1180919B1080931B1180919C10809397
:104330001C1180919D1080931D1180919E1080937F
:104340001E118091A0119091A11190932011809342
:104350001F1182E080932111D0932311C093221169
:1043600082E162E171E10E94F2068FE194E00E9435
:10437000840B00D000D000D0EDB7FEB731960DEA27
:1043800011E1ADB7BEB712961C930E931197B3E02F
:10439000EB2EB5E0FB2EF382E282D583C4830E942C
:1043A0003C818DB79EB706960FB6F8949EBF0FBEA0
:1043B0008DBFC8010E94920B86E194E00E94840B9D
:1043C000CE010E94201C00D000D000D0EDB7FEB777
:1043D0003196ADB7BEB712961C930E931197F38228
:1043E000E282848315820E943C818DB79EB7069637
:1043F0000FB6F8949EBF0FBE8DBFC8010E94920BEE
:1044000083E194E00E94840BCE010E949512DF911B
:10441000CF911F910F91FF90EF9008950895089507
:104420000895FF920F931F93DF93CF93CDB7DEB71D
:10443000C258D0400FB6F894DEBF0FBECDBF8E017C
:104440000D5F1F4FB8010E94D81CF82E82E08F1517
:1044500078F583E698E89C838B8380919D11F80121
:1044600082838F5F80939D1180919E1190919F1107
:1044700094838383108617828BEB81878581968155
:104480009A83898389819A810E94C11BF801628580
:1044900073858617970761F089819A810E94D71BDF
:1044A000FF0C8F2D8A5FB8010E94F20681E001C0E7
:1044B00080E0CE57DF4F0FB6F894DEBF0FBECDBF02
:1044C000CF91DF911F910F91FF9008958FE762E1E7
:1044D00071E10E94F2060895A1E1B1E1EFE8F0E197
:1044E00082E801900D928150E1F75F9A8AE090E0B6
:1044F0006BE872E10E94001080911B1190911C11D9
:104500000E94ED1A20911B1130911C11882309F192
:1045100080919D11809314118F5F80939D11309332
:104520001811209317118091A0119091A1119093CF
:104530001A11809319118AE494E00E94840B8091EF
:104540001B1190911C110E94091B882351F141E01D
:1045500029C080919D11809314118F5F80939D11CC
:10456000C9010E944C1B909318118093171110924F
:104570001A111092191182E394E00E94840B809129
:104580001B1190911C110E941122882351F085E08B
:1045900090E066E672E20E94001081E08093AA112A
:1045A000089540E0209117113091181180911B114E
:1045B00090911C11442341F040911111425062E14D
:1045C00071E10E94B21008952F5F3F4F39F0809142
:1045D0001111825062E171E10E94F206089508957E
:1045E000089580E090E0089508950895CF93DF93B3
:1045F000EC0181E08093D206CA30D10510F5CE01DE
:10460000880F991FDC01E3E0AA0FBB1FEA95E1F7D1
:10461000A80FB91FAD51BD4EFB0180E101900D9275
:104620008150E1F7FE01EE0FFF1FCF0123E0880F5D
:10463000991F2A95E1F7E80FF91FED51FD4E518BB7
:10464000408BDF91CF9108951092D206089580910A
:10465000D206882331F08091A8119091A9110E946F
:10466000391C1092D2060895DF93CF9300D0CDB7B6
:10467000DEB79A838983482F5A81FA01EE0FFF1F14
:10468000CF0123E0880F991F2A95E1F7E80FF91F62
:10469000ED51FD4E208931892115310509F46BC09A
:1046A0001092DA151092D91580E680935616109262
:1046B00059161092581689E080935A1610925B167C
:1046C00080E480935D1681E180935C16CA01880FB7
:1046D000991FFC01A3E0EE0FFF1FAA95E1F7E80F79
:1046E000F91FAEE5B6E1ED51FD4E80E101900D926E
:1046F0008150E1F7AEE6B6E1E1E5FCE180E1019051
:104700000D928150E1F78A8180937C168981809394
:104710007D1680EF92EB90938116809380163093F4
:104720007E1620937F1680E099E090938316809305
:10473000821687E78093861610928516109284164B
:104740000E949A3E8095909590938516809384164A
:10475000892B31F48FEF9FEF909385168093841609
:1047600081E390E09093DA158093D91581E08093EE
:10477000E01C0E94EB740F900F90CF91DF91089591
:104780000F931F93182F092FE82FF92FEE0FFF1FFC
:10479000CF01A3E0880F991FAA95E1F7E80FF91F51
:1047A000ED51FD4E208931892115310569F1909136
:1047B0008016809181168217930731F5612F702F33
:1047C000660F771FCB01E3E0880F991FEA95E1F7A9
:1047D000680F791F6D517D4E8EE696E140E150E005
:1047E0000E94A180009781F4E12FF02FEE0FFF1FB0
:1047F000CF0143E0880F991F4A95E1F7E80FF91FB1
:10480000ED51FD4E118A108A1F910F9108950F935B
:104810001F93DF93CF930F92CDB7DEB78C018091BA
:10482000AC11823041F50115110569F480E990E180
:10483000BE016F5F7F4F4BE954E10E94DF248093FC
:104840008F1001E010E080910E058823A1F0809187
:104850009010813681F480919110883861F48091B4
:104860009D108F77853039F460918F10605180E909
:1048700090E10E94216E80914305809356168091AD
:104880004405809357168091450580935816809172
:104890004605809359168091470580935A1680915A
:1048A000480580935B16E1EEF5E1ACE5B6E1819158
:1048B0008D9385E1E73EF807D1F780E88093621693
:1048C0008AE9809363168EE090E09093DA158093E6
:1048D000D915012B61F484E696E1BE016F5F7F4F2D
:1048E0004BE954E10E94DF2490E00E9613C024E6C9
:1048F00036E140918F10E0E9F0E1C901BF0150E0DD
:104900000E94AE8020918F108091D9159091DA1578
:10491000820F911D9093DA158093D9156091D91566
:104920007091DA1586E596E141E00E94903510928B
:10493000DA151092D9150F90CF91DF911F910F9139
:1049400008951F93182F8093AC118BE993E160E0D9
:1049500071E04BE954E10E94BD24812F82508230E6
:1049600010F486E001C086E10E948B06133019F432
:1049700080E00E94C40D1F910895FA019183808305
:1049800075836483978386839187808761507040A5
:10499000860F971F938382830895FC01408551857C
:1049A000868197814817590728F0481B590B2481A5
:1049B000358101C09C01241B350BC9010895CF939B
:1049C000DF93EC01DA011696ED91FC911797508177
:1049D00057FD02C0452F23C08D919C9111971796CA
:1049E0009C938E93169719969C938E93189780E0BC
:1049F0004EC0019617969C938E93169728173907E9
:104A000038F48D919C91119717969C938E931697DD
:104A10001696ED91FC9117978081899341501696D7
:104A20008D919C91179712962D913C911397442349
:104A300001F7019617969C938E93169728173907BE
:104A400038F48D919C91119717969C938E9316979D
:104A50001696ED91FC9117978081FB018083169645
:104A60008D919C911797019617969C938E9316970C
:104A700012962D913C9113972817390738F48D9190
:104A80009C91119717969C938E931697852FDF9183
:104A9000CF910895EF92FF920F931F93CF93DF93DF
:104AA0008C01F62EE42EE901C9010E94CD242F2DA0
:104AB00030E02E5F3F4F8217930710F460E03BC059
:104AC000E885F985F0828885998501969987888798
:104AD0002A813B812817390720F488819981998799
:104AE00088874F2D14C0D8018C9180838885998543
:104AF0000196998788872A813B812817390720F4F6
:104B000088819981998788870F5F1F4F4150E88579
:104B1000F985442341F7E082888599850196998734
:104B200088872A813B812817390720F48881998159
:104B3000998788876F2D862FDF91CF911F910F91D5
:104B4000FF90EF900895FF920F931F93CF93DF9301
:104B5000EC01289880E20E94790880E00E947908A0
:104B6000F82E83508D3708F04BC0CE010E94CD2423
:104B70002F2D30E02E5F3F4F8217930708F440C07F
:104B8000E885F985F08288859985019699878887D7
:104B90002A813B812817390720F4888199819987D8
:104BA00088870F2D80E00E947908E885F985808349
:104BB000888599850196998788872A813B8128175E
:104BC000390720F48881998199878887015051F7A6
:104BD0000885198580E00E947908F801808388851E
:104BE00099850196998788872A813B8128173907FB
:104BF00020F48881998199878887289A8F2D02C00F
:104C0000289A80E0DF91CF911F910F91FF90089536
:104C1000089580919B11882349F082E102C00E948F
:104C2000E30481518230D8F30E9490058AB18F75D8
:104C30008AB98DB18F738DB980917A008F77809307
:104C40007A0080B7806880BF8FEF809364008FE721
:104C500080936500789483B7817F846083BF83B736
:104C6000816083BF889583B78E7F83BF1092640075
:104C7000109265008AB1806A8AB98DB1806C8DB955
:104C80000E94BC0980919B11882329F00E94C105D4
:104C900089E00E948B0608951F920F920FB60F9223
:104CA0000BB60F9211242F933F934F935F936F9303
:104CB0007F938F939F93AF93BF93EF93FF938091D5
:104CC000DA0080FF31C08091D80080FF2DC08EEFC8
:104CD0008093DA008091D90080FF19C081E0809331
:104CE000B0148091D3069091D40682609093D4063C
:104CF0008093D3068091E20088608093E2000E9456
:104D000094298091E0008E7F8093E0000DC0109286
:104D1000B0141092B5148091D3069091D40684609B
:104D20009093D4068093D3068091E10082FF07C060
:104D30008091E20082FF03C08BEF8093E1008091BD
:104D4000E10080FF1FC08091E20080FF1BC08EEF5A
:104D50008093E1008091E20080618093E2008FEE19
:104D60008093E1008091D80080628093D800809188
:104D7000D3069091D40680629093D4068093D30694
:104D80000E9409268091E10084FF1AC08091E20010
:104D900084FF16C08091D8008F7D8093D8008FEE5D
:104DA0008093E1008091E2008F7E8093E200809109
:104DB000D3069091D40680649093D4068093D30652
:104DC0008091E10085FF1AC08091E20085FF16C046
:104DD0008091E2008F7E8093E2008FED8093E1006E
:104DE0008091E2008F7D8093E2008091D3069091C4
:104DF000D40680689093D4068093D3068091E10016
:104E000083FF12C08091E20083FF0EC087EF809382
:104E1000E1000E94E62C8091D3069091D406916027
:104E20009093D4068093D306FF91EF91BF91AF91F9
:104E30009F918F917F916F915F914F913F912F91B2
:104E40000F900BBE0F900FBE0F901F9018950E94F1
:104E5000B0290895E7EDF0E0808181608083808152
:104E60008F7B80838081806880830E94832908955E
:104E70009C01F999FECF1FBA32BD21BD60BD0FB6AE
:104E8000F894FA9AF99A0FBE08958AB1806A8AB99D
:104E90008DB1806C8DB95F985D9A8EB1806C8EB942
:104EA000089581E080930A050895769888EC8093B0
:104EB000AD1408950F931F9380910B05882311F46F
:104EC00084E003C0833009F055C08093E90030913D
:104ED000B9143323E9F08091E80085FF19C0232F2E
:104EE00090E0E92FF0E0E654FB4E80818093F100E2
:104EF0009F5F2150B1F71092B91403C01092F100D6
:104F00003F5F3032D8F38091E8008F778093E800DC
:104F10000E94E20A882371F180910C05882331F107
:104F20008091E80085FF26C081E08093F10010E0C9
:104F300000E00E94E20A882339F0002331F40E9445
:104F4000E70A8093F10003C001E01092F1001F5FB7
:104F50001F3179F7769888EC8093AD148091E80042
:104F60008F778093E80006C00E94E70A0E94E20A59
:104F70008823D1F71F910F9108950F931F93CF931B
:104F8000DF93162F072F0E941A83AB01BC01EA01A1
:104F9000212F302FC9019C0197FF03C03095219527
:104FA0003F4F2F5F3F4F35952795CB01B9010E94A9
:104FB0001A839B012C0F3D1FC901DF91CF911F91D7
:104FC0000F910895AF92BF92CF92DF92EF92FF922E
:104FD0000F931F93DF93CF93CDB7DEB76B970FB6C9
:104FE000F894DEBF0FBECDBF80910B05882311F46E
:104FF00084E003C0833009F07CC08093E900809195
:10500000A5148823D1F0E4E0F2E180E090E0208173
:1050100031818217930708F4C901329622E1E43204
:10502000F207A9F78F3F910541F038F06FEF70E07C
:105030000E940683B62EB39402C0BB24B39404E04E
:1050400012E15CE0C52ED12CCC0EDD1E7601AA2427
:10505000AA948091A514882351F0F8018081918150
:105060006B2D70E00E940683F701608314C0F80185
:1050700066A977A96115710561F020813181C901A7
:10508000880F991F820F931F0E94BD27F70180830D
:1050900002C0F701A0820E5F1F4F0894E11CF11CB3
:1050A000F2E104321F07A9F68091E80085FFFCCFEA
:1050B00080E18093F1008BE08093F1008093F10018
:1050C0008AE18093F1009E01245E3F4FF6018191B9
:1050D0006F018093F100E217F307C1F783E11092AB
:1050E000F1008F5F8032D9F78091E8008F7780934D
:1050F000E8006B960FB6F894DEBF0FBECDBFCF9120
:10510000DF911F910F91FF90EF90DF90CF90BF90B4
:10511000AF9008950F931F938091AD14882321F0D1
:1051200081508093AD1401C0769A8091B514882384
:1051300009F444C080910B05813009F03FC0809193
:105140000A058823F9F08091AE148823D9F082E310
:1051500090E061E577E20E94001010920A050E943B
:105160005B2910C00093E9000E945129882309F4AB
:105170004FC076981093AD140E94E70A90E00E9409
:10518000662902C005E018EC0E94E20A882351F764
:105190000E94DD0A8F3790F40E941029882349F479
:1051A0000DC076981093AD140E9432290E94320BE4
:1051B00001C018EC8091AF14882399F78091B51441
:1051C000882331F180910B05882311F58091DE064B
:1051D0008823E1F05F985D9A8EB1806C8EB98091E2
:1051E000E00081608093E0008FE090E065E30E9442
:1051F00038272CE088E190E00FB6F894A8958093CA
:1052000060000FBE20936000F894FFCF0E945A27E1
:105210001F910F9108951092AE141092AF1408953B
:105220008091AF148823C9F486E08093E9008091CF
:10523000E80082FF12C08091F3008091F200809319
:10524000AF14882351F48091E8008B7F8093E800AD
:105250008091E8008F778093E8008091AF148111EE
:1052600081E0089586E08093E9008091AF1488235F
:1052700019F40E941029FBCF9091F1008091AF1496
:1052800081508093AF14882351F48091E8008B7F84
:105290008093E8008091E8008F778093E800892F61
:1052A00008958091E80090E025E0969587952A95ED
:1052B000E1F78170089585E08093E900E8EEF0E081
:1052C00080818F7780831092AE1408950F931F937F
:1052D000182F092F85E08093E9000E945129882327
:1052E000E1F31093F1008091AE148F5F8093AE14C0
:1052F0008091E80085FD02C00E945B29812F902FDC
:105300001F910F9108957894E8EDF0E080818F76F9
:10531000808380818069808380818F7B808380818E
:1053200081608083789408958EE089BD09B400FE81
:10533000FDCF8091D8008F7D8093D8008091E200CE
:1053400081608093E2008091E20088608093E200B7
:105350000E94E62C8091E0008E7F8093E00008950B
:105360008091D90080FF09C08091B014882329F46E
:1053700081E08093B0140E9494298091D30690918B
:10538000D40690FF10C08091D3069091D4069E7FE2
:105390009093D4068093D30681E08093EA00109224
:1053A000EA001092B5141092E9008091E80083FFA2
:1053B00002C00E941E2C8091F6068823F9F083E03B
:1053C0008093E9008091E80085FF18C081E0809318
:1053D000F1001092F1001092F1001092F100109281
:1053E000F1001092F1001092F1001092F100809102
:1053F000E8008F778093E8001092F6060895909168
:10540000E3008091F1008F779078892B8093E300FF
:105410008091E800877F8093E8008091E8008E7F8C
:105420008093E8008091E80080FFFCCF8091E3004A
:1054300080688093E30008958091E800877F8093DF
:10544000E8008091B5148093F1008091E8008E7F90
:105450008093E8008091E8008F778093E80004C093
:105460008091E80083FD0EC08091E80082FFF8CFB4
:105470008091E8008B7F8093E8008091E8008F772F
:105480008093E80008958091F1008091F100E0910F
:10549000F1008091DD06813821F0823851F08038AA
:1054A000B1F48091E800877F8093E8001092F100CA
:1054B00019C08091E800877F8093E800F0E0EF77E3
:1054C000F070EA52F94F80818093F1000BC0809117
:1054D000EB0080628093EB008091E800877F8093EF
:1054E000E80008951092F1008091E8008E7F80938B
:1054F000E80004C08091E80083FD0EC08091E800C0
:1055000082FFF8CF8091E8008B7F8093E800809144
:10551000E8008F778093E80008958091DD06813060
:1055200049F18230E1F58091F1009091F1008823FA
:1055300061F5E091F100EF77E9F0E093E900809107
:10554000EB0080FF15C08091EB0080628093EB0040
:105550001092E900F0E0EA52F94F81E080838091F7
:10556000E800877F8093E8008091E8008E7F0AC082
:105570001092E9008091EB0080628093EB008091B3
:10558000E800877F8093E80008958091EB008062B7
:105590008093EB008091E800877F8093E800089576
:1055A0008091DD068823E9F18130D9F1823009F05C
:1055B0004DC08091F1009091F1008823E9F5E091D0
:1055C000F100EF77E093E9008091EB0080FF27C0C6
:1055D000EE23B1F08091EB0080618093EB0081E0DD
:1055E00090E00E2E02C0880F991F0A94E2F7809374
:1055F000EA001092EA008091EB0088608093EB0053
:105600001092E900F0E0EA52F94F10828091E80030
:10561000877F8093E8008091E8008E7F0AC0109217
:10562000E9008091EB0080628093EB008091E800BC
:10563000877F8093E80008958091EB0080628093DB
:10564000EB008091E800877F8093E8000895EBEEFF
:10565000F0E0808180628083E8EEF0E08081877FE7
:10566000808308958091E800877F8093E80080918F
:10567000E8008E7F8093E8008091E80080FFFCCFF7
:105680000895DF93CF9300D0CDB7DEB71092D50643
:105690006091F1008091F1001092B8141092B7144B
:1056A0001092B2141092B114813019F0823099F432
:1056B00007C00E94132D8093B6140E94FE2C06C0D2
:1056C0000E942A2D8093B6140E94152D9093B81431
:1056D0008093B7140DC00E941533882349F480913C
:1056E000EB0080628093EB008091E800877F80C0B0
:1056F0008091F1008091F1008091F1008983809187
:10570000F1008A838091E800877F8093E8002981F7
:105710003A818091B61490E08217930758F48F7302
:105720009070892B21F481E08093D50637C01092C8
:10573000D50634C02093B61431C08091E80080FFB4
:10574000FCCF20E022C0203421F1E091B714F09189
:10575000B814309749F03196F093B814E093B71429
:10576000319784918093F100E091B114F091B214DB
:10577000309739F081918093F100F093B214E09367
:10578000B1142F5F91509093B6149091B614992351
:10579000D1F68091E8008E7F8093E8008091B61466
:1057A000882321F08091E80082FFC7CF8091E80034
:1057B00082FD16C08091D506813071F48091E80099
:1057C00080FFFCCF8091E8008E7F8093E80004C0CA
:1057D0008091E80083FD0EC08091E80082FFF8CF41
:1057E0008091E8008B7F8093E8008091E8008F77BC
:1057F0008093E8000F900F90CF91DF9108959091E2
:10580000F100923080F48091E800877F8093E80077
:105810009093B5148091E8008E7F8093E800892FE3
:105820000E94813208958091EB0080628093EB00AA
:105830008091E800877F8093E80008959091F100BF
:105840009093DD066091F1006630D9F0673058F42E
:105850006130B9F1613008F444C06330D1F1653092
:1058600009F058C01EC0693021F16A3020F4683058
:1058700009F050C00EC06A30F1F16B3009F04AC037
:1058800044C0903819F40E94412B0895892F66E096
:1058900039C0903819F40E941C2A0895892F68E0B5
:1058A00031C0992319F40E94FF290895892F65E0DA
:1058B00029C0992319F40E94FF2B0895892F69E0CC
:1058C00021C0933018F40E94D02A0895892F61E0F6
:1058D00019C0933018F40E948D2A0895892F63E02F
:1058E00011C0892F8058833018F40E94432A0895EC
:1058F000892F60E007C0913819F40E94272B089582
:10590000892F6AE00E94AC330895913091F40E948F
:10591000322B0895892F0E94AC33882351F4809153
:10592000EB0080628093EB008091E800877F80939A
:10593000E80008959091EB0091609093EB008093C4
:10594000EC008091ED008270862B8093ED008091B9
:10595000ED0082608093ED008091EE00881F882723
:10596000881F08959091F40080E090FD06C08F5F3D
:10597000873011F09695F9CF80E00895FB01809370
:10598000E90004C081918093F10041508091E800CA
:1059900085FF02C04423B1F7842F0895FB01809353
:1059A000E90004C08091F100819341508091E800AA
:1059B00085FF02C04423B1F7842F08958093E90046
:1059C000EBEEF0E080818062808308958091D800C2
:1059D0008F7B8093D8008091D90081FF0DC01092F9
:1059E000E9008091EB0080FD07C01092E90082E0A1
:1059F00060E30E949A2C089580E0089580910B0541
:105A0000813019F420E634E00CC0882319F425EB2A
:105A100034E007C0833019F020E635E002C025EB02
:105A200035E0C901089582E1089580910B05813028
:105A300019F422E734E00CC0882319F427EC34E091
:105A400007C0833019F022E735E002C027EC35E0CB
:105A5000C901089580910B05813041F0882311F42C
:105A600084E60895833011F489E3089583E408956A
:105A70008091E800877F8093E8008091A61480934E
:105A8000F1008091A7148093F1008091A814809375
:105A9000F1008091A9148093F1008091AA14809361
:105AA000F1008091AB148093F1008091AC1480934D
:105AB000F1008091E8008E7F8093E8008091E800FB
:105AC00080FFFCCF8091E80082FFFCCF8091E8004E
:105AD0008B7F8093E8008091E8008F778093E800C7
:105AE00008958091E800877F8093E8008091E80026
:105AF00082FFFCCF8091F1008093A6148091F10089
:105B00008093A7148091F1008093A8148091F100F4
:105B10008093A9148091F1008093AA148091F100E0
:105B20008093AB148091F1008093AC148091E800D5
:105B30008B7F8093E8008091E8008F778093E80066
:105B40008091E8008E7F8093E8008091E80080FFDC
:105B5000FCCF08958091E800877F8093E8008091D2
:105B6000E8008E7F8093E8008091E80080FFFCCF02
:105B7000089585E38093B6148BE295E09093B81472
:105B80008093B7148091E800877F8093E8006633A4
:105B9000710528F04091B6142BE235E01CC06093EB
:105BA000B614F8CF8091E80080FFFCCFF90190E0B7
:105BB0000AC0542F5150903449F09F5F84918093D4
:105BC000F1003196452F9F01442399F78091E80019
:105BD0008E7F8093E800442359F08091E80082FF93
:105BE000E1CF3093B8142093B7144093B61406C095
:105BF0003093B8142093B7141092B6148091E80033
:105C000082FF0FC08091E8008B7F8093E800809135
:105C1000E8008F778093E80008958091E80083FD85
:105C20000EC08091E80082FFF8CF8091E8008B7F62
:105C30008093E8008091E8008F778093E8000895D2
:105C40008091E800877F8093E8006093DF06809171
:105C5000E8008E7F8093E8008091E80080FFFCCF11
:105C600008958091E800877F8093E800452B71F0CC
:105C70008091DF068093F1008091E8008E7F809311
:105C8000E80004C08091E80083FD0EC08091E80028
:105C900082FFF8CF8091E8008B7F8093E8008091AD
:105CA000E8008F778093E8000895982F8091E800AE
:105CB000877F8093E800913011F490E205C0933023
:105CC00011F494E001C090E0452B91F0992381F00C
:105CD00080E01092F1008F5F8917D8F38091E8007F
:105CE0008E7F8093E8008091E8008F778093E800B2
:105CF000089589E08093B6148BE195E09093B814F1
:105D00008093B7148091E800877F8093E8006A3021
:105D1000710528F04091B6142BE135E01CC060936A
:105D2000B614F8CF8091E80080FFFCCFF90190E035
:105D30000AC0542F5150903449F09F5F8491809352
:105D4000F1003196452F9F01442399F78091E80097
:105D50008E7F8093E800442359F08091E80082FF11
:105D6000E1CF3093B8142093B7144093B61406C013
:105D70003093B8142093B7141092B6148091E800B1
:105D800082FF0FC08091E8008B7F8093E8008091B4
:105D9000E8008F778093E80008958091E80083FD04
:105DA0000EC08091E80082FFF8CF8091E8008B7FE1
:105DB0008093E8008091E8008F778093E800089551
:105DC000DC01FC0120E030E029C0109721F0809137
:105DD000F100819302C08091F10041505040615028
:105DE0002F5F3F4F6623D1F441155105B9F08091E3
:105DF000E8008B7F8093E8008091E8008F778093A4
:105E0000E8008091E80082FFFCCF6091F2006623F9
:105E100029F466277727621B730B04C041155105CF
:105E2000A1F670E0CB0108952F923F924F925F92BE
:105E30006F927F928F929F92AF92BF92CF92DF929A
:105E4000EF92FF920F931F93DF93CF93CDB7DEB7FF
:105E5000A1970FB6F894DEBF0FBECDBF6C01B62E72
:105E600083E0861708F0ACC2F6019081992309F40B
:105E7000A7C29130C1F480910C05882309F4A0C217
:105E8000E62EEA948601FF24F3940AC0F80181818A
:105E90000F5F1F4F882309F493C20E94320BF394C3
:105EA000FE14A0F38DC2903109F065C18091B91440
:105EB000882309F085C29093BA1481E08093B914C5
:105EC00001E0F4E13F2EE3E12E2E72E1672E61E165
:105ED000562E50E1452E47E0A42E39E7E32EF12C53
:105EE0009924939488248A9425E0722EF601E00F79
:105EF000F11D9081963009F44EC0973038F49430FB
:105F000089F0953070F5992359F029C1983009F43A
:105F1000C5C0983008F484C09B3008F020C1D6C0BA
:105F20000B2D1DC18091B9148F3108F018C1E82FD5
:105F3000F0E0E654FB4E90838F5F90919B11A82F69
:105F4000B0E0E82FEF5F992331F0A654BB4E80916B
:105F5000A7118C9303C0A654BB4E8C92E093B91446
:105F6000FEC08091B9148E3108F0F9C0E82FF0E03E
:105F7000E654FB4E70828F5FE82FF0E0E654FB4E54
:105F800090919E1190838F5FE82FF0E0E654FB4ED6
:105F900090919F117EC08091B9148F3108F0DFC0BD
:105FA000E82FF0E0E654FB4E9083982F9F5F80919E
:105FB000AC11882381F480910D05A92FB0E0E92F61
:105FC000EF5F882321F0A654BB4E4C92C7CFA65456
:105FD000BB4E5C92C3CF813051F480910D05882374
:105FE000C1F4E92FF0E0E654FB4E608217C0823026
:105FF00081F480910E05A92FB0E0E92FEF5F88238F
:1060000021F4A654BB4E2C92A9CFA654BB4E3C9271
:10601000A5CFE92FF0E0E654FB4E10829F5F9DC0B4
:106020008091B9148A3108F09AC0E82FF0E0E65464
:10603000FB4EA0828F5FE82FF0E0E654FB4E90917C
:10604000430590838F5FE82FF0E0E654FB4E90917C
:10605000440590838F5FE82FF0E0E654FB4E90916B
:10606000450590838F5FE82FF0E0E654FB4E90915A
:10607000460590838F5FE82FF0E0E654FB4E909149
:10608000470590838F5FE82FF0E0E654FB4E909138
:10609000480590838F5F8093B91461C01091B91443
:1060A0001F3108F05CC0E12FF0E0E654FB4E908316
:1060B0001F5F1093B9140E940008E12FF0E0E6542E
:1060C000FB4E80831F5F1093B91449C08091B914AF
:1060D0008F3008F044C0E82FF0E0E654FB4E908388
:1060E000482F4F5F4093B91420E030E0993011F40D
:1060F00021E030E02E9DF0012F9DF00D3E9DF00D32
:106100001124E851F44E8081A42FB0E0E42FEF5F1A
:106110008F3F21F0A654BB4E9C9203C0A654BB4EA9
:106120001C92E093B9149091B9142E9DD0012F9D2B
:10613000B00D3E9DB00D1124A852B44E20E030E0C9
:10614000E92FE20FF0E0E654FB4E8D9180832F5F44
:106150003F4F20313105A1F7905F9093B9140F5F45
:106160000B1508F4C3CE8091B914813009F028C111
:106170001092B91425C1913109F01DC111E001E05F
:1061800093E0692E712C6C0E7D1E88E0482E512CF8
:106190004C0E5D1E4E010894811C911CF601E10F0E
:1061A000F11DE081E430E9F0E53040F4E13089F0C0
:1061B000E13068F0E23009F0F2C009C0E63009F4DD
:1061C00050C0E63030F1E73009F0E9C0CEC01B2DF9
:1061D000E6C01F5FF601E10FF11D808180930C0581
:1061E000DEC01F5FF601E10FF11D80810E94630C8C
:1061F00080919E1190919F119A8389838091A7111C
:106200000E94630C89819A810E9461128EE596E05A
:1062100023C0912F9F5FF601E90FF11D8081F401EA
:1062200080831E5FF601E10FF11D8081F4018183FF
:106230008091A7110E94630C89819A810E9461124A
:106240006091A0117091A11180919E1190919F1168
:106250000E941B6A8DE496E00E94840B00939B11C0
:106260009EC01F5FD301EBE0F5E085E001900D9249
:106270008150E1F7FD80D201E3E9F1E18AE101908B
:106280000D928150E1F7E9A0F601E10FF11DE081E7
:10629000E33131F482E00E94A12410920E0507C080
:1062A000E43141F482E00E94A12400930E05109293
:1062B0000D0529C0E23111F481E0F5CFE13111F48F
:1062C00080E0F1CFE53151F483E00E94A1241092E7
:1062D0000D0510920E051092A51415C0E63151F46B
:1062E00083E00E94A12410920D0510920E050093E8
:1062F000A51409C0EE2339F080E00E94A124009388
:106300000D0500930E0580910D058F1549F48091C0
:106310000E058F1529F48091AC118E1509F43FC03C
:1063200080919E1190919F119A8389838091A711EA
:106330000E94630C89819A810E9461120E94B86A4E
:1063400080E090E00E945D6A6091A0117091A111BF
:1063500080919E1190919F110E941B6A8091AC11B7
:106360000E94A12484E396E077CF8091B9148A310A
:10637000B0F41F5FF601E10FF11D808180934305AA
:10638000808180934405808180934505808180933E
:1063900046058081809347058081809348051F5F73
:1063A0001B1508F4FBCE8091AC11823049F486E0D5
:1063B0000E948B0605C0983A19F481E08093DE06AE
:1063C000A1960FB6F894DEBF0FBECDBFCF91DF917F
:1063D0001F910F91FF90EF90DF90CF90BF90AF9003
:1063E0009F908F907F906F905F904F903F902F90F5
:1063F0000895DF93CF9300D000D0CDB7DEB7809162
:10640000E800877F8093E8008091E8008E7F80938A
:10641000E80004C08091E80083FD28C08091E80076
:1064200082FFF8CF8091F10089838091F1008A8307
:106430008091F1008B838091F1008C838091E80042
:106440008B7F8093E8008091E8008F778093E8004D
:106450008091E8008E7F8093E800CE01019664E091
:106460000E94142F8091E80080FFFCCF0F900F90C6
:106470000F900F90CF91DF910895DF93CF93CDB719
:10648000DEB7A0970FB6F894DEBF0FBECDBF8091E8
:10649000E800877F8093E80004C08091E80083FDD6
:1064A00027C08091E80082FFF8CFFE0131969E015F
:1064B0002F5D3F4F8091F1008193E217F307D1F7F1
:1064C0008091E8008B7F8093E8008091E8008F77CF
:1064D0008093E8008091E8008E7F8093E800CE01F1
:1064E000019660E20E94142F8091E80080FFFCCFAB
:1064F000A0960FB6F894DEBF0FBECDBFCF91DF914F
:106500000895FF920F931F9380910B05823011F035
:10651000882319F583E08093E90081EC60E30E9411
:106520009A2C81E08093E90081E864E30E949A2C30
:1065300012E01093E90080E864E30E949A2C88E05E
:106540008093EA001092EA001093EA001092EA00A9
:1065500084E08093EA001092EA0080910B05882382
:1065600079F484E08093E90081EC64E20E949A2C43
:1065700080E18093EA001092EA0082E08093E006D6
:1065800080910B05813021F584E08093E90081EC56
:1065900060E20E949A2C85E08093E90081E860E245
:1065A0000E949A2C86E08093E90080E864E20E94D1
:1065B0009A2C80E18093EA001092EA0080E28093B6
:1065C000EA001092EA0080E48093EA001092EA0068
:1065D00000910B05033029F5FF24F394F092E900B4
:1065E00081E864E30E949A2C12E01093E90080E8AD
:1065F00064E30E949A2C0093E90081EC60E20E941F
:106600009A2C1093EA001092EA0084E08093EA004A
:106610001092EA0088E08093EA001092EA00F0927B
:10662000E0061F910F91FF9008959F92AF92BF9245
:10663000CF92DF92EF92FF920F931F93833009F076
:1066400080C0613071F0613030F0623081F06330D1
:1066500009F077C016C084E08093B61480E396E01A
:106660000BC08CE08093B61480E096E005C084E215
:106670008093B6148CE096E09093B8148093B7148E
:106680005EC010919311B0909411A09095119090CC
:106690009611609197117091981180919911909134
:1066A0009A112DB73EB72C5030400FB6F8943EBF2C
:1066B0000FBE2DBFEDB6FEB60894E11CF11CA1EE95
:1066C000CA2EA6E0DA2EEDB7FEB7D282C18226E34B
:1066D00035E0F70133832283212F3B2D4A2D592D9D
:1066E00000E20E94807FC901BA01F70124839583EB
:1066F000468377831087B186A28693860E943C8169
:10670000F601A2E1B5E02DB73EB7245F3F4F0FB6CB
:10671000F8943EBF0FBE2DBF8191992787FD9095BC
:106720008D939D9336E0E33FF307B1F786E28093C4
:10673000B61480E195E09093B2148093B11481E097
:1067400001C080E01F910F91FF90EF90DF90CF90FC
:10675000BF90AF909F900895DF93CF9300D000D06B
:10676000CDB7DEB7582FA091F1007091F100809164
:10677000F10089838091F1008A838091F1008B83FD
:106780008091F1008C835A9A5A9840910B054423CA
:1067900011F04230B9F4513211F0513A89F4898143
:1067A0009A81892B69F4662319F0613049F405C098
:1067B0008B819C810E94B73B76C00E94DB3673C000
:1067C000442319F0433009F05AC05138D9F42981D3
:1067D0003A818091E00690E02817390799F46630F5
:1067E00089F4713219F0723269F406C06B817C81D0
:1067F000C9010E94792E51C06B817C81C9010E9420
:10680000B92D4BC0442311F04330C9F5513211F07A
:10681000513AA9F5E981FA818091E00690E0E81704
:10682000F90769F5623021F1633018F4613039F508
:1068300018C0693019F06A3011F50BC0723019F0C8
:106840007330E9F403C00E943D3227C00E94F93141
:1068500024C02B813C818A2F672FAF010E94202EFC
:106860001CC04B815C81872FBF010E94552E15C033
:106870004B815C818A2FBF010E94312E0EC04130B6
:1068800089F4613229F0623251F0603259F403C068
:106890000E94382D02C00E94712D81E004C00E9428
:1068A000AA2DFBCF80E00F900F900F900F90CF910B
:1068B000DF9108955D988AE08093DB1408957798BE
:1068C0008AE08093DA140895FF920F931F93CF9379
:1068D000DF938C01EB01F42E8091C815823011F00A
:1068E00080E0A0C081E090E0A0E0B0E08093DC1404
:1068F0009093DD14A093DE14B093DF1484E290E053
:10690000A0E0B0E08093E4149093E514A093E61423
:10691000B093E714CB01A0E0B0E08093E81490932B
:10692000E914A093EA14B093EB141092F0141092AF
:10693000F1141092F2141092F3141092EC141092BD
:10694000ED141092EE141092EF141092F4141092B1
:10695000F5141092F6141092F7141092F814109285
:10696000F9141092FA141092FB141092FC14109265
:10697000FD141092FE141092FF1410920015109244
:106980000115109202151092031510920415109221
:10699000051510920615109207158C96A11DB11DB4
:1069A0008093E0149093E114A093E214B093E31465
:1069B00081E08093E9008091E8008F778093E80080
:1069C0008091E80085FFFCCFECEDF4E181918093AC
:1069D000F10085E1E830F807C9F718C0F8018081B7
:1069E0008093F1008091E80085FD09C08091E80066
:1069F0008F778093E8008091E80085FFFCCFFF202F
:106A000011F00E945F340F5F1F4F2197209731F7DD
:106A10008091E8008F778093E8008091E80085FFFF
:106A2000FCCF81E0DF91CF911F910F91FF900895EE
:106A3000DF92EF92FF920F931F93DF93CF9300D0DB
:106A400000D0CDB7DEB7FC01D42E8091B5148823D9
:106A500009F45AC09B012C5F3F4F81E08093E9000D
:106A60008091E80085FFFCCF2093F100832F8F7386
:106A70008093F10012C081918093F10061507040C9
:106A80008091E80085FD09C08091E8008F778093B0
:106A9000E8008091E80085FFFCCF6115710559F78A
:106AA0008EED89838DEA8A838EEB8B838FEE8C83C8
:106AB0008E010F5F1F4F85E0E82EF12CEC0EFD1EBE
:106AC000F80180818093F1008091E80085FD09C084
:106AD0008091E8008F778093E8008091E80085FF3F
:106AE000FCCFDD2011F00E945F340F5F1F4F0E15A9
:106AF0001F0531F78091E8008F778093E80080913F
:106B0000E80085FFFCCF81E00F900F900F900F9071
:106B1000CF91DF911F910F91FF90EF90DF9008953B
:106B20009C0180910F05813081F080910B058330AD
:106B300021F4C9010E9418350895823011F088238C
:106B400021F4C9010E946434089580E008951F93E0
:106B5000CF93DF938091DB14882321F081508093C1
:106B6000DB1401C05D9A8091DA14882321F08150F2
:106B70008093DA1401C0779A8091B514882309F4C0
:106B80006DC080910B05833009F068C080914F057E
:106B9000882331F089E495E00E945D6A10924F05E8
:106BA0005F9A82E08093E9008091E80082FF56C0FE
:106BB0008091D9159091DA15892B09F04FC08091F9
:106BC000AC11823009F44AC06091F200623068F082
:106BD0002091F1002093DC148091F1008093DD146A
:106BE000162F1250882364F439C08091E8008B7FFF
:106BF0008093E8008091E8008F778093E800E8CFE9
:106C000090E08F739070D82FCC27822F90E0C82B04
:106C1000D92B209719F10E945A3486E596E1612F0D
:106C2000AE010E94E02E8091E8008B7F8093E80007
:106C30008091E8008F778093E800BE016450704037
:106C400080910F05882331F086E596E140E00E94AF
:106C5000183504C086E596E10E94FF7A8091C81538
:106C6000823009F0A0C080910B05882319F0823092
:106C700009F099C080914F05882331F089E495E0AF
:106C80000E945D6A10924F055F9A82E08093E9004E
:106C90008091E80082FF75C08091D9159091DA1536
:106CA000892B09F06EC08091AC11823009F469C063
:106CB0006091F2006C3210F020E00BC08091E8008F
:106CC0008B7F8093E8008091E8008F778093E800C5
:106CD00021E0ECEDF4E18091F100819385E1E83071
:106CE000F807C9F7162F1C528091DC149091DD141F
:106CF000A091DE14B091DF140197A105B10559F000
:106D00008091E8008B7F8093E8008091E8008F7786
:106D10008093E80022E08091E8149091E914A0911A
:106D2000EA14B091EB140097A105B10551F12223AB
:106D300041F50E945A344091E4145091E5144452B4
:106D4000504080E090E0612F0E94E02E4091E814D6
:106D50005091E91486E596E1612F0E94E02E809122
:106D6000E8008B7F8093E8008091E8008F77809324
:106D7000E8006091E8147091E91486E596E10E94BC
:106D8000FF7A8091AC11823071F48091E80082FF2B
:106D90000AC08091E8008B7F8093E8008091E80032
:106DA0008F778093E800DF91CF911F91089581E064
:106DB0008093F60608958091E800877F8093E8002D
:106DC0009091F706392FE0E01DC08091E80080FF28
:106DD000FCCF2E2F5E2F505C0DC0432F4150251746
:106DE00059F0E22FF0E0E45EFA4E80818093F100EA
:106DF0002F5F342F332389F78091E8008E7F8093B3
:106E0000E800E22F332339F08091E80082FFDDCFE4
:106E10003093F70602C01092F7068091E80082FFD7
:106E20000CC08091E8008B7F8093E8008091E8009F
:106E30008F778093E80081E00895892F90E08F7329
:106E40009070892B81F48091E80080FFFCCF8091C5
:106E5000E8008E7F8093E80006C08091E80083FF01
:106E600002C080E008958091E80082FFF6CF809113
:106E7000E8008B7F8093E8008091E8008F77809313
:106E8000E80081E008959B01AC018091E80080FF5B
:106E90004CC08091F706882309F047C087E090E056
:106EA000A0E0B0E080931C1590931D15A0931E15D3
:106EB000B0931F1584E190E0A0E0B0E0809320152E
:106EC00090932115A0932215B09323152093241598
:106ED000309325154093261550932715ECE1F5E1E5
:106EE00081918093F10085E1E033F807C9F7809143
:106EF000E8008E7F8093E8008091E80080FFFCCF5F
:106F000004C08091E80083FD10C08091E80082FFFA
:106F1000F8CF8091E8008B7F8093E8008091E800B3
:106F20008F778093E80081E0089580E008950895C8
:106F3000A0913015B0913115FD01EC5DFA4E248120
:106F4000358146815781233331054105510510F0C4
:106F500082E303C0822F01C082501816ECF3209107
:106F600028153091291540912A1550912B152B3158
:106F700082E0380781E0480780E0580709F480C0C4
:106F80002C3182E0380781E0480780E05807C0F4E0
:106F90002F3081E0380781E0480780E0580709F486
:106FA0006FC0223181E0380781E0480780E0580750
:106FB00009F466C02E50314041405040D1F517C011
:106FC000213081E0380781E048078DE0580741F122
:106FD000223081E0380781E048078DE0580709F446
:106FE0004FC0235031404140514019F549C0AC5D7C
:106FF000BA4E8D919D910D90BC91A02D8093F80675
:107000009093F906A093FA06B093FB060097A105AA
:10701000B10511F082E001C081E08093C81530C055
:10702000AC5DBA4E8D919C91909359058093580513
:1070300027C085E090E0A0E0B0E880931C15909315
:107040001D15A0931E15B0931F1520E130E040E000
:1070500050E0209320153093211540932215509332
:10706000231581E090E0A0E0B0EC80932815909388
:107070002915A0932A15B0932B152093F706089590
:1070800085E090E0A0E0B0E880931C1590931D157A
:10709000A0931E15B0931F1580E190E0A0E0B0E032
:1070A0008093201590932115A0932215B09323155A
:1070B000109228151092291510922A1510922B154E
:1070C0008093F7060895ECE1F5E184E090E0A0E01C
:1070D000B0E880931C1590931D15A0931E15B093D6
:1070E0001F1584E090E0A0E0B0E080932C15909311
:1070F0002D15A0932E15B0932F1580E190E0A0E000
:10710000B0E08093301590933115A0933215B09371
:1071100033158091281590912915A0912A15B091C9
:107120002B15853021E0920722E0A20720E0B2076C
:1071300009F4DCC2863021E0920722E0A20720E0B9
:10714000B20708F0BFC08D3021E0920721E0A2070E
:1071500020E0B20709F4C8C18E3021E0920721E097
:10716000A20720E0B20708F049C0863021E092076C
:1071700021E0A20720E0B20709F4A2C1873021E094
:10718000920721E0A20720E0B207F8F4823021E064
:10719000920721E0A20720E0B20709F4A7C28330DA
:1071A00021E0920721E0A20720E0B20738F48150E5
:1071B0009140A140B04009F0A2C269C18550914000
:1071C000A140B04008F09BC291C28C3021E09207F0
:1071D00021E0A20720E0B20708F081C18A3021E057
:1071E000920721E0A20720E0B20708F073C18750A0
:1071F0009140A140B04009F082C267C1863121E0D0
:10720000920721E0A20720E0B20709F48EC187317E
:1072100021E0920721E0A20720E0B20710F58F30AD
:1072200021E0920721E0A20720E0B20709F482C121
:107230008F3021E0920721E0A20720E0B20708F496
:1072400066C1813121E0920721E0A20720E0B20768
:1072500009F466C184519140A140B04009F04FC289
:1072600045C2823021E0920722E0A20720E0B20767
:1072700009F4FDC1833021E0920722E0A20720E05B
:10728000B20780F4823022E0920721E0A20720E0DA
:10729000B20709F42BC281509140A240B04009F0DE
:1072A0002EC2DCC1833021E0920722E0A20720E059
:1072B000B20709F4EEC184509140A240B04009F0F9
:1072C0001EC2DEC1883021E0920721E0A2072DE036
:1072D000B20709F4F0C0893021E0920721E0A2074B
:1072E0002DE0B20708F06AC0853021E0920721E066
:1072F000A20721E0B20709F4F9C1863021E0920724
:1073000021E0A20721E0B20740F5823021E0920798
:1073100021E0A20721E0B20709F438C1833021E05F
:10732000920721E0A20721E0B20738F48150914092
:10733000A140B14009F0E3C1FDC0833021E09207D4
:1073400021E0A20721E0B20709F441C18450914035
:10735000A140B14009F0D3C13FC1833021E0920781
:1073600022E0A20721E0B20709F4C0C1843021E085
:10737000920722E0A20721E0B20780F4813021E0E9
:10738000920722E0A20721E0B20709F4AFC18250C0
:107390009140A240B14009F0B2C1A8C1813021E0C2
:1073A000920721E0A2072DE0B20709F41AC182502A
:1073B0009140A140BD4009F0A2C136C18E3022E00B
:1073C000920721E0A2072DE0B20709F474C08F30C4
:1073D00022E0920721E0A2072DE0B20740F58B31B1
:1073E00021E0920721E0A2072DE0B20709F463C073
:1073F0008C3121E0920721E0A2072DE0B20738F49A
:1074000088519140A140BD4009F079C154C08430F9
:1074100022E0920721E0A2072DE0B20709F466C13D
:1074200086509240A140BD4009F069C112C1803030
:1074300021E0920721E0A2072DEFB20709F43AC13B
:10744000813021E0920721E0A2072DEFB20778F406
:10745000813122E0920721E0A2072DE0B20759F125
:1074600087519240A140BD4009F049C124C08230FB
:1074700021E0920721E0A2072DEFB20709F42DC108
:1074800086509140A140BD4F09F039C12FC18CE811
:1074900090E0A0E0B0E080932C1590932D15A09380
:1074A0002E15B0932F15CF0148966FE676E04CE885
:1074B00050E00E947E8080E090E0A0E0B0E02BC130
:1074C00080E095E0A0E0B0E0ECC084E690E0A0E0D1
:1074D000B0E0E7C086E690E0A0E0B0E0E2C08FEF69
:1074E0009FEFAFEFB0E0DDC088E090E0A0E0B0E05B
:1074F00080932C1590932D15A0932E15B0932F15D6
:10750000CF01489669E077E048E050E0D2CF809123
:10751000F8069091F906A091FA06B091FB06C1C059
:1075200084E195E0A0E0B0E0BCC080E090E1A0E0A4
:10753000B0E0B7C0109238151092391510923A1574
:1075400010923B1580915505809334158091540518
:10755000809335158091530580933615809152059F
:10756000809337158091510580933815809150058F
:107570008093391580912C1590912D15A0912E1581
:10758000B0912F150296A11DB11D45C0109238155E
:107590001092391510923A1510923B1580915505AD
:1075A000809334158091540580933515809153054F
:1075B000809336158091520580933715809151053F
:1075C00080933815809150058093391520C080E054
:1075D00090E0A0E0BEE065C081E090E0A0E0B0E017
:1075E00060C08091580590915905A0E0B0E080936B
:1075F000341590933515A0933615B0933715109226
:1076000038151092391510923A1510923B1586E0F4
:1076100090E0A0E0B0E080932C1590932D15A093FE
:107620002E15B0932F1547CF8DE090E0A0E0B0E08D
:107630008093341590933515A0933615B093371574
:1076400088E395E16BEF76E04DE050E00E94928098
:1076500032CF8CEE9FEFAFEFBFEF23C08091C91503
:107660009091CA15A091CB15B091CC151AC08091FC
:10767000CD159091CE15A091CF15B091D01511C018
:107680008091D5159091D615A091D715B091D815A8
:1076900008C08091D1159091D215A091D315B091C9
:1076A000D4158093341590933515A0933615B09367
:1076B000371501CF83E090E0A0E0B0E080932C1577
:1076C00090932D15A0932E15B0932F15789683E0E7
:1076D000DF011D928A95E9F7EECE10922C151092DB
:1076E0002D1510922E1510922F15E5CE10923415EF
:1076F000109235151092361510923715DCCE109277
:107700002C1510922D1510922E1510922F1581E028
:1077100090E0A0E0B0EC8093281590932915A093F9
:107720002A15B0932B1580912C1590912D15A091B1
:107730002E15B0912F154896A11DB11D80932015CF
:1077400090932115A0932215B09323154897A10972
:10775000B10941F410923015109231151092321582
:1077600010923315809120158093F706089520918B
:10777000E800277F2093E8009C018D3A910510F0E6
:107780002CEA30E08091E8008F7B8093E800E0E015
:1077900030C08091E8009091E80082FD02C096FF21
:1077A000F8CF8091E80082FF1EC09E2F4E2F405CD4
:1077B0008091F100E92FF0E0E45EFA4E80839F5F54
:1077C00021503040941719F02115310589F7809127
:1077D000E8008B7F8093E8008091E8008F778093AA
:1077E000E800E92F06C08091E8008F7B8093E800D5
:1077F00003C02115310569F68091E8008E7F8093E2
:10780000E80080911C1590911D15A0911E15B09156
:107810001F1584309105A105B10509F4A4C0853078
:107820009105A105B10558F482309105A105B10576
:10783000C1F00397A105B10509F0EFC08AC08630F9
:107840009105A105B10509F494C086309105A10503
:10785000B10508F48BC00897A105B10509F0DDC09A
:10786000B9C082E090E0A0E0B0E880931C1590934E
:107870001D15A0931E15B0931F1524E330E040E0C2
:1078800050E02093201530932115409322155093FA
:10789000231581E090E0A0E0B0E080932C15909358
:1078A0002D15A0932E15B0932F158093301590931E
:1078B0003115A0933215B0933315109228151092FC
:1078C000291510922A1510922B1580933415909338
:1078D0003515A0933615B0933715109238151092C0
:1078E000391510923A1510923B1580933C159093E0
:1078F0003D15A0933E15B0933F158AE395E0A0E0B7
:10790000B0E08093401590934115A0934215B09339
:10791000431583E090E0A0E0B0E08093441590939D
:107920004515A0934615B09347151092481510922F
:10793000491510924A1510924B1510924C15109241
:107940004D1510924E1510924F1581E08093C81579
:107950003EC05F9A5D98779876988091E8008E7F18
:107960008093E800FFCF0E9463385AC00E94983786
:1079700057C01092C81586E090E0A0E0B0E8809370
:107980001C1590931D15A0931E15B0931F1520E193
:1079900030E040E050E020932015309321154093D3
:1079A000221550932315109224151092251510922C
:1079B00026151092271581E090E0A0E0B0E08093BA
:1079C000281590932915A0932A15B0932B15209371
:1079D000F70626C088E090E0A0E0B0E880931C1590
:1079E00090931D15A0931E15B0931F1580E190E094
:1079F000A0E0B0E08093201590932115A09322156C
:107A0000B0932315109228151092291510922A155B
:107A100010922B158093F70603C0779880E00895A5
:107A20008091E80080FFFCCF8091E80082FF0AC0CF
:107A30008091E8008B7F8093E8008091E8008F7749
:107A40008093E8000E94D73681E00895FC015381BD
:107A5000560F5093E015272F33274281420F409352
:107A6000DF15A181A093DE15E081E093DD15842F61
:107A700090E08217930748F48A2F8F5F8093DE157A
:107A8000882319F4EF5FE093DD15852F90E0707087
:107A90008617970790F4842F8F5F8093DF158823D4
:107AA00061F48091DE158F5F8093DE15882329F4C1
:107AB0008091DD158F5F8093DD1508959C01415005
:107AC0005040460F571FFB010EC0708160E081815E
:107AD000DB01A80FB11D2A0F3B1F2A173B0710F42B
:107AE0002F5F3F4F3296E417F50778F3E417F50759
:107AF00049F4908180E0280F391F2817390710F4C6
:107B00002F5F3F4FC9010895AC011092FF0620E09E
:107B100013C0E22FF0E0322F3F5FEE0FFF1FEE5A4F
:107B2000F94E808191818417950729F42093FF06EF
:107B3000118210820895232F223058F32093FF06DC
:107B40000895AC011092FF0620E012C0E22FF0E091
:107B5000322F3F5FEE0FFF1FEE5AF94E8081918169
:107B6000892B29F42093FF06518340830895232F06
:107B7000223060F32093FF060895BC018091F81530
:107B80009091F91544960E94263DE091F815F091E8
:107B9000F9158091DD15848B8091DE15858B8091A0
:107BA000DF15868B8091E015878B0895282F892F0C
:107BB000922F0895AF92BF92CF92DF92EF92FF92F1
:107BC0000F931F93CF93DF93B82EA92E6B010091D3
:107BD0000007109101077CE2E72E0F5F1F4F8DE732
:107BE0000030180710F000E010E1FF2411C0FE9CE7
:107BF000E0011124C650DA4E8DA1882341F0C8015E
:107C00000E94D63D288939892817390731F3F39422
:107C100082E0F81661F700930007109301071092B5
:107C2000FF06C0E0D0E020E03CE216C0239FF00158
:107C30001124E650FA4E85A1882321F42093FF06F3
:107C4000EF010EC0873039F4209721F096A18EA164
:107C5000891708F4EF012F5F223040F32093FF06CD
:107C6000209789F182E08DA380910207888F80910F
:107C70000307898F809104078A8F809105078B8F76
:107C800084EC94E09F8F8E8F99A388A381E090E08D
:107C90009D8F8C8F1FA281E08EA383E08CA31AA2FC
:107CA00080E18BA3C8010E94D63D998B888BDB8A2B
:107CB000CA8ADE012B2D3A2DC901FC0180E1019019
:107CC0000D928150E1F7CE01DF91CF911F910F917D
:107CD000FF90EF90DF90CF90BF90AF9008950F93FB
:107CE0001F9310915A1600E09091FD06091B11098F
:107CF00090915B16090F111D9801280F311DC901C4
:107D00006EE576E140E250E00E945E3D6091FD0646
:107D100070E06258794EA8010E945E3D009719F408
:107D20002FEF3FEF03C00E94D63D9C01C9011F9178
:107D30000F91089581E10E946F3E089586E00E94B0
:107D40006F3E08958AE30E946F3E089580E090E0C0
:107D500066E576E148E250E00E945E3D009719F446
:107D60002FEF3FEF03C00E94D63D9C01C90108954B
:107D70009C01AB0180E090E0B9010E945E3D0E9451
:107D8000D63D0895EF92FF920F931F939C014427D5
:107D90005527F22EE32E00E010E0362F272F40E08B
:107DA00050E0A90133272227E22AF32A042B152BBE
:107DB000B701C8011F910F91FF90EF900895FC014A
:107DC0004091DB155091DC1526E53BE1241B350B7A
:107DD000621773070CF49B011216130664F42093C8
:107DE000581B3093591BE417F50729F0CA01BF014E
:107DF000A9010E94AE80089582E08093FE06A091C2
:107E0000FD062A2F30E0F901E258F94E8181682FF2
:107E100070E0B3E0660F771FBA95E1F7695F7F4FB7
:107E200042E0285D3F4F3CC0F901E80FF91FEA5AD4
:107E3000F94E8081882319F0813019F42EC04F5FEC
:107E40002FC090E0807C90708038910549F0803C94
:107E5000910549F08034910501F54093FE0609C073
:107E60004093FE0608C04093FE0680916E168F3F39
:107E700011F481E00895242F30E040E050E02A0F13
:107E8000311D411D511D285D3F4F4F4F5F4F84E015
:107E900062E00E946A4982E0089581818E5F480F06
:107EA000842F90E0681779070CF0BECF4093FE0650
:107EB00080E008950F931F93CF93DF93C091F8153F
:107EC000D091F915843009F4F5C202E916E1109356
:107ED000F7150093F6151093DC150093DB1583302E
:107EE00069F48DA18F70833011F00C942F488C8D24
:107EF0009D8D892B11F00C942F4894C0823009F08D
:107F000095C01092DA151092D9151092591B109243
:107F1000581B809105078F5F80930507882399F48C
:107F2000809104078F5F80930407882361F4809118
:107F300003078F5F80930307882329F4809102074A
:107F40008F5F809302072DA1273011F0253051F467
:107F50008EA18F5F8EA3883711F00C942F481DA23D
:107F60000C942F48222311F40C942F488C8D9D8D56
:107F7000892B09F452C08EA181508EA38F5F11F01E
:107F80000C942F483FA1383029F02150223048F47A
:107F9000353039F41DA280E88093F1150E94667B8C
:107FA00000C7353010F080E307C083E090E002C0E6
:107FB000880F991F3A95E2F78EA38FA18F5F8FA349
:107FC0008DA190E08F7090708330910501F1843025
:107FD00091054CF48130910509F491C4029711F098
:107FE0000C942F480DC08630910509F4EEC68830F8
:107FF000910509F4EAC6049711F00C942F48E5C6E0
:10800000E091FD06F0E0E258F94E15867FC484E069
:108010008093F1150E94667B06C72F70233011F004
:108020000C942F4888E08093F115AFC6853021F578
:10803000E091F415F091F51580899189892B11F45F
:108040000C942F481092F9151092F815C8010C974E
:108050009093F7158093F6159093DC158093DB15BC
:108060001092591B1092581B1092DA151092D915C4
:1080700088E08093F1151CC280915616807F80366F
:1080800009F0EDC790915A1680E020915B16AC0183
:10809000420F511D9A018091D9159091DA158417DC
:1080A000950708F4DCC7285D3F4F3093DA1520931D
:1080B000D91580915E168F3F09F4D1C7C801849706
:1080C00060E840E00E949761892B09F067C0C80111
:1080D00084970E94FC61882309F060C080916E162D
:1080E0008F3F09F058C080916F16823009F053C05D
:1080F0008091701690917116892B09F04CC0809177
:10810000721690917316892B01F5809174169091D7
:108110007516892BD1F48091761690917716892B5C
:10812000A1F48091781690917916892B71F4809141
:108130007A1690917B16892B41F480917C168823C6
:1081400021F480917D16813049F1809172169091D1
:108150007316892B01F58091741690917516892BF1
:10816000D1F48091761690917716892BA1F48091A5
:10817000781690917916892B71F480917A169091E6
:108180007B16892B41F480917C16882321F4809101
:108190007D16823019F00E943E4869C78CE596E151
:1081A0009093F3158093F2151092FD061092FC0641
:1081B000E091F215F091F31580818B3209F44BC0F8
:1081C0008C3248F4863009F4E0C1813109F4B1C041
:1081D000882389F06BC08A3309F474C08B3320F490
:1081E0008C3209F063C03BC78B3309F438C78C333A
:1081F00009F05CC006C08091FC0680FD57C081601C
:1082000009C08091FC0681FF04C086FD4FC08064D8
:1082100001C082608093FC060E94FC3E813009F41C
:108220001EC7813018F0823019F621C72091FD0653
:10823000E22FF0E0CF018258994E9093F31580938E
:10824000F215285FFC018181880F880F880F280FA5
:108250002093FD06ADCF8091FC0682FD27C084608F
:108260008093FC069091FD06E92FF0E0DF01A25813
:10827000B94E13968C911397882349F0BA969F01B3
:10828000442737FD4095542F84E060E018C0B09338
:10829000F315A093F215985FE258F94E8181880F8B
:1082A000880F880F980F9093FD0682CFE655F64110
:1082B0009F01442737FD4095542F84E061E00E94E0
:1082C0006A49D5C60E94A23E8F5F9F4F09F0C7C67C
:1082D000E091FD06F0E0E258F94EE081E538A9F0C2
:1082E000E63818F4E038C9F413C0E73829F0E73865
:1082F00048F0E83891F403C00E94AD5912C00E94C2
:1083000049580FC00E9475510CC00E94565E09C0AA
:108310000E948F130E94494A04C01092DA151092ED
:10832000D9158091D9159091DA15892B09F497C642
:108330009EC68091D9159091DA15C0979093DA1561
:108340008093D91586E896E19093F7158093F615FA
:10835000E091FD06F0E0E258F94E86819781892B85
:1083600031F00E949A3E8F5F9F4F09F078C68AE5F0
:108370009BE19093F5158093F4154BC028893989BA
:108380002115310509F440C08091FD06E82FF0E089
:10839000E258F94E8281938182179307A9F52A89C1
:1083A0003B892115310529F080819181821793073E
:1083B00059F588819981892BE9F48A819B81892BE0
:1083C000C9F48C819D81892BA9F48E819F81892B91
:1083D00089F488859985892B69F48A859B85892B01
:1083E00049F48C859D85892B29F48E859F85892B61
:1083F00009F449C08EE596E1BE0140E150E00E94DB
:10840000A180009709F43FC06996D093F515C093F9
:10841000F415C091F415D091F515BBE1CC38DB070C
:1084200008F4ACCFE091FD06F0E0E258F94E82810D
:108430009381998B888B808191819B8B8A8B2091F2
:10844000F4153091F515C901DC01EEE5F6E180E1A6
:1084500001900D928150E1F782E08093F11586E85A
:1084600096E19093F7158093F6159093DC15809321
:10847000DB158091D9159091DA15C0979093591B0F
:108480008093581B15C01092F9151092F81582E0D0
:108490008093F11586E896E19093F7158093F61591
:1084A0009093DC158093DB151092591B1092581B8A
:1084B0000E942C782091581B3091591B21153105B1
:1084C00009F4CDC5C901C0969093DA158093D915EA
:1084D000285F3F4F30935A16885280935B16A091C5
:1084E000F415B091F51554968C91549780935D16C0
:1084F00081E180935C16E091FD06F0E0E258F94ED0
:10850000348325831782168250968D919C915197C2
:108510009183808352968D919C915397938382830C
:10852000AEE6B6E12091F4153091F515C901FC01D4
:1085300080E101900D928150E1F78EE596E16EE6C3
:1085400076E10E94785F82E996E19093F715809337
:10855000F6158091FD06C82FD0E0C258D94E0E9472
:108560009A3E809590959F838E838091FD06E82F9B
:10857000F0E0E258F94E86819781892B09F065C5B4
:108580008FEF9FEF9783868360C50E949E3E8F5F2B
:108590009F4F09F064C58091FD06082F10E0025836
:1085A000194ECAEFD5E18DA18823D9F0D8011296D2
:1085B0002D913C911397888999892817390789F457
:1085C0002D913C918A899B892817390751F48EE5B2
:1085D00096E1BE0140E150E00E94A180009709F4BD
:1085E000B2C1AC96B6E1C632DB07E9F2E0F2F801BF
:1085F00085858F73823001F582819381909308077E
:10860000809307071092FF0613C0E42FF0E0EE0FEF
:10861000FF1FEE5AF94E209107073091080780811D
:1086200091812817390709F489C04F5F4093FF06ED
:108630004091FF06423048F38091FD06E82FF0E0BC
:10864000DF01A258B94E1D968C911D9782FD07C57A
:1086500084E11D968C931D978CE390E09093DA153E
:108660008093D915FD0180E5848797811B968C91B5
:108670001B9717968C931797938796811A968C91D0
:108680001A9716968C9316979287958119968C91C6
:10869000199715968C931597918794819093FF065F
:1086A00018968C91189714968C93149790871B9614
:1086B0008C911B978F5F1B968C931B978823C1F41B
:1086C0001A968C911A978F5F1A968C931A97882313
:1086D00079F419968C9119978F5F19968C93199745
:1086E000882331F418968C9118978F5F18968C9385
:1086F000E091FD06F0E0DF01A258B94E2D913C91CA
:1087000011973093080720930707FD018281938119
:108710009183808313963C932E931297EEE6F6E1B5
:10872000DF01509780E10D9001928150E1F78EE5D5
:1087300096E16EE676E10E94785F54C41092FF06DF
:10874000C0E0D0E04CE250E03CE225C0822F90E057
:10875000849FF001859FF00D949FF00D1124E65049
:10876000FA4E85A1882339F48CE2289FE001112478
:10877000C650DA4E14C0873059F4209721F096A1E4
:108780008EA1891728F4239FE0011124C650DA4EE8
:108790002F5F2093FF062091FF062230B8F220972A
:1087A00009F45DC4D093F915C093F81583E08EA346
:1087B0008CA31AA284E08BA31FA2E091FD06F0E037
:1087C000E258F94E82819381998B888B80819181C7
:1087D0009B8B8A8BDE01EEE5F6E180E101900D9244
:1087E0008150E1F781E08DA380910207888F80910D
:1087F0000307898F809104078A8F809105078B8FEB
:1088000081E090E09D8F8C8FE091FD06F0E0E258D2
:10881000F94E87818F8BE091FD06F0E0E258F94E2A
:1088200086818E8BE091FD06F0E0E258F94E85815D
:108830008D8BE091FD06F0E0E258F94E84818C8B3F
:1088400081E090E00E94BD3DE091FD06F0E0E2583D
:10885000F94E848590E0807F9070813591050CF40D
:108860004EC01092FF0635C0F901EA5AF94E84ADA8
:1088700080930607882309F442C0813021F44F5FBA
:108880004093FF0626C08230C1F485AD8430A9F440
:1088900036AD20E087AD90E0822B932B90930807B4
:1088A00080930707F4E0853C9F0710F084EC94E088
:1088B0009F8F8E8F99A388A322C08091FF06E82FF7
:1088C000F0E0ED56F94EE081EE23C9F0E80FE093B9
:1088D000FF064091FF06242F30E0E091FD06F0E016
:1088E000E258F94E848582958F7090E00597880F45
:1088F000991F880F991F281739070CF4B5CFE091FD
:10890000FD06F0E0E258F94E80E18587E091FD0632
:10891000F0E0DF01A258B94E1D968C911D97826040
:108920001D968C931D97FD0182E0848B84E0858BDE
:10893000868B84EC878B80E490E09093DA158093AB
:10894000D91580E60EC3D093F915C093F81510928F
:10895000F1158091FD06A82FB0E0FD01E258F94E17
:10896000858582FF03C01DA280E293C28485829523
:108970008F70880F880F8093FF062091D915309152
:10898000DA1528523040281B31093093DA1520932C
:10899000D9158DA18F70823039F4A258B94E1D9629
:1089A0008C918F73823139F1232B59F4E091FD06BC
:1089B000F0E0E258F94E858590E083709070892B45
:1089C000D1F08091FD06E82FF0E0E258F94E948155
:1089D0008C89981709F0B2C295818D89981709F092
:1089E000ADC296818E89981709F0A8C297818F89A8
:1089F000981709F0A3C2E091FD06F0E0E258F94EA5
:108A0000858584FF52C06C8D7D8D6115710509F4DB
:108A10004CC0CE0148960E94263D8091FD06E82F6D
:108A2000F0E0E258F94E20858091DD152817E9F530
:108A300091858091DE159817C1F592858091DF159B
:108A4000981799F593858091E015981771F5288FFF
:108A50008091DE15898F8091DF158A8F8091E015D6
:108A60008B8F8FA18823D1F42AA19CA18EA1981B62
:108A7000822F869586958695981B392F320F3AA3BB
:108A80008BA1282F26952695821B97FD9195890FFE
:108A90008BA3369536953695830F8CA381E0809312
:108AA000F1158CA18EA31D8E1C8E8DA1282F30E078
:108AB000C9018F7090708430910509F4EFC1853041
:108AC00091055CF48230910591F1833091050CF0B1
:108AD000CAC0019709F0C3C210C08630910509F4DD
:108AE00025C2863091050CF4FDC18730910509F44B
:108AF00025C2089709F0B3C2C6C18091F11580FF65
:108B0000AEC283E08DA380E48093F1151D8E1C8E90
:108B10002091D9153091DA152115310509F431C1AB
:108B200082E48093F115C9010E94BD3D2AC1809164
:108B3000F11580FF8DC08091FD06E82FF0E0E2582E
:108B4000F94E85858F73823109F082C0848590E06B
:108B5000807F9070813591050CF44EC01092FF0615
:108B600035C0F901EA5AF94E84AD8093060788238F
:108B700009F442C0813021F44F5F4093FF0626C0C4
:108B80008230C1F485AD8430A9F436AD20E087ADE4
:108B900090E0822B932B909308078093070724E0A3
:108BA000853C920710F084EC94E09F8F8E8F99A300
:108BB00088A322C08091FF06E82FF0E0ED56F94E21
:108BC000E081EE23C9F0E80FE093FF064091FF0635
:108BD000242F30E0E091FD06F0E0E258F94E848564
:108BE00082958F7090E00597880F991F880F991FC5
:108BF000281739070CF4B5CF83E08DA3E091FD066B
:108C0000F0E0E258F94E84818C8BE091FD06F0E0B3
:108C1000E258F94E85818D8BE091FD06F0E0E25837
:108C2000F94E86818E8BE091FD06F0E0E258F94E18
:108C300087818F8B81E090E00E94BD3D82E480932C
:108C4000F1151D8E1C8E1092DA151092D91599C04F
:108C500080E28093F1150E94667BE091F815F09117
:108C6000F91515A2E9CC8091FD06E82FF0E0E25855
:108C7000F94E858580FF25C024FD23C08C8D9D8DF8
:108C8000892B09F0ECC18091D9159091DA150196E4
:108C90000E94BD3D2091F115822F80618093F115D6
:108CA0008091D9159091DA15892B19F022612093C2
:108CB000F1150E94667B81E090E09D8F8C8F88E0AB
:108CC00082C085FF25C0328920E0838990E0282B6F
:108CD000392B8091F6159091F715820F931F909381
:108CE000F7158093F615E091FD06F0E0E258F94E95
:108CF000328920E0838990E0282B392B8091D91587
:108D00009091DA15821B930B9093DA158093D91505
:108D10002091D9153091DA152115310559F08DA121
:108D200084FD08C08091F11582608093F115C9011E
:108D30000E94BD3DE091FD06F0E0E258F94E9685B7
:108D400080E02785820F911D909308078093070785
:108D500028A139A12817390710F0892B21F4309365
:108D600008072093070780910707909108079F8FB6
:108D70008E8F8091F11590E083709070892B09F4AB
:108D80006EC11092591B1092581B0E94667B8091F5
:108D9000F115282F85FF0CC01092591B1092581BFB
:108DA0001DA2E091FD06F0E0E258F94E84E1CCC04E
:108DB00084FF12C01092591B1092581B81E090E062
:108DC0009D8F8C8F84E08DA31FA2E091FD06F0E0C3
:108DD000E258F94E81E1B8C08091581B9091591B1F
:108DE000892B01F120FF02C01D8E1C8E8C8D9D8D64
:108DF0000097A1F42E8D3F8D8091581B9091591BA7
:108E00002817390720F43093591B2093581B809161
:108E1000581B9091591B9D8F8C8F04C09093591BA8
:108E20008093581B1FA28091DB159091DC159093C5
:108E3000F7158093F6158091581B9091591B892B3B
:108E400081F08C8D9D8D009761F0CC969093DA1512
:108E50008093D915E091FD06F0E0E258F94E88E1E3
:108E600010C08091F11581FFFAC08CE390E09093DF
:108E7000DA158093D915E091FD06F0E0E258F94E3D
:108E800080E1858768C08091F11580FFE8C01DA250
:108E900080E18093F1150E94667BE1C08091D91535
:108EA0009091DA15009711F00E94BD3DE091FD060A
:108EB000F0E0E258F94E85859091F11580FF0BC0E6
:108EC00090FF06C087E08DA31EA21D8E1C8E1DC0C4
:108ED00086E08DA31AC090FF22C085E08DA31D8E71
:108EE0001C8EBDC08091D9159091DA15009711F0B4
:108EF0000E94BD3DE091FD06F0E0E258F94E858507
:108F000080FF0DC087E08DA31EA281E090E00E944B
:108F1000BD3D80E18093F1150E94667B0FC080917A
:108F2000D9159091DA15892B49F499C08091F115E2
:108F300080FF95C087E08DA31EA291C0E091FD0641
:108F4000F0E0E258F94E80E185878CE390E0909361
:108F5000DA158093D915E091FD06F0E0E258F94E5C
:108F600080E58487E091FD06F0E0E258F94E8C89B7
:108F700080878D8981878E8982878F898387888D75
:108F80008483898D85838A8D86838B8D878386E014
:108F900080935C1688899989918380838A899B89CB
:108FA00093838283AEE6B6E1FE0180E101900D92EB
:108FB0008150E1F78EE596E16EE676E10E94785FFA
:108FC0008DA1E091FD0684FF06C0F0E0E258F94E65
:108FD0001786168607C0F0E0E258F94E84E08687CF
:108FE00084EC87878091E01C90E029E730E0829F45
:108FF000F001839FF00D929FF00D1124EB55F44E7C
:10900000848180935D168091D9159091DA158897A7
:1090100090935A168091D915885280935B16E091EF
:10902000FD06F0E08F010258194ED80153961C92AC
:10903000539752961C92F801118A108A0E949E3E04
:1090400080959095F801918B808B80E680935616E1
:1090500010925716109259161092581608C0109276
:10906000DA151092D9151092FD061092FC06109296
:10907000F115DF91CF911F910F9108951F931091DA
:10908000E01C212F30E089E790E0289FF001299F24
:10909000F00D389FF00D1124EB55F44E8389882391
:1090A00099F180916E168E3F29F480916F16803869
:1090B00019F42AC08F3F41F11092E01C0BC08EE6DC
:1090C00096E10E94FE4E8823C1F48091E01C8F5FE0
:1090D0008093E01C8091E01C823088F327C00E94BE
:1090E000354B892B51F48091E01C8F5F8093E01CFD
:1090F0008091E01C823098F31CC080915D168150F5
:1091000080935D16882329F41092DA151092D915F0
:1091100016C086E596E1489660E840E00E949761B7
:10912000892B69F081E00E945A3F09C01092E01C2F
:10913000DFCF1092DA151092D9151093E01C1F9111
:109140000895EF92FF920F931F93CF93DF938C01BB
:109150007B01C0910007D091010721968DE7C030B7
:10916000D80710F0C0E0D0E1CE010E94D63D9C01AE
:1091700080916A1B90916B1B8217930771F380910A
:10918000831B9091841B8217930739F3C0930007C8
:10919000D09301071092FF0620E049E150E01CC087
:1091A000322F3F5F822F90E0849FF001859FF00D6A
:1091B000949FF00D1124E65AF44E80899189892BF1
:1091C00051F42093FF0689E1289FD0011124A65A6B
:1091D000B44E49F434C0232F223010F32093FF06FD
:1091E000A0E0B0E02CC05096DC9350975196CC9301
:1091F00051975396FC92EE9252970115110531F456
:1092000080E1ED0119928A95E9F707C0ED01F801B7
:1092100080E1019009928150E1F78091E01C90E09B
:1092200029E730E0829FF001839FF00D929FF00DBF
:109230001124EB55F44E848154968C935497CD01B0
:10924000DF91CF911F910F91FF90EF9008950F93B1
:109250000E9467650E94D75080E009C0E82FF0E0C7
:10926000EE0FFF1FEE5AF94E118210828F5F82308F
:10927000A8F320E04CE250E00DC0822F90E0849FE4
:10928000F001859FF00D949FF00D1124E650FA4EE9
:1092900015A22F5F223088F380E094E090930107BD
:1092A0008093000720E049E150E00EC0822F90E05B
:1092B000849FF001859FF00D949FF00D1124E65AD4
:1092C000F44E118A108A2F5F223080F32093FF061C
:1092D0000F910895CF92DF92EF92FF920F931F9319
:1092E000CF93DF93D82EC62E79018A011092FD0606
:1092F000A9E0B7E0EEE6F6E180E101900D92815041
:10930000E1F78091D9159091DA15C0969093DA150E
:109310008093D9158150954030F080E095E090938E
:10932000DA158093D91566E576E14091D91550910B
:10933000DA1540535040CB01C0960E94B78080E6BA
:10934000809356161092571610925916109258166E
:109350008AE380935C168091E01C90E029E730E07E
:10936000829FF001839FF00D929FF00D1124EB5529
:10937000F44E848180935D1680915E1690915F1605
:10938000892B51F58091601690916116892B21F5FA
:109390008091621690916316892BF1F48091641686
:1093A00090916516892BC1F480916616909167168D
:1093B000892B91F48091681690916916892B61F43C
:1093C00080916A1690916B16892B31F480916C16FE
:1093D00090916D16892BD1F0EEE6F6E1DF01509702
:1093E00080E10D9001928150E1F7809109078F3F54
:1093F00091F484E0D81651F422E0C21639F48EE5D7
:1094000096E169E077E00E94785F0EC01092DA156D
:109410001092D91535C0AEE5B6E1E9E0F7E080E19C
:1094200001900D928150E1F7E091FD06CE2FD0E042
:10943000FE01E258F94ED082C182C801B7010E94F4
:10944000C23ECE57D94E688379838A839B838091AD
:10945000D9159091DA15889790935A168896885264
:1094600080935B168091FD06C82FD0E0C258D94E7C
:109470001B821A820E94A23E809590959B838A83CC
:10948000DF91CF911F910F91FF90EF90DF90CF90E0
:10949000089546E556E18091E01C90E029E730E030
:1094A000829FF001839FF00D929FF00D1124EB55E8
:1094B000F44E848180935D1680916E168F3F81F407
:1094C000DA015896FA01389680E101900D928150A8
:1094D000E1F78EE596E16EE676E10E94785F1BC0CB
:1094E000A9E0B7E0FA01389680E101900D92815031
:1094F000E1F7EEE5F6E1DF01509680E10D90019293
:109500008150E1F7AEE6B6E1E9E0F7E080E10190F5
:109510000D928150E1F76091FD06662301F18AE327
:1095200080935C1670E04091D9155091DA15461B76
:10953000570B5093DA154093D91548525040509329
:109540005A16485D5F4F842F885280935B166E5782
:10955000794E4C52504082E896E10E94B7801092BA
:10956000FD0681E880937E1610927F161092811678
:10957000109280160E94A23E80959095909381163D
:109580008093801608952091E01C30E040E0ABE02D
:10959000B0E086E190E0289FB001299F700D389FD0
:1095A000700D11240FC0842F90E08A9FF0018B9FD3
:1095B000F00D9A9FF00D1124E60FF71FEF5DF74FA6
:1095C00012864F5F423078F34093D5080895CF93C9
:1095D000DF93DC011092DB081092DA081092D508B4
:1095E0005091E01C252F30E040E0CBE0D0E086E158
:1095F00090E0289FB001299F700D389F700D1124B5
:1096000029C0842F90E08C9FF0018D9FF00D9C9FCE
:10961000F00D1124E60FF71FEF5DF74F82858823C9
:10962000C1F0808191818A179B0799F44093D508F6
:109630008BE0489FC001112426E1529F9001112424
:10964000820F931F8F5D974F9093DB088093DA080A
:1096500005C04F5F4230A8F24093D5088091DA08E8
:109660009091DB08DF91CF9108950F931F93CF93D3
:10967000DF931092DB081092DA081092D5089091CF
:10968000E01C292F30E086E1989FD001112440E0B2
:1096900050E060E00BE010E086E190E0289FE00100
:1096A000299FD00D389FD00D11242BE035C0862F77
:1096B00090E0809FF001819FF00D909FF00D1124AC
:1096C000EC0FFD1FEF5DF74F8285882321F101909C
:1096D000F081E02D3097F9F0818D882311F08530ED
:1096E00059F441155105B9F4629FA00111244A0FA4
:1096F0005B1F4F5D574F0FC06093D5088BE0689F8D
:10970000C00111248A0F9B1F8F5D974F9093DB0838
:109710008093DA0809C06F5F623048F25093DB082B
:109720004093DA086093D5088091DA089091DB08BD
:10973000DF91CF911F910F910895FC011286019046
:10974000F081E02D818D853009F413A60895FC0188
:1097500081A18D7F81A308952091E01C84E4289F3E
:1097600090011124235B374FC90108956F927F92B6
:109770008F929F92AF92BF92CF92DF92EF92FF9221
:109780000F931F93CF93DF931092DB081092DA08A8
:109790009091E01C292F30E086E1989FE001112490
:1097A00040E050E060E00BE010E086E190E0289FB0
:1097B000D001299FB00D389FB00D11242BE018C0A7
:1097C000862F90E0809FF001819FF00D909FF00D1B
:1097D0001124EA0FFB1FEF5DF74F8285813039F4CA
:1097E000629FA00111244C0F5D1F4F5D574F6F5FAB
:1097F000623030F35093DB084093DA081092D908B6
:109800001092D8081092D5088CE2A82EB12C04E84A
:10981000C02ED12C1CE2712EB4E86B2EA2E08A2E51
:10982000F9E7EF2EF12CE4E09E2EBEC05091E01C33
:10983000252F30E0842F90E08A9DF0018B9DF00D64
:109840009A9DF00D11242C9DC0012D9D900D3C9DE5
:10985000900D1124E80FF91FE75EF84F83A58130C2
:1098600009F09DC0479DE0011124569DC0011124BF
:10987000C80FD91FC75ED84FD093D908C093D80856
:10988000898D8130E9F0813030F0833039F18430D6
:1098900009F085C035C08AA5833010F013A67FC0BB
:1098A000CE0182960E943667892B09F478C04091D8
:1098B000D8085091D90880E090E060E070E03EC0A8
:1098C000CE014A960E943667892B09F468C0E09160
:1098D000D808F091D908818E12A661C0CE014A96AF
:1098E0000E943667892B09F45AC0E091D808F0919C
:1098F000D908918E12A680E090E0BF01AF011EC092
:109900008AA5833070F01AA6CE010E94E74A909390
:10991000DB088093DA08009711F00E949D4B1BA68C
:109920003EC0CE0182960E943667892BC1F14091DC
:10993000D8085091D90880E090E0BA010E944057C1
:109940000091D8081091D9088091E01C90E08E9D7C
:10995000F0018F9DF00D9E9DF00D1124EB55F44EFE
:10996000658576858785908928EE33E040E050E074
:109970000E942D83CA01B90128EE33E040E050E097
:109980000E94DB82AB01BC01C80182960E94506735
:10999000E091D808F091D90882A58F5F82A78091C5
:1099A000D5088F5F8093D5084091D508433008F4DF
:1099B0003DCF1092D7081092D60881E08093D50849
:1099C000C4E4D0E002E214E440C05091E01C252F32
:1099D00030E0842F90E0FC0175E0EE0FFF1F7A95D8
:1099E000E1F7880F991FE80FF91F2C9FC0012D9FE9
:1099F000900D3C9F900D1124E80FF91FE259F74F8D
:109A0000808181FF1DC0409FF0011124519FC00142
:109A10001124E80FF91FE35BF74FF093D708E093A9
:109A2000D60881A180FD0CC0CF0141960E94366707
:109A3000892B31F08091D6089091D7080E94A74BCE
:109A40008091D5088F5F8093D5084091D50842302A
:109A500008F4BBCFDF91CF911F910F91FF90EF9052
:109A6000DF90CF90BF90AF909F908F907F906F903E
:109A70000895AF92BF92CF92DF92EF92FF920F9331
:109A80001F93CF93DF93182FB92EA62E69017A0169
:109A90001092D7081092D60881E08093D508809163
:109AA000E01C90E041E024E430E0829FB001839F1D
:109AB000700D929F700D112419C0242F2F5F842FD9
:109AC00090E0FC0155E0EE0FFF1F5A95E1F7880F7B
:109AD000991FE80FF91FE60FF71FE259F74F808132
:109AE00081FD03C04093D5080CC0422F423028F3BB
:109AF0004093D508423029F40E94508081E0809341
:109B0000D5089091D50882E2989FF00111248091A8
:109B1000E01C24E4829FC0011124E80FF91FE35BDD
:109B2000F74FF093D708E093D608EF01212F3B2D94
:109B3000C901DC0180E10D9009928150E1F7A08A12
:109B4000C114D104E104F10469F0CF014196B701D9
:109B5000A6010E945067E091D608F091D70881A134
:109B60008E7F02C081A1816081A32091E01C30E042
:109B70006091D508862F90E0FC01B5E0EE0FFF1F45
:109B8000BA95E1F7880F991FE80FF91F84E490E078
:109B9000289FA001299F500D389F500D1124E40FDC
:109BA000F51FE259F74F80818260808300FF13C068
:109BB000862F90E0FC0175E0EE0FFF1F7A95E1F72C
:109BC000880F991FE80FF91FE40FF51FE259F74FAF
:109BD0008081846012C0862F90E0FC0135E0EE0F9A
:109BE000FF1F3A95E1F7880F991FE80FF91FE40F5F
:109BF000F51FE259F74F80818B7F80838091D608D3
:109C00009091D708DF91CF911F910F91FF90EF9026
:109C1000DF90CF90BF90AF900895EF92FF920F9397
:109C20001F93CF93DF93EC017A018B011092DB0835
:109C30001092DA081092D5082091E01C30E040E044
:109C4000ABE0B0E086E190E0289FB001299F700D65
:109C5000389F700D112416C0242F2F5F842F90E0A1
:109C60008A9FF0018B9FF00D9A9FF00D1124E60F53
:109C7000F71FEF5DF74F8285882319F44093D508CD
:109C80000FC0422F423040F34093D508423041F498
:109C90000E94508062E070E00E941A838093D50891
:109CA000E091D5088BE0E89FF00111248091E01C41
:109CB00026E1829FC0011124E80FF91FEF5DF74FE5
:109CC000F093DB08E093DA08C193D193CF01B80198
:109CD000A7010E9450672091D50830E04091E01C18
:109CE00050E08BE090E0289FF001299FF00D389F15
:109CF000F00D112486E190E09C01429FC001439F3A
:109D0000900D529F900D1124E80FF91FEF5DF74F52
:109D100081E082878091DA089091DB08DF91CF9112
:109D20001F910F91FF90EF900895EF92FF920F9384
:109D30001F93CF93DF937C011092D7081092D6081F
:109D40001092D5080091E01C202F30E084E490E0D0
:109D5000289FE001299FD00D389FD00D11243EC0CF
:109D6000812F90E0FC01B5E0EE0FFF1FBA95E1F7FF
:109D7000880F991FE80FF91FEC0FFD1FE259F74FED
:109D8000808181FF28C0212F30E0C90175E0880F54
:109D9000991F7A95E1F7220F331F820F931F8C0FC3
:109DA0009D1F835B974FB70140E150E00E94A18067
:109DB000009789F482E2189FC001112424E4029FD5
:109DC00090011124820F931F835B974F9093D708C4
:109DD0008093D60808C01F5F1093D5081091D5084E
:109DE000123008F4BDCF8091D6089091D708DF914A
:109DF000CF911F910F91FF90EF900895EF92FF92F6
:109E00001F93CF93DF937C011092D5088091E01CC3
:109E100090E024E430E0829FE001839FD00D929F88
:109E2000D00D112442C0812F90E0FC01B5E0EE0F6F
:109E3000FF1FBA95E1F7880F991FE80FF91FEC0F84
:109E4000FD1FE259F74F808181FF2CC0212F30E0A8
:109E5000C90175E0880F991F7A95E1F7220F331F2A
:109E6000820F931F8C0F9D1F212F30E0F90155E0C9
:109E7000EE0FFF1F5A95E1F7220F331FE20FF31F7A
:109E8000EC0FFD1FE35BF74F4089469546954695DD
:109E9000835B974FB70150E00E94A180009711F4B7
:109EA00081E009C01F5F1093D5081091D5081230CA
:109EB00008F4B9CF80E0DF91CF911F91FF90EF9030
:109EC0000895AF92BF92CF92DF92EF92FF920F93DD
:109ED0001F93CF93DF936C011092D9081092D8088A
:109EE0001092D5080091E01C202F30E01CE2A12E3A
:109EF000B12C84E890E0289F7001299FF00C389FD6
:109F0000F00C1124E901C154DA4F2FC0812F90E0E9
:109F10008A9D90018B9D300D9A9D300D11242E0D40
:109F20003F1DF901E75EF84F83A58823D9F04881EA
:109F3000C901875D984FB60150E00E94A18000974B
:109F400089F48CE2189FC001112424E8029F90013B
:109F50001124820F931F875E984F9093D9088093A6
:109F6000D80807C01F5F1093D5081091D50813308B
:109F700068F28091D8089091D908DF91CF911F9114
:109F80000F91FF90EF90DF90CF90BF90AF9008952A
:109F9000CF92DF92EF92FF920F931F93CF93DF93B5
:109FA0007C011092D9081092D8081092D50800911F
:109FB000E01C202F30E08CE2C82ED12C84E890E009
:109FC000289FE001299FD00D389FD00D11242CC06F
:109FD000812F90E08C9DF0018D9DF00D9C9DF00DEA
:109FE0001124EC0FFD1FE75EF84F83A58823C9F00D
:109FF000CF01B70140E150E00E94A180009789F4B1
:10A000008CE2189FC001112424E8029F90011124C2
:10A01000820F931F875E984F9093D9088093D8083A
:10A0200007C01F5F1093D5081091D508133080F238
:10A030008091D8089091D908DF91CF911F910F910D
:10A04000FF90EF90DF90CF900895EF92FF920F93E3
:10A050001F93CF93DF93182F092FEB01F42EE22EDD
:10A060001092D9081092D8081092D5082091E01CBF
:10A0700030E040E0ACE2B0E084E890E0289FB0013E
:10A08000299F700D389F700D112416C0242F2F5F4B
:10A09000842F90E08A9FF0018B9FF00D9A9FF00D26
:10A0A0001124E60FF71FE75EF84F83A5882319F404
:10A0B0004093D5080FC0422F433040F34093D5085A
:10A0C000433041F40E94508063E070E00E941A83A4
:10A0D0008093D5084091E01C9091D5088CE2989F20
:10A0E000B001112484E8489FC0011124680F791F32
:10A0F000675E784F7093D9086093D808DB01212FF1
:10A10000302FC901FC0180E101900D928150E1F7EF
:10A11000E42FF0E02097B9F01092D508E154FA4FFF
:10A12000408190E00BC0E92FF0E0DB01AE0FBF1FD4
:10A13000EC0FFD1F808150968C939F5F941798F3CE
:10A140009093D5080CC0E154FA4F40819B01205FE9
:10A150003F4FC90160E070E050E00E94C980E0918B
:10A16000D808F091D908F08EE18ECF014A9640E0F0
:10A1700050E060E070E00E9450678091D8089091B4
:10A18000D908829640E050E060E070E00E9450679D
:10A19000E091D808F091D90812A681E083A7CF01F9
:10A1A000DF91CF911F910F91FF90EF900895309123
:10A1B000E01C432F50E020E0ACE2B0E084E890E007
:10A1C000489FB001499F700D589F700D11240FC01A
:10A1D000822F90E08A9FF0018B9FF00D9A9FF00DE7
:10A1E0001124E60FF71FE75EF84F13A62F5F233009
:10A1F00078F320E0ABE0B0E086E190E0489FB0016A
:10A20000499F700D589F700D11240FC0822F90E050
:10A210008A9FF0018B9FF00D9A9FF00D1124E60F9D
:10A22000F71FEF5DF74F12862F5F223078F320E0A3
:10A2300084E490E0489FB001499F700D589F700DD5
:10A24000112414C0822F90E0FC01B5E0EE0FFF1F37
:10A25000BA95E1F7880F991FE80FF91FE60FF71F6E
:10A26000E259F74F80818D7F80832F5F223050F33A
:10A270002093D50889E790E0489FF001499FF00DB1
:10A28000589FF00D1124EB55F44E8589882361F118
:10A2900084E490E0489FD001499FB00D589FB00DD5
:10A2A0001124FD01E35BF74F8EEF90E891838083EB
:10A2B00013821282158214821782168211861086EA
:10A2C00013861286158614861786168680E4808B80
:10A2D000A259B74F8C9183608C93832F44E650E052
:10A2E00060E070E00E94E9680895AF92BF92CF925B
:10A2F000DF92EF92FF920F931F93CF93DF938091A2
:10A300005D168F3F09F0A7C480915E168E3F09F05D
:10A31000A2C480915F16803809F09DC48091FD062B
:10A32000A82FB0E0FD01E258F94E8181882309F0A1
:10A3300092C4AE57B94E4C91442379F08091E01C01
:10A3400090E029E730E0829FF001839FF00D929F1B
:10A35000F00D1124EB55F44E4483E091FD06F0E03E
:10A36000EE57F94EA480B580C680D780A114B10401
:10A37000C104D10409F448C02091E01C30E04D2D07
:10A38000552766277727BA2DAA2799278827482B8C
:10A39000592B6A2B7B2BD601C50180709070B07051
:10A3A000892F9A2FAB2FBB27482B592B6A2B7B2B3E
:10A3B000C501A0E0B0E08070A070B070BA2FA92FE6
:10A3C000982F8827482B592B6A2B7B2B89E790E005
:10A3D000289FE001299FD00D389FD00D1124CB5527
:10A3E000D44E8D819E81AF81B88584179507A607CD
:10A3F000B70751F04D835E836F8378870E94226098
:10A4000069877A878B879C87E091FD06F0E0EE579D
:10A41000F94EA084B184C284D384A114B104C104D0
:10A42000D104C9F18091E01C90E029E730E0829FDF
:10A43000F001839FF00D929FF00D1124EB55F44E27
:10A440002D2D332744275527BA2DAA27992788274A
:10A45000282B392B4A2B5B2BD601C50180709070BD
:10A46000B070892F9A2FAB2FBB27282B392B4A2B63
:10A470005B2BC501A0E0B0E08070A070B070BA2F77
:10A48000A92F982F8827282B392B4A2B5B2B258720
:10A4900036874787508B1092DE081092DD081092A5
:10A4A000E0081092DF0840E009C0E42FF0E0EE0F72
:10A4B000FF1FEF51F74F118210824F5F4230A8F318
:10A4C0004093ED088CE08093DC086091D915709181
:10A4D000DA1539C0F901EA5AF94E8181882309F465
:10A4E000B8C38081833071F0853039F08130D9F480
:10A4F000F093DE08E093DD0816C0F093E008E093E7
:10A50000DF0811C08091E1089091E208892B19F4CD
:10A51000E0E040E0B1C38091E3089091E408892B2A
:10A5200009F4A8C342E08091DC08E091FD06F0E068
:10A53000EA5AF94EE80FF11D95A5990F990F990F59
:10A54000980F9093DC089091FD068091DC08282FED
:10A5500030E0290F311D245D3F4F2617370708F4DF
:10A56000B9CF4093ED08E091DF08F091E008309713
:10A5700009F441C0E480F580068117818091E01CD8
:10A5800090E029E730E0829FF001839FF00D929FD9
:10A59000F00D1124EB55F44E212F33274427552776
:10A5A000BE2DAA2799278827282B392B4A2B5B2BCE
:10A5B000D801C70180709070B070892F9A2FAB2F8F
:10A5C000BB27282B392B4A2B5B2B00E010E080E0C7
:10A5D0009FEFA0E0B0E0E822F9220A231B23102F0E
:10A5E0000F2DFE2CEE242E293F29402B512B2083AA
:10A5F0003183428353831092ED0862C224813581F6
:10A6000046815781E084F18402851385A52EBB2401
:10A61000CC24DD24B22FAA2799278827A82AB92A73
:10A62000CA2ADB2ADA01C90180709070B070892FC4
:10A630009A2FAB2FBB27A82AB92ACA2ADB2A40E0C7
:10A6400050E0207040705070542F432F322F22273B
:10A65000A22AB32AC42AD52A212F332744275527D3
:10A66000BE2DAA2799278827282B392B4A2B5B2B0D
:10A67000D801C70180709070B070892F9A2FAB2FCE
:10A68000BB27282B392B4A2B5B2B00E010E080E006
:10A690009FEFA0E0B0E0E822F9220A231B23102F4D
:10A6A0000F2DFE2CEE242E293F29402B512BA216D4
:10A6B000B306C406D50608F4FEC180898E3F21F496
:10A6C0008189803809F4F7C1838187FFC7C0CF0132
:10A6D00040960E94954EEC019093E8088093E7081D
:10A6E000E091ED08009709F05DC0F0E0EE0FFF1F6C
:10A6F000EF51F74FC081D181AC80BD80CE80DF802B
:10A70000A114B104C104D10409F4A8C08E01005FF2
:10A710001F4F9FEFA9169FEFB9069FEFC9069FEF46
:10A72000D90691F16D2D7727882799275A2D44272F
:10A7300033272227622B732B842B952BA60195019F
:10A74000207030705070232F342F452F5527622BE7
:10A75000732B842B952B950140E050E020704070C6
:10A760005070542F432F322F2227622B732B842BB0
:10A77000952B28EE33E040E050E00E94DB829B0105
:10A78000AC01C8016A8106C0C8016A8120E030E0DE
:10A7900040E050E000E00E94394D9093E80880933B
:10A7A000E7085CC0F0E0EE0FFF1FEF51F74F01909C
:10A7B000F081E02DA480B580C680D780A114B104BB
:10A7C000C104D10451F0AFEFAA16AFEFBA06AFEF54
:10A7D000CA06AFEFDA0641F403C00E94A74B3EC0A1
:10A7E00089A1816089A33AC06D2D77278827992791
:10A7F0005A2D442733272227622B732B842B952B2A
:10A80000A6019501207030705070232F342F452FF2
:10A810005527622B732B842B952B950140E050E03C
:10A82000207040705070542F432F322F2227622BFC
:10A83000732B842B952B28EE33E040E050E00E94F0
:10A84000DB82AB01BC01CE0141960E945067E091D2
:10A85000E708F091E80881A18E7F81A3E091ED08DF
:10A86000F0E0EE0FFF1FEF51F74F0190F081E02D68
:10A87000838186FF20C184819581A681B78100975D
:10A88000A105B10509F417C1CF014096628141E0ED
:10A890000E949761EC019093EC088093EB08E091A3
:10A8A000ED08009709F4B5C0F0E0EE0FFF1FEF517F
:10A8B000F74F0190F081E02D248135814681578149
:10A8C0002F3FBFEF3B07BFEF4B07BFEF5B0709F41D
:10A8D0009DC0A52EBB24CC24DD24B22FAA27992706
:10A8E0008827A82AB92ACA2ADB2ADA01C901807076
:10A8F0009070B070892F9A2FAB2FBB27A82AB92A46
:10A90000CA2ADB2AC901A0E0B0E08070A070B07054
:10A91000BA2FA92F982F8827A82AB92ACA2ADB2A52
:10A9200021E2A2162CE1B20620E0C20620E0D20607
:10A93000A0F4CE0141960E9420677B018C01C601E4
:10A94000B50128EE33E040E050E00E94DB82E616DD
:10A95000F7060807190708F048C0E091ED08F0E095
:10A96000EE0FFF1FEF51F74F0190F081E02DE480D3
:10A97000F58006811781C090EB08D090EC08612F1C
:10A980007727882799275E2D442733272227622B94
:10A99000732B842B952BA801970120703070507079
:10A9A000232F342F452F5527622B732B842B952B68
:10A9B00000E010E020E03FEF40E050E0E222F32230
:10A9C00004231523102F0F2DFE2CEE246E297F2932
:10A9D000802B912B28EE33E040E050E00E94DB8298
:10A9E000AB01BC01C601419609C08091EB08909172
:10A9F000EC08419640E05DED6DE670E00E94506726
:10AA0000E091EB08F091EC08118E55C081E0898F40
:10AA100052C0F0E0EE0FFF1FEF51F74FC081D18120
:10AA2000AC80BD80CE80DF808E01005F1F4F3FEF86
:10AA3000A3163FEFB3063FEFC3063FEFD30691F1F6
:10AA40006D2D7727882799275A2D442733272227CA
:10AA5000622B732B842B952BA601950120703070EF
:10AA60005070232F342F452F5527622B732B842BA7
:10AA7000952B950140E050E0207040705070542FAD
:10AA8000432F322F2227622B732B842B952B28EEFA
:10AA900033E040E050E00E94DB829B01AC01C80142
:10AAA0006A8106C0C8016A8120E030E040E050E0E1
:10AAB00001E00E9469638091ED088F5F8093ED084B
:10AAC000E091ED08E23058F4F0E0EE0FFF1FEF5197
:10AAD000F74F0190F081E02D309709F08FCD8EE592
:10AAE00096E10E94C84FFC019093E6088093E50828
:10AAF0006091DD087091DE086115710509F43FC0B1
:10AB0000009769F46E5F7F4F8EE596E141E022E0A9
:10AB10000E9425509093E6088093E50830C0818D0F
:10AB2000882311F482E0818F0091DD081091DE0806
:10AB30000E5F1F4FC091E508D091E6086096E09146
:10AB4000E01CF0E0E154FA4FE080C801BE014E2D58
:10AB500050E00E94A180009761F0CE01B8014E2D17
:10AB600050E00E94AE80E091E508F091E60882E0B6
:10AB7000818FE091E508F091E60881E0808FE09117
:10AB8000FD06F0E0EE57F94E82819381E091E508F1
:10AB9000F091E608892B09F44CC0309769F48EE5F2
:10ABA00096E160E070E041E025E00E94255090933E
:10ABB000E6088093E50802C081E0808F8091E50877
:10ABC0009091E6080E94E74ADC019093EA0880939E
:10ABD000E908E091FD060097B9F4F0E0EE57F94E70
:10ABE0009281838128EE33E0829FA001839F500DE4
:10ABF000929F500D112460E070E08091E5089091E3
:10AC0000E6080E940D4E22C0F0E0EE57F94E928108
:10AC1000838128EE33E0829FA001839F500D929F95
:10AC2000500D112460E070E0CD0102960E94506743
:10AC30000DC0309759F0CF010E94E74A9093EA087F
:10AC40008093E908009711F00E949D4B0E94E977DC
:10AC500002C04093ED081092DA151092D915DF91D9
:10AC6000CF911F910F91FF90EF90DF90CF90BF9009
:10AC7000AF900895E1E041E0F0E0EE0FFF1FEF51EB
:10AC8000F74F2A5A394E318320834DCCEF92FF92F1
:10AC90000F931F93DF93CF9300D0CDB7DEB7E09132
:10ACA000E01CF0E0E154FA4F2081822F90E0029600
:10ACB000022F0E5F87709070081B892B09F0085FC8
:10ACC00086E596E120E620935616109257161092CC
:10ACD0005916109258162AE320935C162FEF2093F2
:10ACE0005D16FC0178962FEF32E030936F162093BB
:10ACF0006E161382128215821482178216821186B2
:10AD00001086138612861586148620E032E0378777
:10AD100026870896BF010E94785F2091FD06A22F2A
:10AD2000B0E0FD01E258F94E85E880831182FD0113
:10AD3000EE57F94E108211821282138210925A1627
:10AD400080915E1690915F16892B99F5809160161F
:10AD500090916116892B69F5809162169091631626
:10AD6000892B39F58091641690916516892B09F528
:10AD70008091661690916716892BD9F48091681698
:10AD800090916916892BA9F480916A1690916B169F
:10AD9000892B79F480916C1690916D16892B49F46A
:10ADA00088E080935B16D096B093DA15A093D915FE
:10ADB0004EC0E02EFF24822F90E0C0968E0D9F1D86
:10ADC0009093DA158093D915085F00935B160850AD
:10ADD000AA57B94EB093DE08A093DD0881E08C93AA
:10ADE00006950695069511960C9311972091E01CF7
:10ADF000129630E0F901E154FA4F408153E0220FFE
:10AE0000331F5A95E1F72F513A4ECD01B90150E069
:10AE10000E94AE80E091E01CF0E0E154FA4F8081A6
:10AE200090E09701281B390B225030403A83298348
:10AE30002091DD083091DE082E5F3F4F280F391F2B
:10AE4000C90160E070E049815A810E94C980809107
:10AE5000FD06082F10E00258194EF80113821282E5
:10AE60000E94A23E80959095F801938382830F9073
:10AE70000F90CF91DF911F910F91FF90EF90089568
:10AE8000FF920F931F93CF93DF938C01EA01E09120
:10AE9000E01CF0E0E154FA4F2081822F90E002960E
:10AEA000E2E0FE2EF20E87709070F81A892B11F0F6
:10AEB00088E0F80E1092FD0680E6809356161092F8
:10AEC000571610925916109258168AE380935C1602
:10AED0009FEF90935D16EEE6F6E161157105B9F40A
:10AEE00090936E1682E081831382128215821482FF
:10AEF0001782168211861086128681E083879487D6
:10AF00008D8585878E859F859787868707C0DF011A
:10AF1000FB0180E101900D928150E1F787E8809379
:10AF20007E1610927F16109282161092831610923F
:10AF3000841610928516A6E8B6E1FE0180E1019024
:10AF40000D928150E1F710925A16CE0160E840E070
:10AF50000E949761892B09F05FC00115110549F026
:10AF6000AEE5B6E1F80180E101900D928150E1F784
:10AF700006C08EE596E16EE676E10E94785F88E194
:10AF8000F80EF0925B1688EEF80E0F2D10E0005CC4
:10AF90001F4F1093DA150093D91500541040E0911B
:10AFA000FD06F0E0EA56F94EF093DE08E093DD0886
:10AFB00081E08083F694F694F694F1822091E01C6F
:10AFC000329630E0D901A154BA4F4C9163E0220F80
:10AFD000331F6A95E1F72F513A4ECF01B90150E086
:10AFE0000E94AE80E091E01CF0E0E154FA4F8081D5
:10AFF00090E0081B190B025010402091DD083091A1
:10B00000DE082E5F3F4F280F391FC90160E070E056
:10B01000A8010E94C98029C010925F1610925E1686
:10B0200010926116109260161092631610926216BA
:10B03000109265161092641610926716109266169A
:10B04000109269161092681610926B1610926A167A
:10B0500010926D1610926C1688E180935B1680E456
:10B0600090E09093DA158093D9158091FD06C82F52
:10B07000D0E0C258D94E1B821A820E94A23E80950F
:10B0800090959B838A83DF91CF911F910F91FF90C1
:10B090000895CF92DF92EF92FF920F931F93CF9379
:10B0A000DF939091FD06E92FF0E0DF01AE57B94E36
:10B0B000EC9080915D168F3F09F042C1E258F94E45
:10B0C0008181882309F03CC114968C9114978F3F9D
:10B0D00009F436C110E4C12ECE20E6FE05C08091F1
:10B0E0006E168F3F09F42CC184E18093DC08109226
:10B0F000DE081092DD08C091D915D091DA1540E034
:10B1000050E064E1292F30E0245D3F4F0FC0FC0187
:10B11000EA5AF94E9181992309F40CC18081823059
:10B1200009F4AF01990F990F990F690FC901860FA3
:10B13000911D8C179D0758F35093DE084093DD084E
:10B140006093DC08CD01049660E840E00E949761BE
:10B15000FC019093EC088093EB08009761F08089E4
:10B16000882309F0EDC08091FD0690E08A57994E42
:10B170000E940E62E5C08091FD0690E08A57994ECC
:10B180000E94C84FEC019093E6088093E508009771
:10B1900009F4D6C00091DD081091DE0801151105F3
:10B1A00011F4FF240FC0BC01605F7F4FE091E01CF1
:10B1B000F0E0E154FA4F4081C801029650E00E944D
:10B1C000A180F82EF0E8DF2EDE20898D882309F09B
:10B1D00041C00115110509F4B3C0BE01605F7F4F86
:10B1E000E091E01CF0E0E154FA4F408198012E5FBD
:10B1F0003F4FCB01B90150E00E94AE80C091E508FD
:10B20000D091E608CC2019F181E0898F8091E01C73
:10B2100090E029E730E0829FF001839FF00D929F3C
:10B22000F00D1124EB55F44E61857285838594856C
:10B2300028EE33E040E050E00E94DB820E942D8344
:10B24000CE014A96BA01A9010E9450676DC082E002
:10B25000898F6AC0E5FC08C0FF2031F0813009F019
:10B260006FC082E0898F6CC00115110589F0BE01A5
:10B27000605F7F4FE091E01CF0E0E154FA4F4081C5
:10B2800098012E5F3F4FCB01B90150E00E94AE8084
:10B29000CC2041F10091E5081091E60881E0F80129
:10B2A000818F8091E01C90E029E730E0829FF001DF
:10B2B000839FF00D929FF00D1124EB55F44E6185A4
:10B2C00072858385948528EE33E040E050E00E944B
:10B2D000DB820E942D83C8014A96BA01A9010E940F
:10B2E00050670EC08091DD089091DE08892B41F0F7
:10B2F000FF2031F0E091E508F091E60882E0818FCF
:10B30000E091E508F091E608808D882369F0DD2062
:10B3100059F4CF010E94E74A9093EA088093E90824
:10B32000009711F00E949D4BE091E508F091E6082E
:10B33000D08E06C05093DE084093DD086093DC0891
:10B340001092DA151092D915DF91CF911F910F91BC
:10B35000FF90EF90DF90CF900895DF92EF92FF92F1
:10B360000F931F93CF93DF9380915D168F3F09F06A
:10B370002DC28091FD06482F50E0FA01EE57F94E9C
:10B3800084818F3F09F422C2FA01E258F94E81818B
:10B39000882309F01BC21092DE081092DD0884E1B8
:10B3A0008093DC08C091D915D091DA1520E030E007
:10B3B00064E1FA01BC9611C0DC01AA5AB94E11969B
:10B3C0009C911197992309F4FBC18C91813009F468
:10B3D0009D01990F990F990F690FCF01860F911D4C
:10B3E0008C179D0748F32093DD083093DE086093A7
:10B3F000DC08232B09F46FC080915E1690915F16D4
:10B40000892B59F58091601690916116892B29F549
:10B410008091621690916316892BF9F480916416DD
:10B4200090916516892BC9F48091661690916716E4
:10B43000892B99F48091681690916916892B69F48B
:10B4400080916A1690916B16892B39F480916C1655
:10B4500090916D16892B09F4B9C18EE596E10E9491
:10B46000C84F8C019093E6088093E5086091DD0851
:10B470007091DE08009749F46E5F7F4F8EE596E18C
:10B4800040E022E00E94255026C092E0E92EF12CF7
:10B49000E60EF71EE8016096E091E01CF0E0E15452
:10B4A000FA4FD080C701BE014D2D50E00E94A1800F
:10B4B000009759F0CE01B7014D2D50E00E94AE80AB
:10B4C000E091E508F091E60804C0F801818D882339
:10B4D00011F482E0818F8091FD0690E08A57994EA9
:10B4E00060E840E00E9497619093EC088093EB083D
:10B4F000892B09F46BC180915E1690915F16892BA0
:10B5000009F073C08091601690916116892B09F043
:10B510006CC08091621690916316892B09F065C00A
:10B520008091641690916516892B09F05EC0809118
:10B53000661690916716892B09F057C0809168169E
:10B5400090916916892B09F050C080916A169091EC
:10B550006B16892B09F049C080916C1690916D167D
:10B56000892B09F042C08EE696E10E94FC61882397
:10B5700009F42CC1E091EB08F091EC088089882354
:10B5800061F18FEF92E090936F1680936E16109298
:10B590007116109270161092731610927216109205
:10B5A00075161092741610927716109276161092E5
:10B5B00079161092781610927B1610927A1680E007
:10B5C00091E090937D1680937C168EE596E16EE671
:10B5D00076E10E94785F30E253C08091FD0690E0F2
:10B5E0008A57994E0E940E62F1C08EE596E160E89E
:10B5F00040E00E949761892B09F0E8C08EE696E151
:10B600000E94FC618823B9F0EEE6F6E1DF01509775
:10B6100080E10D9001928150E1F78091FD06E82FC5
:10B62000F0E0AEE5B6E1EA57F94E80E101900D9207
:10B630008150E1F724C08EE696E160E840E00E9488
:10B6400097612091EB083091EC082817390709F031
:10B65000BDC0EEE6F6E1DF01509780E10D9001926A
:10B660008150E1F78091FD06E82FF0E0AEE5B6E10C
:10B67000EA57F94E80E101900D928150E1F730E6F2
:10B680001092FD068091E01CA82FB0E089E790E0C1
:10B69000A89FF001A99FF00DB89FF00D1124EB5564
:10B6A000F44E838981113068A154BA4F2C91822FB6
:10B6B00090E00296422F4E5F87709070481B892B56
:10B6C00009F0485F80E68093561610925716109244
:10B6D00059161092581610925A16485E40935B16EF
:10B6E00048518AE380935C168FEF80935D1688E85B
:10B6F00080937E1610927F1630938216A6E8B6E1EC
:10B700002091EB083091EC08C901FC0180E1019027
:10B710000D928150E1F7042F10E0005C1F4F109351
:10B72000DA150093D91500541040E091FD06F0E0C1
:10B73000EA56F94EF093DE08E093DD0882E080835C
:10B7400046954695469541832091E01C329630E01F
:10B75000D901A154BA4F4C9183E0220F331F8A952F
:10B76000E1F72F513A4ECF01B90150E00E94AE806F
:10B77000E091E01CF0E0E154FA4F808190E0081B7A
:10B78000190B025010402091DD083091DE082E5F29
:10B790003F4F280F391FC90160E070E0A8010E94E7
:10B7A000C9808091FD06C82FD0E0C258D94E1B82B7
:10B7B0001A820E94A23E809590959B838A830AC03C
:10B7C0003093DE082093DD086093DC081092DA15D0
:10B7D0001092D915DF91CF911F910F91FF90EF90AB
:10B7E000DF9008952F923F924F925F926F927F92D7
:10B7F0008F929F92AF92BF92CF92DF92EF92FF9281
:10B800000F931F93DF93CF9300D00F92CDB7DEB786
:10B81000AC01E091E01CF0E0E154FA4F2081822F6E
:10B8200090E0029602E0902E920E87709070981A27
:10B83000892B11F088E0980E6115710529F58FEFBD
:10B8400092E090936F1680936E161092711610927C
:10B85000701610927316109272161092751610923E
:10B86000741610927716109276161092791610921E
:10B87000781610927B1610927A1680E091E09093E1
:10B880007D1680937C1608C0AEE6B6E1FB0180E130
:10B8900001900D928150E1F74115510549F0AEE557
:10B8A000B6E1FA0180E101900D928150E1F706C006
:10B8B0008EE596E16EE676E10E94785F1092FD06D5
:10B8C00066E576E180E68093561610925716109240
:10B8D0005916109258168AE380935C168FEF809366
:10B8E0005D1686E880937E16DB0199961C921CE219
:10B8F000C12ED12CC60ED71EE091E01CAE2EBB246B
:10B9000089E790E0A89EF001A99EF00DB89EF00D89
:10B910001124EB55F44E848180938216918982899B
:10B92000D60112968C93129713969C93258136819B
:10B9300047815085E52EFF2400271127B22FAA2723
:10B9400099278827E82AF92A0A2B1B2BDA01C90133
:10B9500080709070B070892F9A2FAB2FBB27E82A88
:10B96000F92A0A2B1B2B40E050E0207040705070E9
:10B97000542F432F322F2227E22AF32A042B152B90
:10B98000D6011496ED92FD920D931C931797258581
:10B99000368547855089E52EFF2400271127B22FD1
:10B9A000AA2799278827E82AF92A0A2B1B2BDA01CC
:10B9B000C90180709070B070892F9A2FAB2FBB2770
:10B9C000E82AF92A0A2B1B2B40E050E02070407037
:10B9D0005070542F432F322F2227E22AF32A042BB0
:10B9E000152BF601E086F18602871387092D10E0FA
:10B9F000085C1F4F1093DA150093D91508531040B7
:10BA0000FB01F896F093DE08E093DD0881E0809377
:10BA10008E16892D8695869586958183665C7F4FE7
:10BA2000F501E154FA4F4081F50153E0EE0FFF1F9D
:10BA30005A95E1F7EF51FA4ECB01BF0150E00E9459
:10BA4000AE80E091E01CF0E0E154FA4F808190E09C
:10BA5000081B190B025010402091DD083091DE08C0
:10BA60002E5F3F4F280F391FC90160E070E0A80129
:10BA70000E94C980FCE09F0E9092DC080E94AC4BB3
:10BA80001C018091FD068B83682E77248090D91548
:10BA90009090DA154090DC085524ACE2B0E06A0ED4
:10BAA0007B1EC5C0B2E25B9E50011124A20CB31CE8
:10BAB000F50181A181FFBAC082FFB8C080818E3FAD
:10BAC00021F48181803809F4B1C06301C40CD11C18
:10BAD00086E596E1C80ED91EE3E0D601EC93F0ECC2
:10BAE0001396FC93139784E011968C93D50150968E
:10BAF0008C915097F601828391968C9180FF0DC0B6
:10BB00008FEF9FEFAFEFBFEF84839583A683B7835B
:10BB100080879187A287B38774C0D50155966D91B0
:10BB20007D918D919C91589728EE33E040E050E054
:10BB30000E942D83C901DA01EB2EFF240027112773
:10BB4000582F442733272227E22AF32A042B152BC8
:10BB50009C01AD01207030705070232F342F452F81
:10BB60005527E22AF32A042B152BA0E0B0E08070C1
:10BB7000A070B070BA2FA92F982F8827E82AF92A29
:10BB80000A2B1B2BF601E482F58206831783D5016D
:10BB90005D966D917D918D919C91909728EE33E00B
:10BBA00040E050E00E942D83C901DA01EB2EFF2412
:10BBB00000271127582F442733272227E22AF32A68
:10BBC000042B152B9C01AD01207030705070232F79
:10BBD000342F452F5527E22AF32A042B152BA0E0FA
:10BBE000B0E08070A070B070BA2FA92F982F88276E
:10BBF000E82AF92A0A2B1B2BF601E086F186028738
:10BC00001387D6011C961D921D921D921C921F97A0
:10BC1000F6017096D50180E10D9001928150E1F717
:10BC2000B0E24B0EE0E2F0E08E0E9F1E5394F1E086
:10BC3000F51508F037CF8092D9159092DA15409219
:10BC4000DC085092ED0888ED9FEF880E991E9A82CD
:10BC500089828A8180935A16898180935B169B81A1
:10BC6000092F10E00258194ED80113961C921E920B
:10BC700012970E94A23E80959095F801938382834B
:10BC80000F900F900F90CF91DF911F910F91FF9028
:10BC9000EF90DF90CF90BF90AF909F908F907F906C
:10BCA0006F905F904F903F902F900895BF92CF92EA
:10BCB000DF92EF92FF920F931F93DF93CF93CDB755
:10BCC000DEB760970FB6F894DEBF0FBECDBF809190
:10BCD000E01C90E029E730E0829FF001839FF00DA7
:10BCE000929FF00D1124EB55F44E8389882309F4BB
:10BCF000CCC080915D168F3F09F0C7C08091FD06D2
:10BD0000682F70E0FB01E258F94E8181882309F029
:10BD1000BCC01092DE081092DD0884E08093DC083D
:10BD20000091D9151091DA1520E030E044E0FB01D4
:10BD3000BC9611C0DC01AA5AB94E11969C9111977C
:10BD4000992309F49CC08C91813009F49D01990FCD
:10BD5000990F990F490FCF01840F911D80179107FB
:10BD600048F32093DD083093DE084093DC08232B52
:10BD700009F470C080915E1690915F16892B59F579
:10BD80008091601690916116892B29F58091621639
:10BD900090916316892BF9F4809164169091651641
:10BDA000892BC9F48091661690916716892B99F4B6
:10BDB0008091681690916916892B69F480916A16B2
:10BDC00090916B16892B39F480916C1690916D16B9
:10BDD000892B09F45AC08EE596E10E94C84F7C0178
:10BDE0009093E6088093E5086091DD087091DE0885
:10BDF000009749F46E5F7F4F8EE596E140E022E0C8
:10BE00000E94255027C082E0C82ED12CC60ED71E16
:10BE10008701005F1F4FE091E01CF0E0E154FA4F12
:10BE2000B080C601B8014B2D50E00E94A180009760
:10BE300059F0C801B6014B2D50E00E94AE80E09150
:10BE4000E508F091E60804C0F701818D882311F41C
:10BE500082E0818F1092DA151092D915DE011196C9
:10BE6000EEE5F6E180E101900D928150E1F780E08E
:10BE700090E0BE016F5F7F4F0E948F600AC03093D9
:10BE8000DE082093DD084093DC081092DA1510924A
:10BE9000D91560960FB6F894DEBF0FBECDBFCF9117
:10BEA000DF911F910F91FF90EF90DF90CF90BF90A7
:10BEB000089540E020E030E0FC01E20FF31F5081E4
:10BEC000FB01E20FF31FE0815E1731F4485F2F5F43
:10BED0003F4F403889F70AC0E527842F885FE7FD88
:10BEE00005C04F5F481711F0EE0FF9CF842F08956A
:10BEF0009F92AF92BF92CF92DF92EF92FF920F93F9
:10BF00001F93CF93DF93E82E992EEB0188818E3F0C
:10BF100021F48981803819F437C08F3FA9F1FF24BB
:10BF200000E011E09BE1A92EB12C89E7C82ED12CAD
:10BF300026C08091E01C90E0212F30E02A9DB001C6
:10BF40002B9D700D3A9D700D11249C012C9DC001FC
:10BF50002D9D900D3C9D900D1124680F791FFB01C4
:10BF6000EB55F44E80A5813049F46354744ECE01F4
:10BF70000E94595F8F1510F0F82E012F1F5F1330AC
:10BF8000C0F21093F80801C000E0402F50E020916B
:10BF9000E01C30E08BE190E0489FF001499FF00DFC
:10BFA000589FF00D112489E790E0AC01249FC00157
:10BFB000259F900D349F900D1124E80FF91F2E2D11
:10BFC000392DC901DC01E354F44E80E101900D925A
:10BFD0008150E1F7DF91CF911F910F91FF90EF908A
:10BFE000DF90CF90BF90AF909F900895E091E01CBC
:10BFF000F0E0DF01A750B74F1C92EE0FFF1FDF01EB
:10C00000A150B74F6D917C91E550F74F80819181A0
:10C010000E94F25B08950E945080AA2797FDA09588
:10C02000BA2FBC01CD0120E532E246E050E00E948B
:10C030002D839B01AC0120593A4F4C4F5F4FB90102
:10C04000CA0108954F925F926F927F928F929F9252
:10C05000BF92CF92DF92EF92FF920F931F93809146
:10C06000E01C90E045EAC42E4BE1D42E39E7432E84
:10C07000512C849DF001859DF00D949DF00D1124AF
:10C08000EC0DFD1D65817681878190850E94EA8196
:10C0900020E030E040E05FE30E9450820E94BE81D9
:10C0A0003B014C010E945080B82E0E945080FB2C16
:10C0B000EE24E80EF91E00E010E08091E01C90E014
:10C0C0009C01249DC001259D900D349D900D11244F
:10C0D000C80ED91EF60165817681878190850E9400
:10C0E000EA810E94BE819B01AC01C801B7010E9498
:10C0F0002D839B01AC01260D371D481D591DB9012B
:10C10000CA011F910F91FF90EF90DF90CF90BF90E9
:10C110009F908F907F906F905F904F9008951F93A6
:10C12000CF93DF939C011091E01CA12FB0E0FD01A3
:10C13000E750F74F8081882309F04AC02115310567
:10C1400091F0C3E0D9E0F90180E1019009928150BA
:10C15000E1F7FD01EE0FFF1FE550F74F83E099E097
:10C160009183808307C0FD01EE0FFF1FE550F74F5D
:10C17000118210826115710591F0C3E1D9E0FB01D4
:10C1800080E1019009928150E1F7FD01EE0FFF1F60
:10C19000E150F74F83E199E09183808307C0FD016F
:10C1A000EE0FFF1FE150F74F11821082A750B74FDB
:10C1B00081E08C930E94508064EF71E00E941A83AA
:10C1C000AC01662757FD6095762F812F0E949367FB
:10C1D000DF91CF911F910895EF92FF920F931F93DC
:10C1E0000E940B607B018C01E091E01CF0E0EA50C2
:10C1F000F74F8081833078F481E8E8168EE3F80603
:10C2000080E0080780E0180730F020E8E22E2EE3F7
:10C21000F22E012D112D80E090E060E070E00E9490
:10C22000F25B8091E01CE82FF0E0EA50F74F90813C
:10C230009F5F9083B801A7010E94D6671F910F915D
:10C24000FF90EF9008958091E01CA82FB0E089E75F
:10C2500090E0A89FF001A99FF00DB89FF00D112468
:10C26000EB55F44E84898823E1F0AA50B74F8C91A6
:10C270008823B9F40E940B60AC01CB01DA01AC0158
:10C28000BD0141388EE3580780E0680780E07807F9
:10C2900020F040E85EE360E070E08091E01C0E94E6
:10C2A000D66708951F931091E01CE12FF0E0EC5049
:10C2B000F74F8081882371F40E94508060ED77E011
:10C2C0000E941A83AC01662757FD6095762F812F57
:10C2D0000E9422681F9108950E94354B892BD1F44A
:10C2E000E091E01CF0E0EC50F74F8081843090F456
:10C2F0000E9446568091E01CE82FF0E0EC50F74F8A
:10C3000090819F5F908348E853E160E070E00E9475
:10C31000226808958091E01C0E947067E091E01C03
:10C32000F0E0EC50F74F10820E9468770895BF92BA
:10C33000CF92DF92EF92FF920F931F93CF93DF93F1
:10C340007C01062FB42E1092F8082091E01C30E0FA
:10C350000695069506954BE1C42ED12C89E790E011
:10C36000289FE001299FD00D389FD00D112433C0A4
:10C37000212F30E02C9DF0012D9DF00D3C9DF00D06
:10C380001124EC0FFD1FEB55F44E80A58F3F01F1FA
:10C3900082A98B1511F0BB20D9F42C9DC0012D9DD5
:10C3A000900D3C9D900D11248C0F9D1F8354944E35
:10C3B000B701402F50E00E94A180009749F48BE123
:10C3C000189F900111242C0F3D1F2354344E09C097
:10C3D0001F5F1093F8081091F808133048F220E01E
:10C3E00030E0C901DF91CF911F910F91FF90EF9045
:10C3F000DF90CF90BF9008956091E01C29E7629F85
:10C40000B0011124625F734E40E150E00E94A180B0
:10C410009C0180E0232B09F481E008951F93CF93C2
:10C42000DF93BC011091E01CE12FF0E0EE0FFF1F45
:10C43000E251F74F8081918140E150E00E94A1805C
:10C440000097A9F4812F0E947A67A091E01CB0E0C8
:10C45000FD01EE0FFF1FE251F74F808191812FEF19
:10C46000EC01288B11821082AE50B74F1C928FEFD7
:10C470009FEF0E94EA741F93DC0150968C915097B5
:10C480008823E1F41091E01CE12FF0E0EE0FFF1F94
:10C49000E251F74F80819181892B81F4B183A08390
:10C4A0000E94508060ED77E00E941A83AC016627FD
:10C4B00057FD6095762F812F0E94AE681F910895D9
:10C4C0001F93CF93DF932091E01CA22FB0E0FD01DA
:10C4D000EE0FFF1FE251F74F408151814115510589
:10C4E00009F489C0C9E7D0E0AC9FF001AD9FF00D21
:10C4F000BC9FF00D1124EB55F44EAE50B74F9C91FC
:10C500008789981788F580E090E060E070E00E94ED
:10C5100040571091E01C212F30E0F901EE50F74F09
:10C5200080818F5F80832C9FF0012D9FF00D3C9FB9
:10C53000F00D1124EB55F44E65857685878590893D
:10C5400028EE33E040E050E00E942D83CA01B9019B
:10C5500028EE33E040E050E00E94DB82AB01BC01FA
:10C56000812F0E94AE6847C0822F0E947A67209177
:10C57000E01C30E0F901EE0FFF1FE251F74FA08100
:10C58000B18181E050968C9311821082F901EE50B6
:10C59000F74F10821092F80840E0ABE1B0E02C9F1A
:10C5A000B0012D9F700D3C9F700D112420C0242FD1
:10C5B0002F5F842F90E08A9FF0018B9FF00D9A9F50
:10C5C000F00D1124E60FF71FEB55F44E80A58823DC
:10C5D00069F44093F8088BE1489FC0011124860F4D
:10C5E000971F8354944E0E943B6205C0422F4330F4
:10C5F000F0F24093F808DF91CF911F910895CF9307
:10C60000DF93DC01EB01E091E01CF0E0E154FA4F34
:10C61000E081E83061F49C01285F3F4FFB0188E036
:10C620000190E90109929E018150D1F723C0E630C3
:10C6300039F59C01285F3F4FAB0183E0FA0101907F
:10C64000AF01F90101929F018150C1F78FEF1B9655
:10C650008C931B978EEF1C968C931C979D01235FE8
:10C660003F4FFE01339683E00190E90109929E015C
:10C670008150D1F718968C91189792E0892720C0A5
:10C68000E23019F589811F968C931F9788811E9639
:10C690008C931E971D961C921D978EEF1C968C9363
:10C6A0001C978FEF1B968C931B971A961C921A97C8
:10C6B0008091BE1C19968C9319978091BD1C8D7F1B
:10C6C00018968C93DF91CF9108958FEF9FEF0E9482
:10C6D000EA749F92AF92BF92CF92DF92EF92FF9255
:10C6E0000F931F93CF93DF93A82E992E69017A01A0
:10C6F000B02E21E0021719F4603409F0BDC0109289
:10C70000F8085091E01CC52FD0E040E00BE110E0AC
:10C7100089E790E0C89FD001C99FB00DD89FB00DA8
:10C720001124A5C0642F70E0942F9F5F609F90013B
:10C73000619F300D709F300D11242A0F3B1FF901AE
:10C74000EB55F44E80A58F3F09F090C04093F80858
:10C75000F901E354F44E8A2D992D9C01D90180E111
:10C760000D9001928150E1F731E0B31619F58BE19C
:10C7700090E09C01629FC001639F900D729F900D9D
:10C78000112429E730E0B901C69F9001C79F300D01
:10C79000D69F300D1124820F931F652F70E043E068
:10C7A000660F771F4A95E1F76F517A4E8354944E86
:10C7B0000E94FF628091E01C90E02091F80830E038
:10C7C0000BE110E0209FA001219F500D309F500DE4
:10C7D0001124C9E7D0E09C012C9FC0012D9F900D32
:10C7E0003C9F900D1124480F591FFA01EB55F44E50
:10C7F00010A6B2AAC114D104E104F10411F1CA01D6
:10C800008253944EB701A6010E9450672091F80808
:10C8100030E08091E01C90E0209FF001219FF00D1E
:10C82000309FF00D1124BC016C9FC0016D9F900DD5
:10C830007C9F900D1124E80FF91FEB55F44E11AABF
:10C8400002C081E081AB8091F8082BE1829FC0019A
:10C8500011242091E01C49E7249F90011124820FAC
:10C86000931F8354944E0E943B6206C0492F43306D
:10C8700008F458CF4093F808DF91CF911F910F91A2
:10C88000FF90EF90DF90CF90BF90AF909F90089572
:10C89000FF920F931F93CF93DF9381E08093F8086B
:10C8A0000BE110E0C9E7D0E0FF24FA9444C0809186
:10C8B000E01C90E030E0209FA001219F500D309FB0
:10C8C000500D11249C012C9FC0012D9F900D3C9F69
:10C8D000900D1124480F591FFA01EB55F44E80A515
:10C8E0008F3F21F181A9813009F1CA018253944E11
:10C8F0000E943667892BD1F02091F80830E08091B2
:10C90000E01C90E0209FF001219FF00D309FF00D82
:10C9100011249C012C9FC0012D9F900D3C9F900DD8
:10C920001124E80FF91FEB55F44EF0A68091F8089A
:10C930008F5F8093F8082091F808233008F4B7CF70
:10C94000DF91CF911F910F91FF9008958F929F9249
:10C95000AF92BF92CF92DF92EF92FF920F931F930D
:10C96000DF93CF93CDB7DEB7E2970FB6F894DEBF73
:10C970000FBECDBF1092F808FBE1CF2ED12CE9E716
:10C98000EE2EF12C8E010F5F1F4F7AE5A72E75E07A
:10C99000B72E6BE1862E59E7952E81C030E080914D
:10C9A000E01C90E02C9DF0012D9DF00D3C9DF00DC4
:10C9B00011249C012E9DC0012F9D900D3E9D900D38
:10C9C0001124E80FF91FEB55F44E80A58F3F09F4B1
:10C9D00061C086E197E00E94840B2091F80830E066
:10C9E0008DB79EB708970FB6F8949EBF0FBE8DBF48
:10C9F000ADB7BEB71196EDB7FEB71283018313969C
:10CA0000BC92AE92129715963C932E9314978091F8
:10CA1000E01C90E02C9DF0012D9DF00D3C9DF00D53
:10CA200011249C012E9DC0012F9D900D3E9D900DC7
:10CA30001124E80FF91FEB55F44E80A5992787FDC7
:10CA4000909517969C938E9316970E943C818DB774
:10CA50009EB708960FB6F8949EBF0FBE8DBFC80153
:10CA60000E94920B6091F808689DB001112480919A
:10CA7000E01C899DC0011124680F791F6354744E16
:10CA8000C8010E94ED79C8010E94920B83E197E0F2
:10CA90000E94840B8091F8088F5F8093F8082091A2
:10CAA000F808233008F47ACFE2960FB6F894DEBF88
:10CAB0000FBECDBFCF91DF911F910F91FF90EF90EF
:10CAC000DF90CF90BF90AF909F908F9008957F920E
:10CAD0008F929F92AF92BF92CF92DF92EF92FF928E
:10CAE0000F931F934B015C01142F722E8091E01C59
:10CAF00090E029E7C22ED12C8C9D70018D9DF00C09
:10CB00009C9DF00C112425EA3BE1E20EF31E80E02F
:10CB100095E0A0E0B0E0F70180839183A283B38326
:10CB200080E4848380E395E7A0E0B0E0858396838A
:10CB3000A783B0870E942260F7016187728783878D
:10CB40009487F090E01C6F2D70E06C9D90016D9DBE
:10CB5000300D7C9D300D1124F901EB55F44E88EE1B
:10CB600093E0A0E0B0E085879687A787B08B81E04F
:10CB7000878B928A818A138A148B758A068B40E090
:10CB8000ABE1B0E05FEF0FC0842F90E08A9FF0012F
:10CB90008B9FF00D9A9FF00D1124E20FF31FEB55C0
:10CBA000F44E50A74F5F433078F34093F80809E7FD
:10CBB00010E0609F9001619F300D709F300D112437
:10CBC000D901AB55B44EA759BF4F9FEF9D9382E05B
:10CBD0008D931D921D921D921D921D921D921D926C
:10CBE0001D921D92EE24E394ED929D93FB01E1547E
:10CBF000FA4F8081FB0193E0EE0FFF1F9A95E1F75A
:10CC0000EF51FA4EE80FF11D339781918D93819189
:10CC10008D9380818C93A857B040772009F45AC037
:10CC20008EEF90E859969C938E9358975B961C9242
:10CC30001E925A975D961C921E925C975F961C926C
:10CC40001E925E9791961C921E92909793961C92BC
:10CC50001E92929795961C921E92949797961C926C
:10CC60001E9296976F2D70E0A3E0660F771FAA952E
:10CC7000E1F76F517A4EC9018354944E0E94FF62CE
:10CC80008091E01C90E09C01209FC001219F900DAD
:10CC9000309F900D1124FC01EB55F44E10A623E0BB
:10CCA00022ABE1AA8354944E0E943B620E945261DF
:10CCB00081149104A104B10469F08091E01C90E01A
:10CCC000809FF001819FF00D909FF00D1124EB5596
:10CCD000F44EE38A8091E01C48EE53E060E070E09F
:10CCE0000E945D681F910F91FF90EF90DF90CF90B1
:10CCF000BF90AF909F908F907F900895FFCF089541
:10CD000008950F931F93DF93CF93CDB7DEB7289786
:10CD10000FB6F894DEBF0FBECDBF8C018091E01C32
:10CD2000882309F055C00115110591F483E3898327
:10CD30008A8380917A168B8380917B168C83809175
:10CD40007C168D8380917D168E838E010F5F1F4F21
:10CD50006091D9157091DA15FB01EB5AF94E03C0B9
:10CD600080818687319726E1E535F207C9F7D8013A
:10CD70008C91818311968C911197828312968C915C
:10CD80001297838313968C911397848314968C91B6
:10CD90001497858315968C918683A1EEB5E137961D
:10CDA0008D91819325E1A73EB207D1F786E8809364
:10CDB00062168DED80936316625F7F4F7093DA1574
:10CDC0006093D91586E596E141E00E94903527C031
:10CDD000813049F580915C168131F1F48EE696E15F
:10CDE000B8010E9449738823B9F090918016809110
:10CDF0008116825B904F81F480918616873761F4AB
:10CE000050917E1640917F1680917D1690917C16F0
:10CE10006EE576E10E94F622C8010E94937310929B
:10CE2000DA151092D91580E090E028960FB6F894A4
:10CE3000DEBF0FBECDBFCF91DF911F910F9108953F
:10CE4000EF92FF920F931F93FC01E080F18002812B
:10CE500013810E94B80EE61AF70A080B190BB701E6
:10CE6000C8011F910F91FF90EF900895EF92FF92EC
:10CE70000F931F93FC01E080F180028113810E94D7
:10CE8000B80E20E030E0E616F7060807190710F4A0
:10CE900021E030E0C9011F910F91FF90EF900895BC
:10CEA000CF92DF92EF92FF920F931F936C017A0162
:10CEB0008B01FC0144835583668377830E94B80EFF
:10CEC0006E0D7F1D801F911FF60160837183828329
:10CED00093831F910F91FF90EF90DF90CF90089573
:10CEE000E82FF0E0E754F34E8081882311F00E9490
:10CEF000080F0895E82FF0E0E954F34E808188236D
:10CF000011F00E94080F0895CF93DF93C9EADCE186
:10CF100088810E94080F19928CE1C53BD807C1F7A0
:10CF2000DF91CF910895CF92DF92EF92FF920F930E
:10CF30001F93C82ECB01BA0128EE33E040E050E049
:10CF40000E942D83C901DA017C018D0181E0E81680
:10CF500080E0F80681E0080780E0180728F0E12C5F
:10CF6000F12C81E0082F112D81E0C81621F4C701B2
:10CF700062E979E603C0C7016BE879E60E94B70F62
:10CF8000D82E882339F4E114F1040105110511F0BC
:10CF90000E947E66EC2DF0E0E755F34ED2861F919D
:10CFA0000F91FF90EF90DF90CF900895CF92DF9296
:10CFB000EF92FF920F931F93C82E7A018B0141309D
:10CFC00080E0580781E0680780E0780768F481E036
:10CFD000C81621F4CA0161EA79E603C0CA016AE908
:10CFE00079E60E94001018C0CB01BA0128EE33E0A8
:10CFF00040E050E00E942D83C901DA017C018D01DF
:10D0000081E0C81621F4C70161EA79E603C0C701CF
:10D010006AE979E60E94B70FD82E882339F4E11423
:10D02000F1040105110511F00E947E66EC2DF0E07F
:10D03000E755F34ED0861F910F91FF90EF90DF9050
:10D04000CF900895CF92DF92EF92FF920F931F93AC
:10D05000C82ECA01DB017C018D0181E0E81680E069
:10D06000F80681E0080780E0180728F0E12CF12C91
:10D0700091E0092F112D81E0C81621F4C70160EB62
:10D0800079E603C0C70169EA79E60E940010D82E4C
:10D09000882339F4E114F1040105110511F00E940F
:10D0A0007E66EC2DF0E0E754F34ED0821F910F9195
:10D0B000FF90EF90DF90CF900895CF92DF92EF92A4
:10D0C000FF920F931F93C82E7A018B01413080E0AD
:10D0D000580781E0680780E0780788F4411551051A
:10D0E0006105710589F4EC2DF0E0EE0FFF1FED5D99
:10D0F000F64F808191817C0100E010E00DC0E12CB1
:10D10000F12C31E0032F112DEC2DF0E0EE0FFF1F7D
:10D11000ED5DF64FF182E08281E0C81621F4C7018F
:10D1200066EC79E603C0C70168EB79E60E9400105F
:10D13000D82E882339F4E114F1040105110511F00A
:10D140000E947E66EC2DF0E0E755F34ED6821F91EB
:10D150000F91FF90EF90DF90CF900895CF92DF92E4
:10D16000EF92FF920F931F93C82ECA01DB017C013F
:10D170008D0181E0E81680E0F80681E0080780E094
:10D18000180728F0E12CF12C51E0052F112D81E03A
:10D19000C81621F4C7016BED79E603C0C70164ED41
:10D1A00079E60E940010D82E882339F4E114F104A6
:10D1B0000105110511F00E947E66EC2DF0E0E954A6
:10D1C000F34ED0821F910F91FF90EF90DF90CF90A0
:10D1D0000895CF92DF92EF92FF920F931F93C82E84
:10D1E0007A018B01413080E0580781E0680780E0D8
:10D1F000780788F4411551056105710589F4EC2D16
:10D20000F0E0EE0FFF1FE95DF64F808191817C0118
:10D2100000E010E00DC0E12CF12C71E0072F112D82
:10D22000EC2DF0E0EE0FFF1FE95DF64FF182E0829A
:10D2300081E0C81621F4C70161EF79E603C0C70198
:10D2400063EE79E60E940010D82E882339F4E114A9
:10D25000F1040105110511F00E947E66EC2DF0E04D
:10D26000E755F34ED2821F910F91FF90EF90DF9020
:10D27000CF900895CF92DF92EF92FF920F931F937A
:10D28000C82E7A018B01413080E0580781E06807A1
:10D2900080E0780788F4411551056105710589F42E
:10D2A000EC2DF0E0EE0FFF1FE55DF64F80819181E0
:10D2B0007C0100E010E00DC0E12CF12C11E0012F09
:10D2C000112DEC2DF0E0EE0FFF1FE55DF64FF18222
:10D2D000E08281E0C81621F4C7016DE07AE603C060
:10D2E000C7016FEF79E60E940010D82E882339F429
:10D2F000E114F1040105110511F00E947E66EC2D88
:10D30000F0E0E755F34ED0821F910F91FF90EF9020
:10D31000DF90CF9008951092E01C0E94F65F0E946B
:10D32000EB74089581E08093E01C0E94F65F0E94F8
:10D33000EB7408951092E01C0E94EC600E94EB7464
:10D34000089581E08093E01C0E94EC600E94EB74E1
:10D3500008951092E01C0E946C610E94EB74089585
:10D3600081E08093E01C0E946C610E94EB74089540
:10D370001092E01C80E040E050E060E070E00E942D
:10D380005D680E9448640E94EB74089581E0809378
:10D39000E01C40E050E060E070E00E945D680E94A8
:10D3A00048640E94EB7408951092E01C0E94606231
:10D3B0000E94EB74089581E08093E01C0E946062FB
:10D3C0000E94EB7408951092E01C80E040E050E071
:10D3D00060E070E00E94E9680E94B64B0E94EB7426
:10D3E000089581E08093E01C40E050E060E070E050
:10D3F0000E94E9680E94B64B0E94EB740895109257
:10D40000E01C80E040E050E060E070E00E943A699B
:10D410000E940D780E94EB74089581E08093E01CD7
:10D4200040E050E060E070E00E943A690E940D78B0
:10D430000E94EB7408950F93DF93CF9300D000D038
:10D44000CDB7DEB79A8389837C836B8381E0809339
:10D45000E01C8C818093E9158B818093EA158A8189
:10D460008093BD1C89818093BE1C80910D0588230B
:10D4700041F460E070E080E090E040E020E001E016
:10D480000BC08AE695E00E94CA7468EE73E080E003
:10D4900090E041E021E000E00E94274981E044EF74
:10D4A00051E060E070E00E943A690F900F900F9099
:10D4B0000F90CF91DF910F9108950F93DF93CF934A
:10D4C000CDB7DEB760970FB6F894DEBF0FBECDBF05
:10D4D000AC011092E01C009779F020E030E0F901F7
:10D4E000EF51FA4EDA01A20FB31F8C9180832F5FA8
:10D4F0003F4F2630310599F780910D05882341F47F
:10D5000060E070E080E090E040E021E001E01DC0DC
:10D51000FE01319680E1DF011D928A95E9F780E2F4
:10D52000898381E08A8384E08B8380E78C8381EF29
:10D530008D838CE38E83CF010E94CA7468E077E00C
:10D5400080E090E041E021E000E00E94274980E097
:10D5500044EF51E060E070E00E943A6960960FB6D7
:10D56000F894DEBF0FBECDBFCF91DF910F9108952C
:10D570008FE299E090939C1C80939B1C0E9484678F
:10D580000E94316B0895382F1092DB0E20E02CC0E2
:10D59000822F90E0FC0173E0EE0FFF1F7A95E1F718
:10D5A000880F991FE80FF91FED53F14F80818130EB
:10D5B000D1F4822F90E0FC0153E0EE0FFF1F5A954B
:10D5C000E1F7880F991FE80FF91FED53F14F8181A3
:10D5D000831749F42093DB0E8AE0289F90011124E1
:10D5E0002D53314F07C02F5F223090F22093DB0E76
:10D5F00020E030E0C9010895AC0181E08093DB0EAA
:10D6000021E02AC0322F3F5F822F90E0FC01B3E07F
:10D61000EE0FFF1FBA95E1F7880F991FE80FF91F6A
:10D62000ED53F14F80818823B1F481E08093CD0EDA
:10D630002093CE0E90E00AC0E92FF0E0DA01AE0FA1
:10D64000BF1F8C91ED53F14F84879F5F9830A0F3FB
:10D650009093DB0E0895232F2230A0F22093DB0E4F
:10D66000089581E08093C30E1092C40E8EEF8093D4
:10D67000C50E80E88093C60E21E010C0822F90E096
:10D68000FC0143E0EE0FFF1F4A95E1F7880F991F59
:10D69000E80FF91FED53F14F10822F5F223070F326
:10D6A0002093DB0E0895EF92FF920F931F93CF9379
:10D6B000DF937C01E091AE09F091AF098091B00950
:10D6C00090E00396DF01A80FB91F0397B093DA0E1D
:10D6D000A093D90EE80FF91F818186FD29C087FD2F
:10D6E00012C0FD0181919191A191B1918093B309F3
:10D6F0009093B409A093B509B093B609F093DA0EEC
:10D70000E093D90E31C080E68093B3098C918F707D
:10D710008093B40911968D919C9112979093B609BC
:10D720008093B5091396B093DA0EA093D90E1CC05E
:10D7300087FD11C08C9182958F7080668093B309AC
:10D74000FD0181918295807F8093B409F093DA0E78
:10D75000E093D90E05C080E68093B3091092B40916
:10D760001092B6091092B5098091B009C091AE0926
:10D77000D091AF09C80FD11D898185FD0BC0E09103
:10D78000D90EF091DA0E81918093B909F093DA0EF7
:10D79000E093D90E898190E088719070883091056E
:10D7A00061F0893091051CF4892B79F019C0803122
:10D7B000910529F04897A1F406C081E001C080E4FA
:10D7C0008093BA090DC08FEFFBCFE091D90EF09195
:10D7D000DA0E81918093BA09F093DA0EE093D90EB4
:10D7E0008A8190E08073907054E0959587955A9562
:10D7F000E1F70E94C36AAC019093D80E8093D70ED4
:10D800008A81282F30E0207C30702034310509F4E3
:10D8100077C02134310524F4232B09F493C0A8C028
:10D8200020383105D1F0203C310509F0A1C0411567
:10D83000510519F482E099E01CC0ABEBB9E0FA01A4
:10D84000329688E001900D928150E1F78BEB99E0E0
:10D8500067E97CE10E94FF628BC0A091D90EB09174
:10D86000DA0E8C9187FD27C04115510529F48DEC06
:10D8700098E00E94840BDEC1ABEBB9E0FA0132966E
:10D8800088E001900D928150E1F786E0E3ECF9E049
:10D89000DF011D928A95E9F7E091D90EF091DA0E39
:10D8A000819191919093CA098093C909F093DA0EFE
:10D8B000E093D90E5DC080FD20C011968C91119728
:10D8C00081508230D0F48FEF8093BB098C91869584
:10D8D0008F708093BC098DE0EDEBF9E0EF011992B8
:10D8E0008A95E9F711968C9111978093CA0912963F
:10D8F000B093DA0EA093D90E3BC089E898E0B9CF77
:10D900004115510519F484E598E0B3CFABEBB9E0CC
:10D91000FA01329688E001900D928150E1F7A3EC74
:10D92000B9E08091D90E9091DA0E9C01F90188E05E
:10D9300001900D928150E1F78091D90E9091DA0E0D
:10D94000089612C0ABEBB9E08091D90E9091DA0E37
:10D950009C01F90180E101900D928150E1F78091E5
:10D96000D90E9091DA0E40969093DA0E8093D90EEC
:10D970008091B0090091AE091091AF09080F111DF7
:10D98000F801828183700E94C36AAC019093D80E23
:10D990008093D70ED80112968C91282F30E02C70EE
:10D9A00030702430310509F475C02530310524F478
:10D9B000232B09F491C0A6C028303105D1F02C30BA
:10D9C000310509F09FC04115510519F48FE198E028
:10D9D00050CFABECB9E0FA01329688E001900D929D
:10D9E0008150E1F78BEC99E069E97CE10E94FF62EC
:10D9F00089C0A091D90EB091DA0E8C9187FD25C017
:10DA00004115510519F48AEE97E033CFABECB9E03C
:10DA1000FA01329688E001900D928150E1F786E09C
:10DA2000E3EDF9E0EF0119928A95E9F7E091D90E5B
:10DA3000F091DA0E819191919093DA098093D9094E
:10DA4000F093DA0EE093D90E5DC080FD20C01196F0
:10DA50008C91119781508230D0F48FEF8093CB0955
:10DA60008C9186958F708093CC098DE0EDECF9E078
:10DA7000EF0119928A95E9F711968C91119780938D
:10DA8000DA091296B093DA0EA093D90E3BC086EA5B
:10DA900097E0EFCE4115510519F481E797E0E9CE03
:10DAA000ABECB9E0FA01329688E001900D9281501A
:10DAB000E1F7A3EDB9E08091D90E9091DA0E9C01C7
:10DAC000F90188E001900D928150E1F78091D90E23
:10DAD0009091DA0E089612C0ABECB9E08091D90EA5
:10DAE0009091DA0E9C01F90180E101900D92815034
:10DAF000E1F78091D90E9091DA0E40969093DA0E6C
:10DB00008093D90E8091B209885D8093B20980918B
:10DB1000B009E091AE09F091AF09E80FF11D8181E4
:10DB200085FF5AC0A091D90EB091DA0E8C918C7FEE
:10DB3000883F09F051C081E18093B9098C91883FF9
:10DB400029F18B3F09F045C0E3EBF9E0B896119657
:10DB50008C91119782958F7090E080559F409093A3
:10DB6000DB09818311968C91119790E08F709070F2
:10DB700080559F409283838312968D919C91139739
:10DB80009093E2098093E109149619C011968D9142
:10DB90009C9112979093DC098093DB0913968D91E9
:10DBA0009C9114979093DE098093DD0915968D91D1
:10DBB0009C9116979093E2098093E1091796B09390
:10DBC000DA0EA093D90E8091B209885F8093B209D2
:10DBD00003C082E397E04DCE2091D90E8091AE092B
:10DBE000281B2093B009E114F10451F41092B709F5
:10DBF0008091B209885290919D1C890F821B0CC0A4
:10DC0000E8EDFFEFEE0EFF1EF092B70988E290E01C
:10DC1000E80EF91E8E2D88528093B8098091B909BB
:10DC2000813141F48091B7099091B8099093E0094E
:10DC30008093DF09DF91CF911F910F91FF90EF90BB
:10DC40000895FF920F931F93DF93CF93CDB7DEB765
:10DC500064970FB6F894DEBF0FBECDBF8C01462F80
:10DC600081E08093E01C1092B2091092B00980917B
:10DC70009B1C90919C1C8093AE099093AF0960937C
:10DC80009D1C10929E1C9801225F3F4FB90150E0ED
:10DC90000E94AE80D8011B962D913C911C973A832F
:10DCA0002983FE01319681818093971C898180931D
:10DCB000981C19968D919C911A979A8389838181DA
:10DCC0008093991C898180939A1CE091AE09F09110
:10DCD000AF098081813021F4C9010E9434232DC114
:10DCE0008BEB9EE00E943667892B41F01092B40EB8
:10DCF0001092B30E1092B60E1092B50EE091AE09CE
:10DD0000F091AF0930812181C9018070987F892FFE
:10DD10009927803C910549F0803E910589F000E00B
:10DD200010E0FF2440E050E015C0890117705281D7
:10DD300043818091B0098C5F8093B009FF240AC0B1
:10DD4000F48052814381890117708091B0098B5F03
:10DD50008093B0098091B50E9091B60E892B19F180
:10DD60000115110509F4E9C08091B30E9091B40E2C
:10DD70000817190709F0E1C08091B90E9091BA0E09
:10DD80008417950709F0D9C09091BB1C8091971C0E
:10DD9000981709F0D2C09091BC1C8091981C9817DC
:10DDA00009F0CBC01BC001151105C1F01093B40ED2
:10DDB0000093B30E5093BA0E4093B90E8BEB9EE0D6
:10DDC00044EF51E060E070E00E9450678091971C42
:10DDD0008093BB1C8091981C8093BC1C8091B009DF
:10DDE000853049F12091AE093091AF09F901E80F72
:10DDF000F11DE081E33021F0E13409F09EC004C060
:10DE0000C8010E94536B17C08F5F8093B009A3EBCA
:10DE1000B9E0F901E80FF11D88E201900D928150FF
:10DE2000E1F78091B009885D8093B0098091B209D3
:10DE3000885D8093B2099091B00940919D1C491B67
:10DE40004093B1092F2D30E063E0220F331F6A9514
:10DE5000E1F78091B209280F311D2D54364FE09122
:10DE6000AE09F091AF09E90FF11DC901BF0150E002
:10DE70000E94AE80012BC9F08091B50E9091B60E34
:10DE8000892B31F48091B2098093B50E1092B60EB1
:10DE90002091B1098091B50E9091B60E820F911D1F
:10DEA0009093B60E8093B50E0BC02091B20980916D
:10DEB000B10990E0820F911D9093B40E8093B30E40
:10DEC0002091B50E3091B60E2115310539F08091B3
:10DED000B30E9091B40E2817390779F506E516E1CF
:10DEE00023EB39E04091B30E5091B40EC801B90153
:10DEF0000E94AE806091B30E7091B40E1092B40E79
:10DF00001092B30E1092B60E1092B50E1092DA1552
:10DF10001092D9151B829091971C8091981C8C832C
:10DF20009D831C861E861D86C801AE014D5F5F4F16
:10DF30009E01245F3F4F0E94C67A64960FB6F89404
:10DF4000DEBF0FBECDBFCF91DF911F910F91FF902C
:10DF500008951F93CF93DF93EC011092DB0E30C036
:10DF6000812F90E0FC01B3E0EE0FFF1FBA95E1F7BF
:10DF7000880F991FE80FF91FED53F14F8081813011
:10DF8000E1F4212F30E0C901F3E0880F991FFA95E1
:10DF9000E1F7220F331F820F931F8B53914FBE0166
:10DFA00048E050E00E94A180009739F48AE0189F71
:10DFB000900111242D53314F09C01F5F1093DB0EC8
:10DFC0001091DB0E123060F220E030E0C901DF91E9
:10DFD000CF911F9108950F931F93182F092FE09150
:10DFE000AE09F091AF093396F093DA0EE093D90EB3
:10DFF00033978091B009E80FF11D12821182809150
:10E00000B009E091AE09F091AF09E80FF11D83E08E
:10E01000808380915716282F30E0C9018F7090704F
:10E02000892B09F03FC08091581690915916892B81
:10E03000C9F58091B009E091AE09F091AF09E80F00
:10E04000F11D81818064818380915616282F30E0F4
:10E05000C9018F709070892B81F480915716807F51
:10E0600061F48091B009E091AE09F091AF09E80F39
:10E07000F11D8181806881835FC0E091D90EF091AC
:10E08000DA0E94E0220F331F9A95E1F7809157162C
:10E0900082958F70822B80838091D90E9091DA0EB9
:10E0A000019646C08091561690E08F709070892B33
:10E0B00051F5822F807F39F58091B009E091AE094A
:10E0C000F091AF09E80FF11D818180688183E091B3
:10E0D000D90EF091DA0E909157169F7080915616D6
:10E0E000807F982B9083E091D90EF091DA0E809189
:10E0F000581690915916928381838091D90E9091F0
:10E10000DA0E039615C0E091D90EF091DA0E8091E7
:10E11000561690915716A0915816B09159168083B3
:10E120009183A283B3838091D90E9091DA0E0496E5
:10E130009093DA0E8093D90E80915C16813161F450
:10E140008091B009E091AE09F091AF09E80FF11D9F
:10E150008181806281830EC0E091D90EF091DA0E48
:10E1600080838091D90E9091DA0E01969093DA0E09
:10E170008093D90E80915D16803479F08F3FC9F07D
:10E18000813011F58091B009E091AE09F091AF09AD
:10E19000E80FF11D818188600AC08091B009E0918B
:10E1A000AE09F091AF09E80FF11D81818061818393
:10E1B00019C08091B009E091AE09F091AF09E80F64
:10E1C000F11D81818861F3CFE091D90EF091DA0ED3
:10E1D00080838091D90E9091DA0E01969093DA0E99
:10E1E0008093D90E8EE596E10E94A96FDC01909391
:10E1F000D80E8093D70E009709F49FC08091B00984
:10E20000E091AE09F091AF09E80FF11D11968C91E4
:10E210008295807F9281892B82832091661630E0DF
:10E220008091BD1C90E08D7F28173907B9F590913A
:10E2300067168091BE1C981789F58091681688230F
:10E2400069F5809169168F3F49F580916A168E3F76
:10E2500029F580916B16882309F58091E01CE82F41
:10E26000F0E083E0EE0FFF1F8A95E1F7EF51FA4EE1
:10E2700090916C168081981789F490916D16818128
:10E28000981761F48091B009E091AE09F091AF095F
:10E29000E80FF11D8281806C828365C080916616D3
:10E2A00090916716892B59F580916816909169169F
:10E2B000892B29F580916A1690916B16892BF9F4B8
:10E2C00080916C1687FD1BC08091B009E091AE096A
:10E2D000F091AF09E80FF11D828180688283E0919F
:10E2E000D90EF091DA0E80916C1690916D16918393
:10E2F00080838091D90E9091DA0E029630C0809181
:10E30000B009E091AE09F091AF09E80FF11D8281EB
:10E31000806482832091D90E3091DA0EC901DC012C
:10E32000E6E6F6E188E001900D928150E1F78091F8
:10E33000D90E9091DA0E089612C08091D90E909164
:10E34000DA0E9C01D901EEE5F6E180E101900D9233
:10E350008150E1F78091D90E9091DA0E409690931A
:10E36000DA0E8093D90E80916E168F3F09F065C04A
:10E370008091701690917116892B09F050C0809190
:10E38000721690917316892B09F049C0809174160A
:10E3900090917516892B09F042C080917616909164
:10E3A0007716892BE1F58091781690917916892B53
:10E3B000B1F580917A1690917B16892B81F5809129
:10E3C0007C16882361F580917D168150823038F566
:10E3D0008091B009E091AE09F091AF09E80FF11D0D
:10E3E000828188608283E091D90EF091DA0E80EA12
:10E3F0008083E091D90EF091DA0E80916F1690E053
:10E400008F709070880F991F2081282B2083E091B6
:10E41000D90EF091DA0E80917D1681838AC08091A9
:10E42000D90E9091DA0E9C01D901EEE6F6E180E179
:10E4300001900D928150E1F7ADC08EE696E10E9409
:10E44000A96FDC019093D80E8093D70E009709F442
:10E4500094C08091B009E091AE09F091AF09E80F46
:10E46000F11D828111969C91892B828320917616D1
:10E4700030E08091BD1C90E08D7F2817390771F541
:10E48000909177168091BE1C981741F5809178166F
:10E49000882321F5809179168F3F01F580917A16B6
:10E4A0008E3FE1F480917B168823C1F4E12FF02F99
:10E4B00090917C168081981789F490917D168181C6
:10E4C000981761F48091B009E091AE09F091AF091D
:10E4D000E80FF11D82818C60828365C08091761681
:10E4E00090917716892B59F580917816909179162D
:10E4F000892B29F580917A1690917B16892BF9F456
:10E5000080917C1687FD1BC08091B009E091AE0917
:10E51000F091AF09E80FF11D828188608283E0915C
:10E52000D90EF091DA0E80917C1690917D16918330
:10E5300080838091D90E9091DA0E029630C080913E
:10E54000B009E091AE09F091AF09E80FF11D8281A9
:10E55000846082832091D90E3091DA0EC901DC01EA
:10E56000E6E7F6E188E001900D928150E1F78091B5
:10E57000D90E9091DA0E089612C08091D90E909122
:10E58000DA0E9C01D901EEE6F6E180E101900D92F0
:10E590008150E1F78091D90E9091DA0E40969093D8
:10E5A000DA0E8093D90E88E28093B20980915C16CE
:10E5B000813109F064C090917E1680917F16805B56
:10E5C000904F0F9770F5909180168091811620EFF3
:10E5D000803B920730F18F5B904F18F5E091D90E98
:10E5E000F091DA0E8BEF8083E091D90EF091DA0E84
:10E5F00090918116905B80917F168295807F980F15
:10E600009183E091D90EF091DA0E80918416909169
:10E610008516938382838091D90E9091DA0E0496A9
:10E6200025C0E091D90EF091DA0E88EF8083E09159
:10E63000D90EF091DA0E80917E1690917F16A091FE
:10E640008016B091811681839283A383B483E09175
:10E65000D90EF091DA0E80918416909185169683EA
:10E6600085838091D90E9091DA0E07969093DA0EF9
:10E670008093D90E8091B209885F8093B20980910E
:10E68000D90E9091AE09891B8093B0091F910F910B
:10E6900008950F931F93CF93DF93EC018B010E949A
:10E6A000A96F892B31F1288530E08091BD1C90E065
:10E6B0008D7F28173907E9F499858091BE1C98173A
:10E6C000C1F48A858823A9F48B858F3F91F48C85CA
:10E6D0008E3F79F48D85882361F49E85F8018081D1
:10E6E000981739F420E09F858181981719F421E06B
:10E6F00001C020E0822FDF91CF911F910F910895EB
:10E70000FC0190818181009769F040919B1C5091A0
:10E710009C1C60919D1C21E00E940D1210929E1C79
:10E7200010929D1C08950F931F93DF93CF9300D0F9
:10E73000CDB7DEB7FC011092B2091092B009109269
:10E740009E1C10929D1C80919B1C90919C1C9093F0
:10E75000AF098093AE09309709F580915C168A3332
:10E76000D1F48091FD06282F30E0F901E258F94EEE
:10E770008081873881F4F901EE57F94E82898983C7
:10E7800083898A83AEE6B6E1349680E101900D92EA
:10E790008150E1F707C019821A8204C08081898301
:10E7A00081818A838E010F5F1F4FC8010E94EB6F2A
:10E7B0008091B209482F50E0E091D915F091DA1517
:10E7C000E41BF50BA091B0092A2F30E08FE690E012
:10E7D000821B930B6091AE097091AF098E179F0752
:10E7E00008F0B4C0CB0104964A2F50E00E94B780D5
:10E7F000E091AE09F091AF098091D9159091DA15A9
:10E80000906C908381839091B70E8091B80E828333
:10E8100093838091B0098C5F8093B0094FE6481BC9
:10E82000487F4093B109E80FF11D2091B20930E013
:10E830002A5A394ECF01B90150E00E94AE80209192
:10E84000B0098091B10990E0820F911D90939E1CB8
:10E8500080939D1CC8010E9480732091B209809111
:10E86000B10990E0820F911D9093B60E8093B50E82
:10E8700085E08093B009E091AE09F091AF098091F5
:10E88000D9159091DA15906E9083818388E68093F4
:10E89000B10942C0A091AE09B091AF09CF0123E008
:10E8A000969587952A95E1F714968C9314979A017B
:10E8B0002E1B3F0B8091B10990E02817390720F4F7
:10E8C000842F8E1B8093B1098091B0099D01280F80
:10E8D000311D4091B109EA5AF94EC901BF0150E01A
:10E8E0000E94AE802091B0098091B10990E0820F22
:10E8F000911D90939E1C80939D1CC8010E94807363
:10E900002091B1098091B50E9091B60E820F911DA4
:10E910009093B60E8093B50EE091B50EF091B60EC1
:10E920004091D9155091DA15E417F50708F4B2CFE4
:10E930008091B70E9091B80E01969093B80E809387
:10E94000B70E1092B60E1092B50E1CC0260F371FD0
:10E950004A5A594EC901BA01AF010E94AE802091B6
:10E96000B0098091D9159091DA15820F911D2091EF
:10E97000B209821B910990939E1C80939D1CC80133
:10E980000E94807381E00F900F90CF91DF911F91D3
:10E990000F910895CF93DF932091E01CE22FF0E0D8
:10E9A000DF0124E0AA0FBB1F2A95E1F7A054B34E64
:10E9B000EC0180E109900D928150E1F784E0EE0FC7
:10E9C000FF1F8A95E1F7E054F34E8FEF8787DF91C1
:10E9D000CF910895FFCF0F931F93DF93CF93CDB7C0
:10E9E000DEB728970FB6F894DEBF0FBECDBF80917B
:10E9F000D9159091DA15009709F435C181509540E9
:10EA000008F022C180916E1690916F16892B59F5EE
:10EA10008091701690917116892B29F5809172164C
:10EA200090917316892BF9F4809174169091751654
:10EA3000892BC9F48091761690917716892B99F4D9
:10EA40008091781690917916892B69F480917A16C5
:10EA500090917B16892B39F480917C1690917D16CC
:10EA6000892B09F4F1C09091E01C913029F4809138
:10EA70000D05882309F4E8C080916E168F3F09F4D4
:10EA8000E8C0913041F48EE696E10E94FE4E882364
:10EA900011F41092E01C8EE696E10E94FE4E88234F
:10EAA00041F08EE696E10E94C84F8C01E0E0F0E074
:10EAB0000EC08091E01C813011F41092E01C0E9485
:10EAC000354BFC01009709F4BFC000811181809192
:10EAD000E01C813071F5EF2B01F52091761630E0C6
:10EAE0008091BD1C90E08D7F28173907B1F490917B
:10EAF00077168091BE1C981781F480917816882330
:10EB000061F4809179168F3F41F480917A168E3F9F
:10EB100021F480917B16882319F019821A8206C08D
:10EB200080917C16898380917D168A83CE0101961F
:10EB300089C00115110531F0F801818D853009F08A
:10EB400049C00AC08EE696E160E070E040E020E057
:10EB50000E9425508C0102C0F801118E8EE596E1CD
:10EB600060E840E00E949761892B19F08EE596E1FC
:10EB700002C080E090E060E070E0A8010E94405791
:10EB80008091E01C90E029E730E0829FF001839FB4
:10EB9000F00D929FF00D1124EB55F44E65857685AE
:10EBA0008785908928EE33E040E050E00E942D8375
:10EBB000CA01B90128EE33E040E050E00E94DB8258
:10EBC000AB01BC01C80182960E94506781E0F80148
:10EBD00082A73FC0882309F446C0823059F483E0FD
:10EBE000F801818FC8014A9648E853E160E070E07F
:10EBF0000E9450678091E01C90E029E730E0829FFE
:10EC0000F001839FF00D929FF00D1124EB55F44E0F
:10EC1000658576858785908928EE33E040E050E071
:10EC20000E942D83CA01B90128EE33E040E050E094
:10EC30000E94DB82AB01BC01C80182960E94506732
:10EC4000C80140960E9481661092DA151092D9157B
:10EC50000AC080E090E00E9481661092DA1510925E
:10EC6000D9151092FD0628960FB6F894DEBF0FBE98
:10EC7000CDBFCF91DF911F910F9108951F93DF9327
:10EC8000CF93CDB7DEB760970FB6F894DEBF0FBE57
:10EC9000CDBFDC016A30710518F01C9280E031C0F4
:10ECA000FB01E156F34E8081882311F41C9229C0A8
:10ECB0001091611CAE014F5F5F4F20E030E01130DA
:10ECC00019F4EBE1F0E002C0E0E0F0E0C901880FE8
:10ECD000991FE80FF91FEA5CF34E80819181FA01D8
:10ECE00081939193AF012F5F3F4F2730310539F763
:10ECF0007F87688BCD01BE016F5F7F4F0E94ED79EA
:10ED000081E060960FB6F894DEBF0FBECDBFCF9105
:10ED1000DF911F910895CF92DF92EF92FF920F93B0
:10ED20001F93DF93CF9300D0CDB7DEB71092E01CD6
:10ED30000EE616E18FEF92E090936F1680936E16B9
:10ED4000109271161092701610927316109272161D
:10ED500010927516109274161092771610927616FD
:10ED6000109279161092781610927B1610927A16DD
:10ED700080E092E090937D1680937C1698EEE92EC9
:10ED80009FEFF92EE00EF11E89E0D70197968C9344
:10ED9000C8014097B8010E94785F1092FD0680E696
:10EDA00080935616F70111821382128281E18683C5
:10EDB0002FEF278380E1C82ED12CC00ED11E82E018
:10EDC00099E0D60113969C938E93129790937F1699
:10EDD00080937E1680E094E315969C938E9314970F
:10EDE00017961C921E921697085E1F4F82E0809322
:10EDF000861681E0F801818313821282278B158A9F
:10EE0000148A168A8091E01C90E029E730E0829F06
:10EE1000A001839F500D929F500D1124FA01EB55D4
:10EE2000F44E82A98823B1F0D701D496FA01E354B5
:10EE3000F44E80E101900D928150E1F781E08093E2
:10EE4000E01C0E94AC4B1092E01CFC01B29681A128
:10EE500081FD05C01092DA151092D9152EC02EE949
:10EE600036E1AF0180E1DA010D90AD01D9010D92DB
:10EE70009D018150C1F78089F80182A711A610A6D3
:10EE800081E083A78CE590E09093DA158093D91503
:10EE900084E390E09A8389838A81D70114968C93C6
:10EEA0001497898115968C930E949A3E809590952F
:10EEB000F601978386830E94EB740F900F90CF9199
:10EEC000DF911F910F91FF90EF90DF90CF90089509
:10EED0000F93CF93DF930E94354B892BB9F5809127
:10EEE000E01CE82FF0E034E0EE0FFF1F3A95E1F769
:10EEF000E054F34E87858823D9F01786CF0160E46C
:10EF000020E030E040E050E001E00E94394D809187
:10EF1000E01C90E024E0880F991F2A95E1F78054C7
:10EF2000934E60E420E030E040E050E00E946963EE
:10EF30008091E01C882311F40E9480668091E01C7F
:10EF4000813021F481E59CE10E94FC6A8091E01C03
:10EF500090E0C9E7D0E08C9FF0018D9FF00D9C9F61
:10EF6000F00D1124EB55F44E83898823A1F00E9403
:10EF7000354B892B71F08091E01C90E08C9FF00163
:10EF80008D9FF00D9C9FF00D1124EB55F44E128ACD
:10EF9000118A0E9423618AE795E00E94920B80917A
:10EFA000E01C882319F486E895E007C0813019F445
:10EFB0008FE895E002C087E995E00E94920B8DE909
:10EFC00095E00E94920B0E94A664DF91CF910F9171
:10EFD00008958091E01C813059F48091611C8F3F2D
:10EFE000D9F081E59CE10E94FC6A0E949312089589
:10EFF0008091311C882381F48091611C8F3F61F4E2
:10F000008091E81B8F3F41F08091BA1B882321F04B
:10F0100088ED9BE10E94FC6A089580911F16882369
:10F0200059F08AEF95E19093F9158093F81582E0F5
:10F030000E945A3F0E94EB7480914B16882359F02E
:10F0400086E296E19093F9158093F81582E00E948C
:10F050005A3F0E94EB7408958091F1158830E9F4CD
:10F06000E091DC0EF091DD0E3097F9F02EED3EE0F0
:10F070008091DB159091DC15B901AF010E94AE8043
:10F080008091DC0E9091DD0E9093591B8093581B5C
:10F090001092DD0E1092DC0E0895823031F4109241
:10F0A000591B1092581B10924F0F0895FF920F9307
:10F0B0001F93DF93CF93CDB7DEB769970FB6F89460
:10F0C000DEBF0FBECDBFF82E092FE62F6237D0F579
:10F0D0001091611C1130B1F58091DC0E9091DD0E24
:10F0E000892B81F580914F0F882361F56093DC0EA9
:10F0F0001092DD0E2EED3EE0C901BA014E2F50E018
:10F100000E94AE801093E01C80EF93EB9A8B898B6A
:10F110009C8B8B8B80E48D8BDE011196E1E5FCE10D
:10F1200080E101900D928150E1F70F87F88ACE01BE
:10F1300001969093F5158093F41585E00E945A3F4F
:10F140000E94EB7469960FB6F894DEBF0FBECDBF78
:10F15000CF91DF911F910F91FF900895FC0120E066
:10F1600090818181808391832E5F32962031C1F717
:10F170000895992787FD90950E949A838833A1F17D
:10F18000893384F4843341F185333CF4823301F1D3
:10F19000833304F58133D1F417C0863309F1873303
:10F1A0000CF51CC0833641F184363CF4813601F104
:10F1B000823604F5893351F419C0853609F1853654
:10F1C000ECF0863619F41EC081E0089580E00895C1
:10F1D00082E0089583E0089584E0089585E008952D
:10F1E00086E0089587E0089588E0089589E008950D
:10F1F0008AE008958BE008958CE008958DE00895ED
:10F200008EE008958FE00895EF92FF921F93CF93C1
:10F21000DF937C01EC0110E001C01F5F888199271A
:10F2200087FD90950E948683892B19F4C0E0D0E079
:10F2300022C02196143089F7F9CFF70180810E940E
:10F24000B97890E0143029F4982F88279295907F10
:10F250000CC0133019F4982F882707C0123029F4F6
:10F2600024E0880F991F2A95E1F7C80FD91F115084
:10F270000894E11CF11C112301F7CE01DF91CF911D
:10F280001F91FF90EF9008955F926F927F928F92FF
:10F290009F92AF92BF92CF92DF92EF92FF920F9325
:10F2A0001F93DF93CF9300D000D00F92CDB7DEB77E
:10F2B0004C016B018C019C01A8E0EA2EFF24F8E0D0
:10F2C0005F2E5E010894A11CB11CE5E06E2E712C2E
:10F2D0006C0E7D1E02C00F5F1F4FF80140814A3344
:10F2E00011F04423C1F7C801821B930B059714F05A
:10F2F00080E05EC0F80182918F010F5F1F4F8A335B
:10F3000019F0D501F9012FC0442319F0F40190E060
:10F310000EC0EF2DF0E0EE0FFF1FEC0DFD1D118272
:10F320001082F39440C08A3309F49F5F3196808144
:10F330008823C9F7252D291B9F2D822F0AC0E92F6D
:10F34000F0E0EE0FFF1FEC0DFD1D118210828150C9
:10F350009F5F8823A1F7F20EE21A0F5F1F4F9801FB
:10F360001FC08D9331969E2F921B80818A3319F096
:10F37000A615B705B1F7F501E90FF11D1082C5011A
:10F380000E940479EF2DF0E0EE0FFF1FEC0DFD1D44
:10F390009183808398012F5F3F4FF394EA94890112
:10F3A000EE2009F09ACF80E0F8E0FF1609F481E042
:10F3B0000F900F900F900F900F90CF91DF911F91B2
:10F3C0000F91FF90EF90DF90CF90BF90AF909F9004
:10F3D0008F907F906F905F900895AF92BF92CF9281
:10F3E000DF92EF92FF920F931F93CF93DF938C01E5
:10F3F000EB016115710509F469C0EE24FF2435EBBA
:10F40000C32E35E0D32E20E3A22E9AE3B92E8881B5
:10F410009981009779F5EE2069F540E06F2D70E055
:10F4200001C04F5F242F30E0F901EE0FFF1FEC0FFA
:10F43000FD1F80819181892B29F4260F371F2830E9
:10F4400031057CF3413039F4D801AD928D01F3944C
:10F45000229640E02EC08F2D90E0840F911D0897DA
:10F4600009F44150842F90E0880F991FC80FD91FCD
:10F47000F40E1FC000D000D000D0EDB7FEB731961B
:10F48000ADB7BEB712961C930E931197D382C2826A
:10F49000948385830E943C81080F191F2296F39460
:10F4A0004E2DEDB7FEB736960FB6F894FEBF0FBEE1
:10F4B000EDBFF8E0FF1641F0D801BD928D01B7E035
:10F4C000BF1510F0E42EA3CFF8011082DF91CF9189
:10F4D0001F910F91FF90EF90DF90CF90BF90AF9072
:10F4E0000895AF92BF92CF92DF92EF92FF920F9367
:10F4F0001F93DF93CF9300D000D000D0CDB7DEB7FD
:10F500007C0188EB95E00E94920B00E010E06E0118
:10F510000894C11CD11C4AEBA42E45E0B42E00D0A7
:10F5200000D000D0EDB7FEB73196ADB7BEB712969A
:10F53000DC92CE921197B382A282D701A00FB11FA5
:10F540008C91848315820E943C818DB79EB706966C
:10F550000FB6F8949EBF0FBE8DBFC6010E94920BDE
:10F560000F5F1F4F00311105D1F626960FB6F894A4
:10F57000DEBF0FBECDBFCF91DF911F910F91FF90E6
:10F58000EF90DF90CF90BF90AF900895CF92DF9231
:10F59000EF92FF920F931F93CF93DF938C017B0128
:10F5A000EA0169018881882319F020E030E002C077
:10F5B00029813A81C9010197099740F4F901E1567F
:10F5C000F34E81E08083C9010E94C02380910D0524
:10F5D000882339F4C801B701AE0196010E943D7D30
:10F5E00005C0C801B70141E00E94377BDF91CF9190
:10F5F0001F910F91FF90EF90DF90CF9008950F93A0
:10F600001F93CF93DF93EC018B0180910D0588232D
:10F6100019F4CE010E94A27C8881833319F4898178
:10F62000833389F020E030E0FE01E20FF31FD901BF
:10F63000AF51BA4E90818C919817A1F42F5F3F4F34
:10F640002630310589F78C859D8586589D4D51F46E
:10F650001092E01C0E501040CE010E96B80140E012
:10F660000E94377BDF91CF911F910F9108951F93D7
:10F67000CF93DF939C01EB01142F8091D9159091CA
:10F68000DA15892B19F02FEF3FEF13C086E596E1CD
:10F69000B901AE010E94B7801093E01CD093DA1537
:10F6A000C093D91581E00E945A3F0E94EB7420E07C
:10F6B00030E0C901DF91CF911F910895FC0171A73E
:10F6C00060A70895FC01768B658B0895A091F815CD
:10F6D000B091F915109719F0FD01B89605C0E091A9
:10F6E000F415F091F51575968091F11586FF22C0FD
:10F6F00050962D913C9151978091520F9091530FBC
:10F700008217930731F48091540F9091550F009711
:10F7100069F48091560F9091570F8217930751F417
:10F720008091580F9091590F009721F09183808319
:10F7300013821282208131812115310521F08281CD
:10F740009381F90109950895009749F09093F9156F
:10F750008093F81583E00E945A3F0E94EB7408954D
:10F76000009749F09093F5158093F41585E00E9479
:10F770005A3F0E94EB740895CF93DF93EC01809180
:10F78000540F9091550F8C179D0771F48091520F73
:10F790009091530F0E94843D1092530F1092520F7C
:10F7A0001092550F1092540F8091580F9091590F4D
:10F7B0008C179D0771F48091560F9091570F0E94FE
:10F7C000843D1092570F1092560F1092590F1092BD
:10F7D000580FEFE1F6E1838194818C179D0719F4AE
:10F7E000148213821082BC96CF0185978255964170
:10F7F00090F3EAE5FBE1858996898C179D0711F462
:10F80000118A108A79968BE1EC38F807A0F3DF9122
:10F81000CF910895AC011092510FE2E5FFE020E096
:10F8200014C0808191818417950769F48281938146
:10F830008617970741F42093510F11821082CA0155
:10F840000E94843D089534962F5F223050F3209318
:10F85000510F0895CF93DF93EA010E94A148FC0164
:10F86000009711F0D68BC58BCF01DF91CF91089512
:10F870000F931F93DF93CF93CDB7DEB760970FB68B
:10F88000F894DEBF0FBECDBF8C01AB018FEF92E0CD
:10F890009A8389831C821B821E821D8218861F8286
:10F8A0001A8619861C861B861E861D8680E091E0BE
:10F8B000988B8F87CE010196B8010E942A7CFC01AB
:10F8C000009711F0118B008BCF0160960FB6F89462
:10F8D000DEBF0FBECDBFCF91DF911F910F91089575
:10F8E000AC011092500FE2E5FFE020E012C0322F91
:10F8F0003F5F80819181892B51F42093500F518378
:10F90000408373836283CA010E94A13D08953496A7
:10F91000232F223060F32093500F08950F931F93ED
:10F92000CF93DF938A010E94DA3DEC01009721F02A
:10F9300019A708A70E94A47BCE01DF91CF911F9148
:10F940000F910895CF92DF92EF92FF920F931F9342
:10F95000DF93CF93CDB7DEB766970FB6F894DEBFCF
:10F960000FBECDBF8C01FC012081233381F4818146
:10F97000833369F48281882331F480915E0F898317
:10F9800080915D0F2DC08F3F11F4F80112C080915E
:10F99000BD1C8C708260281781F4F80191818091E0
:10F9A000BE1C981751F48281882339F483818823FF
:10F9B00021F484818983858113C0F80182818823A1
:10F9C00009F04CC08381882309F048C084818823D2
:10F9D00009F044C08581882309F040C029838181D2
:10F9E0008A83F8018485958586589D4DB9F5DE0199
:10F9F0001996E6E5F6E18EE001900D928150E1F76F
:10FA000092EFE92E9FEFF92EE60EF71EF092DA152F
:10FA1000E092D9158EE0C82ED12CC00ED11E86E5FD
:10FA200096E1B601A7010E94B780CE0101960E941F
:10FA3000937326E10635120769F4C601B801A701E0
:10FA40000E94B780D801FE0139968EE001900D9298
:10FA50008150E1F71092DA151092D91566960FB61B
:10FA6000F894DEBF0FBECDBFCF91DF911F910F91F4
:10FA7000FF90EF90DF90CF900895EF92FF920F9359
:10FA80001F93CF93DF939C018B017A0186E596E16A
:10FA9000B901A8010E94B7801092E01C80916E16F7
:10FAA0008F3F09F4B4C08EE696E10E94FE4E882393
:10FAB00031F08EE696E10E94C84FEC0108C00E942A
:10FAC000354BFC01009709F4F5C0C081D181209726
:10FAD00029F0898D853009F047C00AC08EE696E18D
:10FAE00060E070E040E020E00E942550EC0101C0A1
:10FAF000198E8EE596E160E840E00E949761892BBF
:10FB000019F08EE596E102C080E090E060E070E0E0
:10FB1000AE010E9440578091E01C90E029E730E060
:10FB2000829FF001839FF00D929FF00D1124EB5501
:10FB3000F44E658576858785908928EE33E040E030
:10FB400050E00E942D83CA01B90128EE33E040E065
:10FB500050E00E94DB82AB01BC01CE0182960E9484
:10FB6000506781E08AA75AC0882309F4A3C0823075
:10FB700051F483E0898FCE014A9648E853E160E072
:10FB800070E00E9450678091E01C90E029E730E02F
:10FB9000829FF001839FF00D929FF00D1124EB5591
:10FBA000F44E658576858785908928EE33E040E0C0
:10FBB00050E00E942D83CA01B90128EE33E040E0F5
:10FBC00050E00E94DB82AB01BC01CE0182960E9414
:10FBD000506784E696E166E576E1A8010E94B78069
:10FBE00080917C168F3FD1F0888980935616898941
:10FBF000809357168A89809358168B89809359165B
:10FC00008C8980935A168D8980935B1607C084E691
:10FC100096E166E576E1A8010E94B78080917C16A6
:10FC20008F3FE9F483E380935616809357168091B3
:10FC30008816809358168091891680935916809162
:10FC40008A1680935A1680918B1680935B16ACE5CA
:10FC5000BFE0F70189E001900D928150E1F78091BA
:10FC6000BD1C8C70826080935C168091BE1C80935A
:10FC70005D1610925E1610925F16F70182818093D6
:10FC8000601681818093611686E8809362168DEDFF
:10FC900080936316B801625F7F4F7093DA156093AB
:10FCA000D91586E596E141E00E9490351092DA156B
:10FCB0001092D915DF91CF911F910F91FF90EF9086
:10FCC0000895ABE0B0E0E7E6FEE70C9453835C01F7
:10FCD0004B017A01FC0117821682838181FD08C0E5
:10FCE0006FEF7FEF08C142E050E0E40EF51E04C064
:10FCF0003E010894611C711CF501D380F401D3FC12
:10FD00008591D3FE81914F01882309F4F1C085329A
:10FD100059F4D3FC6591D3FE61914F01653219F01E
:10FD2000062F10E01BC085E290E02BC0002309F4F1
:10FD3000DFC08EE399E0602F70E00E948780892BFE
:10FD400039F4033211F4106103C00C3661F4106809
:10FD5000F401D3FC0591D3FE01914F0117FFE6CFCB
:10FD6000002309F4C5C087E399E0602F70E00E948A
:10FD70008780892B51F044E050E0E40EF51E8FE3BC
:10FD800090E0B5010E941081B7CF033629F0033708
:10FD900079F00335F1F40BC087010E5F1F4FF701B7
:10FDA00080819181B5010E9410817801A5CF1160F9
:10FDB000F701C080D18004C090E0B5010E9410819D
:10FDC000F60110FD859110FF81916F018823A1F745
:10FDD0008ACF043611F0093639F517FF08C0F7014C
:10FDE000208131814281538184E090E00AC0F70193
:10FDF000808191819C01442737FD4095542F82E0FA
:10FE000090E0E80EF91E1F7E57FF08C05095409500
:10FE1000309521953F4F4F4F5F4F1064CA01B90194
:10FE2000A3012AE030E034C00037A9F0013730F4F4
:10FE30000835B1F00F3609F05BC006C0053739F060
:10FE4000083709F055C008C028E030E00CC01F7E1C
:10FE50002AE030E008C01061146220E130E003C005
:10FE6000146020E132E017FF08C0F7016081718162
:10FE70008281938144E050E008C0F7018081918144
:10FE8000BC0180E090E042E050E0E40EF51EA301EA
:10FE90000E946081D82ED618012F10E006FF05C001
:10FEA0008DE290E0B5010E94108104FF15C0FE01B3
:10FEB000ED0DF11D8081803379F080E390E0B50194
:10FEC0000E94108102FF08C000721070C801885A99
:10FED0009F4FB5010E941081DA94F301ED0DF11DE1
:10FEE000808190E0B5010E941081DD20A9F704CF48
:10FEF000F50166817781CB012B96EEE00C946F8340
:10FF0000EF92FF920F93DF93CF93CDB7DEB7609759
:10FF10000FB6F894DEBF0FBECDBFA82F002309F4A3
:10FF200061C07E010894E11CF11C88E0F701119288
:10FF30008A95E9F729833A834B835C836D837E83BB
:10FF4000AF83988780E2801BE82FFF27E7FDF095BD
:10FF50004D815E816F817885181684F01D861E861E
:10FF60001F86188A882799278E1B9F0B04C07695B9
:10FF70006795579547958A95D2F728C0202F332744
:10FF800027FD3095DB01CA01022E04C0B695A79566
:10FF9000979587950A94D2F78D879E87AF87B88B00
:10FFA00004C0440F551F661F771FEA95D2F7898159
:10FFB0009A81AB81BC8104C0B695A795979587952A
:10FFC0002A95D2F7482B592B6A2B7B2B49875A87C6
:10FFD0006B877C8729853A854B855C856D857E8519
:10FFE000AF8598898A2F60960FB6F894DEBF0FBE52
:10FFF000CDBFCF91DF910F91FF90EF900895A0E0DA
:020000021000EC
:10000000B0E0E5E0F0E80C945783EC01A880B980FB
:10001000CA80DB80A114B104C104D10441F484E29C
:10002000A82E89EDB82E8BE5C82E87E0D82EC60104
:10003000B5012DE133EF41E050E00E94A28327EAB1
:1000400031E440E050E00E94DB827B018C01C6017C
:10005000B5012DE133EF41E050E00E94A283CA01D7
:10006000B9012CEE34EF4FEF5FEF0E94DB826E0D93
:100070007F1D801F911F97FF04C06150704080401A
:100080009048688379838A839B839B013F77C9016A
:10009000CDB7DEB7EAE00C9473830E94FF7F08952A
:1000A00081EC95E00E94FF7F0895A0E0B0E080938E
:1000B000C1059093C205A093C305B093C4050895EC
:1000C000FC0188279927E89421912032E9F329300F
:1000D00010F02E30C8F32B3241F02D3239F46894F1
:1000E00004C00E940881820F911D219120532A3063
:1000F000C0F31EF4909581959F4F0895FB01DC019C
:1001000002C005900D9241505040D8F70895FC016F
:100110000590061621F00020D9F7C0010895319707
:10012000CF010895FB01DC014150504048F005909B
:100130000D920020C9F701C01D9241505040E0F7D8
:100140000895FB01DC0104C08D910190801921F418
:1001500041505040C8F7881B990B0895FB01DC0102
:1001600002C001900D9241505040D8F70895681791
:10017000790768F4FB01DC01E40FF51FA40FB51F3C
:1001800002C002900E9241505040D8F708950C944E
:10019000AE80DC0101C06D9341505040E0F70895FE
:1001A000A0E0B0E0E6EDF0E80C9459837C01EB01AF
:1001B0008A01690109C0CE012196F6010995F7016E
:1001C00081937F010150104001151105A1F7CDB7B2
:1001D000DEB7E8E00C947583A0E0B0E0E2EFF0E871
:1001E0000C945983EC017B018A01690109C0CE019D
:1001F0002196F70161917F01F601099501501040A8
:1002000001151105A1F7CDB7DEB7E8E00C947583B1
:100210007AE0979F902D879F802D910D112408954E
:100220000F931F93CF93DF938C01EB018B8181FFA1
:100230001BC082FF0DC02E813F818C819D812817BC
:10024000390764F4E881F9810193F983E88306C0F2
:10025000E885F985802F0995892B31F48E819F815E
:1002600001969F838E8302C00FEF1FEFC801DF91BD
:10027000CF911F910F910895AEE0B0E0E2E4F1E874
:100280000C945D830D891E8986E08C831A83098313
:100290008FEF9FE79E838D839E01275E3F4FCE01A8
:1002A00001966F89788DA9010E94617E2F81388522
:1002B000020F131FF80110822E96E4E00C9479834C
:1002C000FA01AA27283051F1203181F1E8946F9387
:1002D0006E7F6E5F7F4F8F4F9F4FAF4FB1E03ED02D
:1002E000B4E03CD0670F781F891F9A1FA11D680FCB
:1002F000791F8A1F911DA11D6A0F711D811D911DFE
:10030000A11D20D009F468943F912AE0269F112472
:100310003019305D3193DEF6CF010895462F4770D6
:10032000405D4193B3E00FD0C9F7F6CF462F4F7031
:10033000405D4A3318F0495D31FD4052419302D08F
:10034000A9F7EACFB4E0A695979587957795679535
:10035000BA95C9F700976105710508959B01AC0135
:100360000A2E06945795479537952795BA95C9F75C
:10037000620F731F841F951FA01D089570D088F011
:100380009F5790F0B92F9927B751A0F0D1F0660F81
:10039000771F881F991F1AF0BA95C9F712C0B1309C
:1003A00081F077D0B1E0089574C0672F782F882747
:1003B000B85F39F0B93FCCF3869577956795B395DB
:1003C000D9F73EF490958095709561957F4F8F4F4A
:1003D0009F4F0895E89409C097FB3EF4909580954F
:1003E000709561957F4F8F4F9F4F9923A9F0F92FFB
:1003F00096E9BB279395F695879577956795B79579
:10040000F111F8CFFAF4BB0F11F460FF1BC06F5F5E
:100410007F4F8F4F9F4F16C0882311F096E911C070
:10042000772321F09EE8872F762F05C0662371F091
:1004300096E8862F70E060E02AF09A95660F771FA5
:10044000881FDAF7880F9695879597F9089557FDD5
:100450009058440F551F59F05F3F71F04795880F32
:1004600097FB991F61F09F3F79F0879508951216C9
:1004700013061406551FF2CF4695F1DF08C0161675
:1004800017061806991FF1CF869571056105089426
:100490000895E894BB2766277727CB0197F908953D
:1004A0000BD078C069D028F06ED018F0952309F0F1
:1004B0005AC05FC01124EECFCADFA0F3959FD1F3DD
:1004C000950F50E0551F629FF001729FBB27F00D02
:1004D000B11D639FAA27F00DB11DAA1F649F662757
:1004E000B00DA11D661F829F2227B00DA11D621FA6
:1004F000739FB00DA11D621F839FA00D611D221F60
:10050000749F3327A00D611D231F849F600D211D43
:10051000822F762F6A2F11249F5750408AF0E1F0E6
:1005200088234AF0EE0FFF1FBB1F661F771F881F2F
:1005300091505040A9F79E3F510570F014C0AACFCA
:100540005F3FECF3983EDCF3869577956795B7951A
:10055000F795E7959F5FC1F7FE2B880F911D969544
:10056000879597F9089597F99F6780E870E060E0B4
:1005700008959FEF80EC089500240A94161617063C
:1005800018060906089500240A9412161306140684
:1005900005060895092E0394000C11F4882352F0E7
:1005A000BB0F40F4BF2B11F460FF04C06F5F7F4F9F
:1005B0008F4F9F4F0895629FD001739FF001829FDC
:1005C000E00DF11D649FE00DF11D929FF00D839FE2
:1005D000F00D749FF00D659FF00D9927729FB00D7F
:1005E000E11DF91F639FB00DE11DF91FBD01CF0192
:1005F00011240895991B79E004C0991F961708F0FB
:10060000961B881F7A95C9F780950895AA1BBB1B76
:1006100051E107C0AA1FBB1FA617B70710F0A61B02
:10062000B70B881F991F5A95A9F780959095BC0123
:10063000CD01089597FB092E07260AD077FD04D037
:10064000E5DF06D000201AF4709561957F4F08957C
:10065000F6F7909581959F4F0895A1E21A2EAA1B57
:10066000BB1BFD010DC0AA1FBB1FEE1FFF1FA21762
:10067000B307E407F50720F0A21BB30BE40BF50B5F
:10068000661F771F881F991F1A9469F760957095E8
:10069000809590959B01AC01BD01CF0108952F92EB
:1006A0003F924F925F926F927F928F929F92AF9202
:1006B000BF92CF92DF92EF92FF920F931F93CF934F
:1006C000DF93CDB7DEB7CA1BDB0B0FB6F894DEBFE6
:1006D0000FBECDBF09942A88398848885F846E840C
:1006E0007D848C849B84AA84B984C884DF80EE8056
:1006F000FD800C811B81AA81B981CE0FD11D0FB65F
:10070000F894DEBF0FBECDBFED010895911106C074
:1007100080538A5010F0865C06C008959927882778
:10072000089585FDFBCF80629111F8CF81568A51E3
:10073000E0F708959111089581548A5108F4805E7C
:10074000855A089597FB092E05260ED057FD04D033
:1007500084DF0AD0001C38F45095409530952195DF
:100760003F4F4F4F5F4F0895F6F7909580957095E6
:0A07700061957F4F8F4F9F4F089552
:10077A0080E803252D313573202D2025303258206D
:10078A00000D0A002564000D0A73686F7274203D1B
:10079A0020253034580D0A706172656E74203D2030
:1007AA00253034580D0A726F7574653D25303458FA
:1007BA000D0A006368616E203D2025640D0A00253C
:1007CA0078006C6F6E67203D2030782530386C5881
:1007DA002530386C580D0A0066616C7365007472B6
:1007EA007565006173736F63203D2025730D0A4898
:1007FA006F7073203D20253034580D0A0072616EE7
:10080A0064203D20253032580D0A0025752C2052CF
:10081A0065763D25640D0A00536C656570203D20A0
:10082A0025730D0A005965730046726571203D20D3
:10083A0025644D487A0D0A00364C6F5750414E20B8
:10084A003D2025730D0A0044656D6F206D6F646548
:10085A00203D2025730D0A004E6F005452585F53F5
:10086A0054415455530000000000005452585F533D
:10087A0054415445000000000000005452585F43A0
:10088A0054524C5F300000000000005452585F433D
:10089A0054524C5F310000000000005048595F5428
:1008AA00585F5057520000000000005048595F52EC
:1008BA0053534900000000000000005048595F45AA
:1008CA00445F4C4556454C000000005048595F4370
:1008DA00435F4343410000000000004343415F542B
:1008EA0048524553000000000000005452585F432C
:1008FA0054524C5F320000000000004952515F4DD3
:10090A0041534B00000000000000004952515F5360
:10091A005441545553000000000000565245475FA9
:10092A004354524C000000000000004241544D4F15
:10093A004E00000000000000000000584F53435FC3
:10094A004354524C0000000000000052585F5359B3
:10095A004E0000000000000000000052465F4354B1
:10096A00524C5F30000000000000005841485F43CD
:10097A0054524C5F3100000000000046544E5F4361
:10098A0054524C000000000000000052465F4354DD
:10099A00524C5F3100000000000000504C4C5F4395
:1009AA004600000000000000000000504C4C5F446C
:1009BA004355000000000000000000504152545FFF
:1009CA004E554D00000000000000005645525349A4
:1009DA004F4E5F4E554D00000000004D414E5F499D
:1009EA00445F3000000000000000004D414E5F49A6
:1009FA00445F31000000000000000053484F525489
:100A0A005F414444525F300000000053484F525443
:100A1A005F414444525F310000000050414E5F493B
:100A2A00445F30000000000000000050414E5F4962
:100A3A00445F310000000000000000494545455F61
:100A4A00414444525F300000000000494545455F7B
:100A5A00414444525F310000000000494545455F6A
:100A6A00414444525F320000000000494545455F59
:100A7A00414444525F330000000000494545455F48
:100A8A00414444525F340000000000494545455F37
:100A9A00414444525F350000000000494545455F26
:100AAA00414444525F360000000000494545455F15
:100ABA00414444525F3700000000005841485F43F8
:100ACA0054524C5F3000000000000043534D415F18
:100ADA00534545445F30000000000043534D415FD9
:100AEA00534545445F31000000000043534D415FC8
:100AFA004245000000000000000000010203040556
:100B0A00060708090C0E0F10111215161718161AD7
:100B1A001B1C1D1E1F202122232425262728292AA3
:100B2A002B2C2D2E2F256325303258202563253076
:100B3A00325820253032582030782530386C5825E4
:100B4A0030386C580D0A002563253032582000438E
:100B5A004352450025780030782530386C582530C6
:100B6A00386C58202020202530345820202020207E
:100B7A0020200025640014000F000100000101007C
:100B8A002603000000000000000000000000000032
:100B9A00000000000000000000000000000000004B
:100BAA0000000000000030782530386C58253038B5
:100BBA006C5800AAABACADAEAF3A3B3C3D3E3F01F0
:100BCA002383927834200000ADBA202020256420A7
:100BDA000909202020256409090020010470F13C3C
:100BEA0001000000000000000000525320446F6E14
:100BFA0065206F6E200045746865726E65740036F4
:100C0A004C6F7750414E004F74686572002C20413A
:100C1A00737369676E656420616464726573736572
:100C2A00733A0D0A00257800200025303278000634
:060C3A00020100000000B1
:10FC00002F923F924F925F926F927F928F929F922C
:10FC1000AF92BF92CF92DF92EF92FF920F931F931A
:10FC2000DF93CF9300D000D0CDB7DEB7F8948091AA
:10FC3000971390919813A0919913B0919A13898377
:10FC40009A83AB83BC83612C712C91E0892E912C1B
:10FC500071E065E052C0F999FECF93E0F101409266
:10FC60005B0090935700E89507B600FCFDCFA1E13B
:10FC7000A0935700E89507B606FCFDCF6401530139
:10FC8000EE24FF248701CBBEF501279137914791E0
:10FC90005691D801C701820D931DA41DB51D090100
:10FCA000FC01A0935B0070935700E895112482E05B
:10FCB00090E0A0E0B0E0A80EB91ECA1EDB1EE80E60
:10FCC000F91E0A1F1B1F90E0E91691E0F90690E06B
:10FCD000090790E01907B9F680E091E0A0E0B0E0F4
:10FCE000680E791E8A1E9B1EF10140925B00609394
:10FCF0005700E89507B600FCFDCF212C312C8FEF83
:10FD0000482E8FEF582E260C371C481C591C898111
:10FD10009A81AB81BC81681679068A069B0608F435
:10FD20009ACF81E180935700E8952BE088E190E03D
:10FD30000FB6F894A895809360000FBE20936000E2
:10FD4000FFCFAF92BF92CF92DF92EF92FF920F93CD
:10FD50001F93CF93DF937B018C016A01AFB6F894B8
:10FD6000F999FECF83E0F70100935B008093570081
:10FD7000E89507B600FCFDCF40E050E060E070E0A1
:10FD8000BB24B394F6018081D181C0E09E01280F8D
:10FD9000311D82E090E0C80ED91EDB01CA018E0D34
:10FDA0009F1DA01FB11F0901FC01A0935B00B09231
:10FDB0005700E89511244E5F5F4F6F4F7F4F4030E3
:10FDC00091E0590790E0690790E07907D9F685E05E
:10FDD000F70100935B0080935700E89507B600FC9D
:10FDE000FDCF81E180935700E895AFBEDF91CF91C1
:10FDF0001F910F91FF90EF90DF90CF90BF90AF9049
:02FE0000089563
:00000001FF
